:020000040800F2
:1080000090EC0020A1810008A981000815AB0008B0
:10801000AD810008AF810008B181000800000000B8
:10802000000000000000000000000000B381000814
:10803000B581000800000000B7810008B981000880
:10804000BB810008BB810008BB810008BB81000820
:10805000BB810008BB810008A59D0008B59D0008F4
:10806000BB810008BB810008BB810008BB81000800
:10807000BB810008BB810008379900083F990008C0
:10808000BB81000847990008BB810008BB8100083C
:10809000BB810008BB810008BB810008BB810008D0
:1080A000BB810008BB810008BB810008BB810008C0
:1080B00071280308BB810008BB810008BB81000850
:1080C000BB810008BB810008BB810008BB810008A0
:1080D000BB810008533803085B3803086338030882
:1080E000AD9D0008BB810008BB810008BB81000872
:1080F000BB810008BB810008BB8100084F990008C4
:10810000BB810008BB810008BB810008BB8100085F
:10811000433803084B380308BB810008BB810008C3
:10812000BB810008BB810008BB810008BB8100083F
:10813000BB810008BB810008BB810008BB8100082F
:10814000BB810008BB810008BB810008BB8100081F
:10815000BB810008579900085F9900086B38030835
:10816000BB810008BB810008BB810008BB810008FF
:10817000BB810008BB810008BB810008BB810008EF
:10818000BB810008BB810008DFF810D000F058FC6C
:1081900000480047B1560308AFF3008090EC002080
:1081A0000648804706480047FEE7FEE7FEE7FEE791
:1081B000FEE7FEE7FEE7FEE7FEE7FEE70928030825
:1081C000898100082DE9F0410024061B254671F144
:1081D000000605DA01240027D0EB070067EB010158
:1081E000161E73F1000605DA0027D2EB07020125FF
:1081F00067EB030300F0C1FA86460E4617469C461D
:10820000AC4204D00025D0EB050E65EB010624B18D
:108210000020D2EB000760EB030C704631463A4673
:108220006346BDE8F081202A06DBCB17203A41FAED
:1082300002F043EAE07306E041FA02F3D040C2F1F3
:108240002002914008431946704740EA01039B070A
:1082500003D009E008C9121F08C0042AFAD203E0BB
:1082600011F8013B00F8013B521EF9D27047421E43
:1082700012F8013F002BFBD111F8013B02F8013B42
:10828000002BF9D17047421C10F8011B0029FBD1CB
:10829000801A704730B505460020034600E05B1C9D
:1082A000934205D2EC5CC85C201A01D1002CF6D1B7
:1082B00030BD2DE9FE4F804681EA0300C00F0C4619
:1082C000009021F0004123F00045B8EB0200A941E5
:1082D00005D24046214690461C460B46024623F0F6
:1082E0000040104347D0270DC7F30A00C3F30A51DB
:1082F0000290401A019040286BDAC3F3130040F457
:10830000801B0098924620B10023D2EB030A63EB56
:108310000B0B01985946C0F14002504600F05EFA3E
:1083200006460D4650465946019AFFF77CFF10EB72
:1083300008006141002487EA115284EAE7731A4376
:1083400040D0009A62B3019A012A4FEA075215DC25
:10835000001B61EB02014FF0004202EA0752CDE937
:108360000042001C41F5801132462B4600F0EAFA2B
:1083700003B0BDE8F08F40462146F9E7001B61EBF2
:108380000201001C41F5801300185B412018A2F582
:10839000001747EB030140EAD570B6196D4111E0B3
:1083A0006D084FEA360645EAC0754FEA0752001BD2
:1083B00061EB0201001C41F5801149084FEA3000D1
:1083C0000019514132462B4603B0BDE8F04F00F092
:1083D000AABA0098012240000023D0EB020263EB0E
:1083E000E073009821464FEAE074B8EB000061EBBF
:1083F0000401E9E783F000435BE781F0004158E7BF
:108400002DE9FE4F81EA030404F0004421F000410D
:1084100000944FF0000B23F0004350EA01045ED0BB
:1084200052EA03045BD0C3F30A54C1F30A552C4447
:10843000A4F2F3340194A0FB0254C1F3130141F4FC
:108440008011C3F3130343F4801301FB024400FBC8
:10845000034E840A970A44EA815447EA8357A4FBEF
:10846000076802958D0A05FB07854FEA932C04FBEC
:108470000C542705029D4FEA065847EA1637B5EB1C
:1084800008056EEB070C870E920E47EA811742EA49
:108490008312A7FB0201B6EB0B0164EB00042B0D6A
:1084A00043EA0C335E1844EB1C50DA465146E7FBB6
:1084B0000201C5F313044FEA0B3343EA14534FEAA6
:1084C0000432019C43EA0603A4F10C040294009CCC
:1084D000CDE900B400F036FA03B0BDE8F08F00201B
:1084E0000146F9E72DE9F04D81EA030404F0004B61
:1084F00021F0004514464FF0000A23F0004150EAF5
:10850000050220D054EA01021DD0C5F30A570246E5
:10851000C5F31303C1F31300C1F30A5640F48015E9
:1085200043F48013A7EB0608101BD64608F2FD386B
:1085300073EB050002D308F1010801E092185B41DA
:10854000B8F1000F03DA00200146BDE8F08D0020ED
:108550004FF48011064684460EE0171B73EB0507A7
:1085600005D3121B63EB050306434CEA010C4908D3
:108570004FEA300092185B4150EA0107EDD152EA10
:10858000030012D082EA040083EA0501084305D003
:10859000101BAB4106D20122002306E000224FF05F
:1085A000004302E06FF0010253101AEB06004CEB9F
:1085B000085110EB0A0041EB0B01BDE8F04D00F053
:1085C000B2B9F0B4CA17CB0F50405140C61841F1B0
:1085D00000054FEAC372314628004FF0960303D0DE
:1085E000B623F0BC00F071B930460021F9E70EB5B2
:1085F000C10F80EAE0700844CA07002140F233430B
:108600008DE80E000A460B4600F09CF903B000BD51
:108610000EB540F2334102910021CDE900110A4626
:108620000B4600F08FF903B000BD3EB5CA17CB0F63
:10863000002450405140C0186141DA0740F23343F2
:108640000094CDE901232246234600F07BF903B0D4
:1086500030BD10B500F0004420F00040C20DC0F362
:10866000160040F400007F2A02DA0020014610BD07
:108670000021962A03DCC2F19602D04002E0963A2D
:1086800000F0ACF8002CF2D00023D0EB030063EB39
:10869000010110BD70B5C1F30A5201F0004500247C
:1086A000C1F3130140F2FF3341F480119A4201DA21
:1086B000002070BD40F233439A42A2F2334203DC01
:1086C000524200F09AF800E090402C43F1D0404232
:1086D00070BD70B5C1F30A5201F000450024C1F32A
:1086E000130140F2FF3341F480119A4202DA002074
:1086F000014670BD40F233439A42A2F2334203DC9A
:10870000524200F07AF801E000F068F82C43F0D013
:108710000023D0EB030063EB010170BD00F00042C9
:1087200030F000400AD0C10D01F56071C0F31600B1
:1087300042EA0151C2084007114370470020014638
:10874000704701F0004330B421F0004150EA0102CB
:1087500006D00A0DA2F56072C1F31301002A02DCF3
:1087600030BC00207047440F44EAC104C100E01847
:1087700030BC00EBC25000F09FB82DE9F05F054619
:10878000002092469B4688460646814640241BE0D0
:10879000284641464746224600F02FF853465A469F
:1087A000C01A914110D311461846224600F016F81F
:1087B0002D1A67EB01084F4622460120002100F0E8
:1087C0000DF817EB00094E41201EA4F10104DFDC77
:1087D000484631462A464346BDE8F09F202A04DB3E
:1087E000203A00FA02F1002070479140C2F12003C4
:1087F00020FA03F3194390407047202A04DB203A03
:1088000021FA02F00021704721FA02F3D040C2F1B0
:108810002002914008431946704700000FB400231E
:1088200000B589B00CA900910B996FF00042CB60A4
:108830001E4B06931E4B07930423CDE901321D4ABC
:10884000089202466B46002000F0A6F909B05DF8D8
:1088500014FB70B586B006464FF0FF300091CDE9AD
:108860000101002015460C4604903246694604A8D2
:10887000FFF7D4FF02460498211825B108B1084635
:1088800000E020462860049800280DD0002A02DD70
:108890000098884208D0081B0094CDE901043246B4
:1088A000694604A8FFF7BAFF06B070BDD18D000875
:1088B000EF8D0008658A00080029A8BF7047401C9A
:1088C000490008BF20F00100704710B4B0FA80FCE6
:1088D00000FA0CF050EA010404BF10BC704749B123
:1088E000CCF1200421FA04F411FA0CF118BF012193
:1088F00021430843A3EB0C01CB1D4FEA00614FEA73
:10890000102042BF002010BC704700EBC350104441
:108910000029A4BF10BC7047401C490008BF20F0CC
:10892000010010BC704710B5141E73F1000408DA82
:10893000401C41F1000192185B411A4301D120F023
:10894000010010BD2DE9F04D92469B4611B1B1FAE0
:1089500081F202E0B0FA80F220329046FFF73EFF4B
:1089600004460F4640EA0A0041EA0B0153465A46C4
:10897000084313D0114653EA010019D0C8F1400250
:108980005046FFF73AFF05460E46504659464246C6
:10899000FFF724FF084305D0012004E020463946B4
:1089A000BDE8F08D0020054346EAE0762C433743CE
:1089B0000A986305E40AA0EB08000022FD0A44EAD5
:1089C00047540A3002D500200146E9E70105101995
:1089D0006941DDE9084500196941BDE8F04DA2E7AC
:1089E00070B521F0004303430CD0C1F30A550024B5
:1089F000D5EB040564EB0403D617AD1AB34102DBD3
:108A00000020014670BD201841EB025170BD0000EE
:108A100030B5041E71F1000404DB4FF00044404205
:108A200064EB0101141E73F1000405DB1C464FF0DA
:108A30000043524263EB0403994208BF904230BDA9
:108A4000064C074D06E0E06840F0010394E807009B
:108A500098471034AC42F6D3FFF79AFB98DC030832
:108A6000B8DC0308C0B24FF4F05100F03BBA00008C
:108A70002DE9FF4F087883B09946FF2805D0491C9F
:108A80002D2804D00024002008E000200BE0012461
:108A9000F9E700EB800003EB4000491C0B78FF2B4B
:108AA000F7D104B1404200230293147819461D46C1
:108AB0002D2C01D02B2C04D1521C2D2C13D0002492
:108AC0000294AA461478FF2C0FD00A25A3FB057840
:108AD00001FB05814FF0000C03FB0C11521CE31944
:108AE0004AEB0101EEE70124EAE7814453EA010081
:108AF00002D019F5C87F06DA03980021C0E90011F9
:108B000007B0BDE8F08F0025AE4E2F46DFF8B882E3
:108B1000184600F0FBF9CDE90001B9F1000002DAD6
:108B2000C9F1000400E004460023A74A1AEB030B36
:108B300042EB045A12E0E00707D02A463346384693
:108B40004146FFF75DFC074688462A4633461046F5
:108B50001946FFF755FC05460E466410002CEAD175
:108B6000DDE90001B9F1000F5A46534606DAFFF776
:108B7000B9FC3A464346FFF7B5FC05E0FFF740FC79
:108B80003A464346FFF73CFC029A0AB181F00041A5
:108B9000039AC2E90001B3E72DE9FF4F1F468DB0EC
:108BA000D7E901464FF0FF382E2045464FF0000927
:108BB0000B90B9696D1C0E988847396A82468847C0
:108BC0000028F6D1BAF1FF3F0AD024F4D064002E79
:108BD00011DDBAF12B0F08D0BAF12D0F0BD102E045
:108BE000404611B08DE744F48064B9696D1C0E985D
:108BF00088478246761E6946600501D52D2000E033
:108C00002B208DF8000001F1010B0DF1200809E087
:108C1000B9696D1C0E98884782460F9844F4007419
:108C2000761E0560002E02DDBAF1300FF0D00B99F0
:108C30008A453ED144F0800406E00F99681CA9F1F2
:108C4000010944F400740860B9696D1C761E0E9821
:108C5000884782463028F0D02BE00B998A4505D111
:108C6000200603D444F08004761E18E050462CF011
:108C700039F908B30DF11301761E44F400748B45E5
:108C800008D2AAF130000BF8010B200607D5A9F194
:108C9000010003E0200602D409F101008146A0058D
:108CA00002D50F99681C0860B9696D1C0E98884739
:108CB0008246002ED1DC53E0002E51DDBAF1650F63
:108CC00002D0BAF1450F4BD1A00549D5B9696D1C49
:108CD00024F44074761E0E9888478246002E0CDDE0
:108CE0002B2804D0BAF12D0F07D144F48074B96950
:108CF0006D1C0E9888478246761EE00501D52D2111
:108D000000E02B2108F8011BCDF82C8021E00DF1AB
:108D10002901761E44F4007488450CD2AAF1300073
:108D200010F0FF0088F8000002D10B99884509D99E
:108D300008F1010806E0E00501D5244801E042F20F
:108D40000F708146B9696D1C0E98884782460F984E
:108D50000560002E04DD50462CF0C4F80028D6D162
:108D6000F9690E988847FF208BF8000088F800000A
:108D70000020069007904B466A4608A906A8FFF710
:108D800077FEA00502D46FF001002AE714F0240F4B
:108D90000AD0E00714D1DDE906123868031D3B60F4
:108DA0000068C0E900120BE0DDE90601FFF7C9FC2D
:108DB0000146E00704D13868021D3A60006801608E
:108DC00028460EE7000014400000F03FF1D8FFFFF6
:108DD000426842B1016811F8013B23B1521EC0E95B
:108DE0000012184670470121C160881E7047426812
:108DF0005AB1C368016843B983688B4205D0491EE4
:108E0000521CC0E90012002070474FF0FF3070473D
:108E10002DE9F04D00231A461B1A8A4103DB00207E
:108E20000146BDE8F08DC1F30A52C1F3130141F4CC
:108E300080154FF0000BD10702D100186D41521E72
:108E40000027044640F2FF11384601EB620A3E4615
:108E50008046024600204FF48011FFF7CEFCC21975
:108E60007141BB1846EB0100B4EB030C75EB000C31
:108E700004D3E41A65EB000517460E46241908F1E1
:108E800001006D4180463428E3DDF91946EB060008
:108E9000091BA84103D24FF0FF32134601E0002224
:108EA00013461BEB070046EB0A51BDE8F04DFFF7F8
:108EB0003ABD000030B5041E71F1000404DB4FF030
:108EC0000044404264EB0101141E73F1000405DB11
:108ED0001C464FF00043524263EB04038B4208BF31
:108EE000824230BD7F2801D9002208E0064A02EB09
:108EF0005002C007127800D1120902F00F020120BF
:108F0000904008407047000058DC03080EB540F25E
:108F1000334202920022CDE900221346FFF712FDF0
:108F200003B000BD70B58C1810F8015B15F0070395
:108F300001D110F8013B2A1106D110F8012B03E0F2
:108F400010F8016B01F8016B5B1EF9D12B0705D4FA
:108F50000023521E0DD401F8013BFAE710F8013B43
:108F6000CB1A921C03E013F8015B01F8015B521E5F
:108F7000F9D5A142D8D3002070BD10B502461078B3
:108F800003E012F8014B2318D8B20B1EA1F1010423
:108F9000A1B2F6D110BD000070B5ADF5287D044634
:108FA0000D460020A790A690002604EB44004549FA
:108FB00001EBC000408AA84203DC00200DF5287DAB
:108FC00070BD0020A69077E004EB44003D4B03EB1E
:108FD000C000028A04EB440003EBC00080892844EF
:108FE00081B2394800F010F90020A79011E004EB9D
:108FF0004400344901EBC0004068BDF89C12405C5D
:1090000001A9BDF89C228854BDF89C02401C80B286
:10901000A79004EB44002B4901EBC000008ABDF887
:109020009C128842E3DC04EB4400264A02EBC000B9
:10903000008A401E81B201A8FFF79FFF23490870F4
:1090400004EB44001F4901EBC000008A401E01A947
:10905000085C1E490978884226D10020A79016E0B6
:1090600004EB4400174901EBC0004068BDF89C12B6
:10907000405C04EB4401134A02EBC1018968BDF86E
:109080009C228854BDF89C02401C80B2A79004EB3F
:1090900044000C4901EBC000008A401EBDF89C1240
:1090A0008842DDDC012089E764202CF059F9BDF805
:1090B0009802401C80B2A690BDF89802062883DB77
:1090C00000207BE7A4B40308FCA50020310A00209F
:1090D0002DE9F043ADF5257D04460E460025002719
:1090E000A846A94604EB4400324901EBC000408A7F
:1090F000B04204DC00200DF5257DBDE8F08300259D
:1091000018E004EB44002B4901EBC0008068405D8F
:1091100004EB4401274A02EBC1014968485504EBBE
:109120004400114601EBC0004068405D0DF80500A9
:10913000681C85B204EB44001E4901EBC000008AA4
:10914000401EA842DDDC04EB44000A4602EBC000EE
:10915000008A401E81B26846FFF70FFF04EB44010E
:10916000144A02EBC101098A491E0DF801000027CB
:109170001BE004EB44000F4B03EBC000028A04EB3E
:10918000440003EBC0008089304481B2684600F09F
:109190004FF931462046FFF7FFFE012800D1AAE72C
:1091A00064202CF0DDF8781C87B2062FE1DB00206C
:1091B000A1E70000A4B4030808B50020009026F041
:1091C000D1FD0F49087000F09BF80D480078242865
:1091D00004D0272807D028280FD109E0002109480A
:1091E00080F8081D09E00121064880F8081D04E008
:1091F0000221044880F8081D00BF00BF08BD000020
:109200002C0A0020BC2200202DE9F04106460D4624
:109210001746002401202BF05BFE0020284908801F
:109220000DE026F081FD00F0800000B10BE0012090
:109230002CF096F822480088401C214908802048DC
:109240000088C828EDDB00BF1D480088C82832DA36
:1092500010211C4801F052FC08211A4801F050FC72
:10926000E82000F031F8C5F3871000F02DF8A906CA
:10927000080E00F029F8002000F026F8002404E091
:10928000002000F021F8601C84B2042CF8DB0024DC
:1092900005E0FF2000F018F83055601C84B2BC4295
:1092A000F7DB1021074801F02BFC00202BF010FE0B
:1092B0000120BDE8F08100202BF00AFE0020F8E735
:1092C0002E0A00200000024010B5044600BF022113
:1092D0000A4826F057FE0028F9D02146074826F014
:1092E0005DFE00BF0121054826F04CFE0028F9D0A4
:1092F000024826F050FEC0B210BD00000030014010
:1093000010B501202BF0E4FD00201E4908800DE07F
:1093100026F00AFD00F0800000B10BE001202CF0E7
:109320001FF818480088401C164908801548008816
:10933000C828EDDB00BF13480088C8281CDA1021BC
:10934000114801F0DBFB08210F4801F0D9FB3D205B
:10935000FFF7BAFF2A20FFF7B7FF8020FFF7B4FF1F
:10936000A720FFF7B1FF1021074801F0C9FB00203B
:109370002BF0AEFD012010BD00202BF0A9FD002038
:10938000F9E700002E0A00200000024070B50546F3
:109390000E46002401202BF09BFD0020224908806E
:1093A0000DE026F0C1FC00F0800000B10BE00120D0
:1093B0002BF0D6FF1C480088401C1B4908801A4827
:1093C0000088C828EDDB00BF17480088C82825DAC8
:1093D0001021164801F092FB0821144801F090FB7F
:1093E0008420FFF771FF0020FFF76EFF0020FFF7DA
:1093F0006BFF0020FFF768FF002404E0285DFFF703
:1094000063FF601C84B2B442F8DB1021074801F00E
:1094100077FB00202BF05CFD012070BD00202BF0BD
:1094200057FD0020F9E700002E0A0020000002404E
:1094300070B506460C46154601202BF049FD29461D
:109440003046FFF7A3FF08B9002070BD00201F4978
:1094500008800DE026F068FC00F0800000B10BE011
:1094600001202BF07DFF19480088401C1749088017
:1094700016480088C828EDDB00BF14480088C828BB
:109480001EDA1021124801F039FB0821104801F0C2
:1094900037FB8320FFF718FFC4F38710FFF714FF93
:1094A000A106080EFFF710FF0020FFF70DFF1021A7
:1094B000074801F025FB00202BF00AFD0120C4E73E
:1094C00000202BF005FD0020BFE700002E0A002041
:1094D0000000024030B502460020002304E012F8EC
:1094E000014B60405C1CE3B28B42F8DB30BD0000F6
:1094F00010B5044639202CF075F9E0B22CF092F941
:10950000C4F307202CF08EF9C4F307402CF08AF93D
:10951000200E2CF087F94FF48051034801F0F0FA47
:109520002AF0E6FA10BD0000000402402DE9F041E7
:1095300007460E4614463A202CF054F9F0B22CF0AF
:1095400071F930122CF06EF94FF480510F4801F090
:10955000D7FA19E02AF0CCFA05461D2D11D138466C
:1095600000F0ACF805463B202CF03CF94FF480515C
:10957000064801F0C5FA2F4434B1208828442080E1
:1095800002E02846BDE8F081E4E700000004024064
:109590002DE9F04107460E4614463C202CF022F9F6
:1095A000F0B22CF03FF930122CF03CF94FF480511E
:1095B000104801F0A5FA0CB10020208019E02AF033
:1095C00097FA05461E2D11D1384600F02BF90546B5
:1095D0003D202CF007F94FF48051064801F090FA35
:1095E0002F4434B120882844208002E02846BDE87A
:1095F000F081E4E70004024010B526F08DFA08B1CE
:1096000000F02EF8302000F0A9F810BD10B5044687
:109610002146362000F08EF810BD10B5044614B176
:10962000204600F0ABF8342000F098F810BD10B5DB
:109630000446204600F0A2F820785C2802D020786A
:109640002F2803D10021642000F008F9322000F017
:1096500085F810BD10B5682000F04CF810BD000072
:1096600010B522202CF0BEF82CF0B1F804464FF4CF
:109670008051024801F044FA204610BD0004024027
:109680002DE9F0412CF0A3F804462CF0A0F8054693
:109690002CF09DF806462CF09AF807464FF48051BE
:1096A000054801F02DFA44EA052040EA064040EA68
:1096B0000760BDE8F08100000004024070B5044678
:1096C00027202CF08FF82CF082F80646054646B18C
:1096D00000BF2CF07CF82070641C701EC0B2061E07
:1096E000F7D14FF48051024801F00AFA284670BDC4
:1096F0000004024010B504460C202CF073F82046FC
:109700002CF090F8FFF7BCFF10BD000070B50446C8
:109710000A202CF067F820462CF084F82CF057F83B
:1097200005464FF48051024801F0EAF9284670BD21
:109730000004024070B505460C4628462CF052F84D
:1097400020462CF06FF84FF48051034801F0D8F90F
:109750002AF0CEF970BD00000004024010B50446A6
:1097600020462CF03FF84FF48051034801F0C8F92F
:109770002AF0BEF910BD0000000402402DE9F041BE
:10978000064601202CF02EF82CF021F843282BDA85
:109790002B20FFF7BBFF102826DA2F202CF022F811
:1097A00000202CF03FF83220FFF7D8FF0446142C9D
:1097B0001AD1CF20FFF7AAFF0446ACB14C20FFF727
:1097C00099FF00EB042739464C2000F047F8502061
:1097D000FFF790FF00EB04273946502000F03EF8D9
:1097E0000021702000F03AF82F202BF0FBFF357895
:1097F00028462CF017F809E0761C35785C2D01D04E
:109800002F2D00D1002528462CF00CF8002DF3D187
:109810004FF48051024801F073F9BDE8F081000077
:109820000004024070B504462D202BF0DBFF2BF026
:10983000CEFF0646054646B100BF20782BF0F2FF6A
:10984000641C701EC0B2061EF7D14FF4805102484E
:1098500001F056F9284670BD0004024070B5054677
:109860000C460D202BF0BEFF28462BF0DBFFE0B2AC
:109870002BF0D8FFC4F307202BF0D4FFC4F307402C
:109880002BF0D0FF200E2BF0CDFF4FF4805102487B
:1098900001F036F970BD00000004024070B50246C8
:1098A0000C46FF25FF2309E012F8010B80EA0501B1
:1098B0000648405C80EA03050548435C201EA4F18D
:1098C0000106B4B2F0D145EA032070BD0CB2030822
:1098D0000CB303082DE9F04103460C460020014675
:1098E000024606E013F8010B411842F10002601E27
:1098F00084B2002CF6DC080C40EA024C100C8DB24D
:109900001CEB050140F10002080C40EA024041183E
:109910006FEA010080B2BDE8F08130B50246002058
:10992000002305E012F8015B2C18E0B25C1CE3B2E6
:109930008B42F7DB30BD10B51CF036F910BD10B509
:109940001CF0D0F810BD10B51CF09CF810BD10B57F
:109950001CF0F8F810BD10B51EF0CAF910BD10B516
:1099600025F022FC10BD00000246094B9A4201D2AC
:10997000084801E00648103801F000531BB1064BBF
:109980000B40C36002E0044B0B4083607047000053
:1099900010640240006002407D0F7D0F21B102681B
:1099A00042F00102026003E0026822F0010202605C
:1099B00070470000016821F0010101600021016091
:1099C00041608160C1600161212141614A49884251
:1099D00004D13D21484A103A91608CE04649183143
:1099E000884205D14FF47461434A103A916082E095
:1099F00041493031884205D14FF474113E4A103A42
:109A0000916078E03C494831884205D14FF074615B
:109A1000394A103A91606EE037496031884204D18A
:109A20003649354A103AD16065E033497831884289
:109A300004D13349304A103AD1605CE02E4990316C
:109A4000884204D12F492C4A103AD16053E02A4968
:109A5000A831884205D14FF03D51274A103AD160D4
:109A600049E02949884204D13D21274A083A11603A
:109A700041E025491831884205D14FF47461224AEA
:109A8000083A116037E020493031884205D14FF45F
:109A900074111D4A083A11602DE01B494831884273
:109AA00005D14FF07461184A083A116023E0164955
:109AB0006031884204D11149134A121F11601AE023
:109AC00011497831884204D10D490F4A121F1160A3
:109AD00011E00D499031884204D10A490A4A121F07
:109AE000116008E00849A831884204D14FF03D5187
:109AF000054A121F11607047106002403D000020AF
:109B0000400F002000003D201064024010B501F01D
:109B100080034BB122B1436943F08003436103E00A
:109B2000436923F08003436180290BD02AB1036885
:109B300001F01E042343036004E0036801F01E04E7
:109B4000A343036010BD000010B500220268134B50
:109B50001A40CC680B6823434C6923438C69234328
:109B6000CC6923430C6A23434C6A23438C6A234306
:109B70004C6B23438C6B23431A430260426922F0EF
:109B80000702D1E90B3423431A4342610B69436056
:109B90004B6883608B68C36010BD00003F801CF081
:109BA0001CB500240121202025F0C2FF30200090A8
:109BB00001208DF8040000208DF8060003208DF8A8
:109BC000050000208DF807006946174800F022FFC5
:109BD0003021154800F094FF0021144880F8341615
:109BE00000201349887001204870C8704FF4FA7043
:109BF000886000F021F80F4890F80B0F592811DD0C
:109C000024200A49F5394871082008713020C870AD
:109C100014208870202048700021064880F80B1F0F
:109C200000F04EF81CBD000000140240BC320020C1
:109C3000F0380020BC2200201CB52BF099FCD0206D
:109C40002BF062FC2BF0C8FC00202BF05DFC2BF00D
:109C5000C3FC2BF08DFCD1202BF056FC2BF0BCFC70
:109C600000240EE0062C05DA01202BF01DFC0DF877
:109C7000040004E000202BF017FC0DF80400601C29
:109C8000C4B2072CEEDB2BF08DFC9DF806000A49D0
:109C900048719DF8050008719DF80400C8709DF892
:109CA000020088709DF8010048709DF8001003487C
:109CB00080F80B1F1CBD0000C7310020BC22002013
:109CC0001CB500241B4890F80B0F8DF800001A48B3
:109CD00040788DF80100184880788DF80200012046
:109CE0008DF803001448C0788DF8040012480079FC
:109CF0008DF80500104840798DF806002BF038FCEF
:109D0000D0202BF001FC2BF067FC00202BF0FCFB9B
:109D10002BF062FC00BF07E01DF804002BF0F4FB01
:109D20002BF05AFC601CC4B2072CF5DB2BF03AFC7C
:109D30001CBD0000BC220020C731002070B50246C7
:109D40000C460025002309E012F8010B80EA05010A
:109D50000648405C80EA03050548435C201EA4F1E8
:109D60000106B4B2F0D145EA032070BD0CB203087D
:109D70000CB3030810B504460B460021072A00DD8A
:109D8000072244EA042001462BB901FA02F081B20D
:109D90000912084610BD012B02D11141C8B2F9E7E2
:109DA00000BFF7E710B525F0F5FC10BD10B525F0A4
:109DB000F1FC10BD10B525F0EDFC10BD01490860A7
:109DC00070470000143C0140014600200022074B70
:109DD0001B6803EA0102054B14331B680B4013B1E7
:109DE0000AB1012000E0002070470000003C014063
:109DF000002123498279002A3AD00A461268036872
:109E00009A430B461A600A1D126803689A430B1D99
:109E10001A60027911440A6803681A430A60184AF2
:109E20000832126803689A43154B08331A601A1DEA
:109E3000126803689A43124B0C331A604279102A55
:109E40000ED11A1F126803681A430D4B08331A60AB
:109E50001A1D126803681A43094B0C331A600DE08F
:109E60000749427911440A6803681A430A6005E009
:109E7000027911440A6803689A430A607047000037
:109E8000003C014010B504460B460021072A00DDC6
:109E9000072244EA0420014613B91141C8B210BD9B
:109EA000012B05D101FA02F081B209120846F6E74A
:109EB00000BFF4E7F0B5ADF21C5D04460D4600208E
:109EC000CDF81805CDF81405002604EB44005849D8
:109ED00001EBC000408AA84203DC00200DF21C5DAB
:109EE000F0BD0020CDF814059AE051480122C16868
:109EF000504800F0A9FA4E48406800788DF80000FC
:109F00009DF8000038287DD104EB4400484B03EB5A
:109F1000C000C06804EB4403454F07EBC3031B8A32
:109F200003FB050104EB44003B4603EBC000028A3F
:109F3000404800F089FA0020CDF8180512E004EB43
:109F400044003B4901EBC0004068BDF81815405C77
:109F5000BDF818250DF80200BDF81805401C80B2A8
:109F6000CDF8180504EB4400314901EBC000008A2C
:109F7000BDF818158842E2DC04EB44002C4A02EBE1
:109F8000C000008A401E81B2684600F023FB0646EE
:109F900004EB4400264901EBC000008A401E1DF876
:109FA0000000B04233D10020CDF8180520E004EBCA
:109FB00044001F4901EBC0004068BDF81815415C22
:109FC00004EB44001A4A02EBC0008068BDF8182573
:109FD000024404EB4400164B03EBC000008A401E11
:109FE00068431154BDF81805401C80B2CDF818051F
:109FF00004EB44000E4901EBC000008A401EBDF88E
:10A00000181500E003E08842D1DC012066E76420F7
:10A010002BF0A6F9BDF81405401C80B2CDF814054C
:10A02000BDF814050628FFF660AF002056E70000D3
:10A03000F86203084C7800202DE9F041ADF5A36DDE
:10A0400004460E4600250027A8460020009004EB99
:10A050004400494901EBC000408AB04204DC0020C2
:10A060000DF5A36DBDE8F0814448807B002878D1D0
:10A0700000210846FFF71EFF01287AD1002520E0C5
:10A0800004EB44003C4901EBC0008068411904EB3B
:10A090004400394A02EBC000008A401E7043085C4D
:10A0A00004EB440102EBC1014968485504EB44004C
:10A0B000114601EBC0004068405D01A94855681C8D
:10A0C00085B204EB44002C4901EBC000008AA84291
:10A0D000D6DC00274BE004EB4400274B03EBC00029
:10A0E000C06804EB4403DFF890C00CEBC3031B8A89
:10A0F00003FB060104EB4400634603EBC000008A47
:10A10000401E82B21E4800F021FA04EB44001A4AB5
:10A1100002EBC000008A401E81B201A800F05AFA8A
:10A12000009004EB4400144A02EBC000C06804EB4A
:10A130004402114B03EBC202128A104404EB4402A6
:10A1400003EBC202128A02FB0600411E012268468E
:10A1500000F0FCF931462046FFF7ACFE012801D1A2
:10A160007EE706E064202BF0FBF8781C87B2062F10
:10A17000B1DB002074E70000F8620308BC12002085
:10A180004C780020F0B5ADF21C5D002500240020C5
:10A190000190002600210120FFF78CFE4B4890F82B
:10A1A000FC6C00204A49088080E000256FE0002414
:10A1B00014E04748008800EB4000464951F8300061
:10A1C000005D4349098801EB4101424A02EBC101AC
:10A1D0004968085502A90855601C84B23C480088AB
:10A1E00000EB40003B4901EBC000008A401EA0424A
:10A1F000DFDC3748008800EB40000A4602EBC00075
:10A20000008A401E81B202A800F0E4F901903048B3
:10A21000008800EB40002F4B03EBC000C0682C4BC4
:10A220001B8803EB43032B4F07EBC3031B8A03FB82
:10A2300005012748008800EB40003B4603EBC000C7
:10A24000008A401E82B2244800F080F9204800882D
:10A2500000EB40003A4602EBC000C0681C4A12887E
:10A2600002EB42023B4603EBC202128A1044184A38
:10A27000128802EB420203EBC202128A02FB0500C3
:10A28000411E012201A800F061F9681C85B2104846
:10A29000008800EB40000F4901EBC000408AA84253
:10A2A00085DC0B480088401C094908800848008864
:10A2B0000D28FFF67AAF054880F8FC6C00210120DC
:10A2C000FFF7BAFE0DF21C5DF0BD0000BC220020BD
:10A2D00010000020F86203084C7800201CB5012112
:10A2E000084625F025FC01208DF8040002208DF899
:10A2F000050000208DF8060001208DF807001820C9
:10A3000000906946144800F085FB0522114612486A
:10A3100000F0C8FB052206210F4800F0C3FB052210
:10A3200007210D4800F0BEFBA020009002208DF810
:10A33000040003208DF8050000208DF806008DF83C
:10A3400007006946044800F065FB4020009069461C
:10A35000014800F05FFB1CBD000002402DE9F843FE
:10A36000002400250027002000908046FFF7B6FF5C
:10A3700000F0BCF80A202AF0F3FF6E4608212D48B1
:10A3800000F0BCFB10212B4800F0BAFB062000F0C7
:10A3900091F80821274800F0B3FB0821254800F078
:10A3A000ADFB1021234800F0ABFB012000F082F848
:10A3B000002000F07FF808211E4800F0A1FB1E4895
:10A3C000D0F82C11B0F83021B0F8320102FB0010A7
:10A3D000B0F5003F02D900BE00BFFEE71748006895
:10A3E00008B9FFF7CFFE00201549088017E00024C8
:10A3F00006E0134908782146FFF75CFD601C84B233
:10A400000F48008800EB40000B4901EBC000408A78
:10A41000A042EEDC0A480088401C09490880084830
:10A4200000880D28E3DB0748D0F80C020549C87303
:10A43000BDE8F88300000240F86203081C024342B2
:10A4400010000020BC1200202DE9F04105460C460A
:10A450001646002701202AF038FD0821144800F094
:10A460004DFB1021124800F04BFB032000F022F8B6
:10A47000C4F3074000F01EF8C4F3072000F01AF8F8
:10A48000E0B200F017F800BF06E0002000F012F87C
:10A4900028706D1C781C87B2B742F6DB082104488F
:10A4A00000F02EFB00202AF010FDBDE8F081000036
:10A4B0000000024010B5044600BF02210A4825F002
:10A4C00061FD0028F9D02146074825F067FD00BF4F
:10A4D0000121054825F056FD0028F9D0024825F055
:10A4E0005AFDC0B210BD00000030014000B585B07B
:10A4F0000121080325F06CFB134825F017FD00200F
:10A50000ADF80000ADF80400ADF80600ADF80800A5
:10A510004FF40070ADF80A000820ADF80C000020E0
:10A52000ADF80E000720ADF810004FF48270ADF8C2
:10A5300002006946044825F033FD0121024825F058
:10A54000E9FC05B000BD0000003001402DE9F041FC
:10A5500005460C461646002701202AF0B6FC0821C5
:10A560001B4800F0CBFA1021194800F0C9FA062068
:10A57000FFF7A0FF0821164800F0C2FA082114488E
:10A5800000F0BCFA1021124800F0BAFA0220FFF7DE
:10A5900091FFC4F30740FFF78DFFC4F30720FFF7D7
:10A5A00089FFE0B2FFF786FF00BF05E02878FFF7DC
:10A5B00081FF6D1C781C87B2B742F7DB0821044885
:10A5C00000F09EFA00202AF080FCBDE8F081000037
:10A5D0000000024010B50246107803E012F8014B6B
:10A5E0002318D8B20B1EA1F10104A1B2F6D110BDFF
:10A5F0002C48807F012854D100212A4881772A489D
:10A600000078C0B901202849087028480068C000B7
:10A610002749D1F8301240EA81002549D1F82C129F
:10A6200040EA41002249D1F8281208430F21814312
:10A630002048017017E000201B4908701B48006883
:10A64000C0001B49D1F8301240EA81001849D1F806
:10A650002C1240EA41001649D1F8281208430F2174
:10A6600081431548017013480078134909788842DE
:10A6700017D1104800781149087008460078104931
:10A68000097888420DD00D480078064908760B48B5
:10A6900000780B4908700948007810B10120014981
:10A6A000C8757047BC120020DE0A00203402424206
:10A6B00000004242DF0A0020E00A0020E10A0020F8
:10A6C000DD0A002010B5ADF57C7D00247DA000687A
:10A6D000FB9000200090FEF78FFF14287CD17A4871
:10A6E000FEF7A5FF7949087008460078142874D150
:10A6F000FEF7B0FF0021764A03C2BDF80000FEF766
:10A70000F7FE6A464FF4FA7101A8FEF70FFF71A138
:10A7100001A82BF003F8714908800846008810B39F
:10A7200000BF04E000216E480155601C84B2282C53
:10A73000F8DB01A9694A128888186AA12AF0EEFF9D
:10A7400069490880002409E064480088C01C20444E
:10A7500001A9095C62480155601C84B26248008806
:10A76000001FA042F0DC61A101A82AF0D7FF5B49DD
:10A7700008800846008820B3002405E000215848DE
:10A7800028300155601C84B2282CF7DB01A9534AFC
:10A790001288881853A12AF0C1FF53490880002469
:10A7A0000AE04E4800880830204401A9095C4C4862
:10A7B00028300155601C84B24B4800880938A042FB
:10A7C000EFDC4DA101A82AF0A9FF44490880084602
:10A7D000008830B3002407E06BE05BE000214048D4
:10A7E00050300155601C84B2142CF7DB01A93B4AA0
:10A7F000128888183BA12AF091FF3B490880002469
:10A800000AE0364800880C30204401A9095C34482D
:10A8100050300155601C84B2334800880D38A04286
:10A82000EFDC39A101A82AF079FF2C4908800846FD
:10A83000008820B3002405E0002029494639085546
:10A84000601C84B2322CF7DB01A9244A12888818D4
:10A8500024A12AF063FF2449088000240AE01F484D
:10A860000088801D204401A9085C1D49463908550F
:10A87000601C84B21C480088C01FA042EFDC00218D
:10A880000320FFF7D9FB0120FEF7C0FE01200DF5E4
:10A890007C7D10BD0D480078422803D10A48FEF7A0
:10A8A000BCFE0CE00120FEF7B1FE00200749087055
:10A8B00005E00021164880F80A1F2AF0C3FE00BFF9
:10A8C000E5E700000D0A0000480A0020380A0020D1
:10A8D000400A002041504E3D000000005E0A00206A
:10A8E000D03900203B0000005C0A0020574946494F
:10A8F0004E414D453D000000574946495041535394
:10A90000574F52443D0000005345525645523D00BA
:10A91000BC22002010B504463548844208D10121EC
:10A92000084625F015F90021012025F011F95EE017
:10A930003048844208D10121022025F009F9002184
:10A94000022025F005F952E02B48844208D101216C
:10A95000042025F0FDF80021042025F0F9F846E058
:10A960002648844208D10121082025F0F1F8002171
:10A97000082025F0EDF83AE02148844208D1012171
:10A98000102025F0E5F80021102025F0E1F82EE058
:10A990001C48844208D10121202025F0D9F800214B
:10A9A000202025F0D5F822E01748844208D1012163
:10A9B000402025F0CDF80021402025F0C9F816E010
:10A9C0001248844208D10121802025F0C1F80021DD
:10A9D000802025F0BDF80AE00D48844207D101210E
:10A9E000801525F0B5F80021A01525F0B1F810BDAF
:10A9F000000002400004024000080240000C024037
:10AA0000001002400014024000180240001C0240E6
:10AA100000200240F0B50A4600210023002400BFB8
:10AA20003DE0012505FA01F3156805EA03049C429F
:10AA300034D105684F000326BE40B5430560157943
:10AA40004E00B5400668354305601579012D02D0EA
:10AA50001579022D16D185684F000326BE40B543F7
:10AA6000856055794E00B5408668354385604568F8
:10AA700001268E40B5434560456896798E40B6B252
:10AA800035434560C5684F000326BE40B543C560E9
:10AA9000D5794E00B540C6683543C560491C1029BC
:10AAA000BFD3F0BDF0B5002300244D07ED0E02FA30
:10AAB00005F3CE1000F1200555F826504E07F70E8D
:10AAC0000F26BE40B543CF1000F1200646F82750B0
:10AAD000CE1000F1200555F8265045EA0304CE10AB
:10AAE00000F1200545F82640F0BD0246002013691C
:10AAF0000B400BB1012000E00020704741837047FC
:10AB0000018370470249087E0021014A117670478F
:10AB1000BC1200200E48006800F0010000B100BE29
:10AB2000012080F3138800BF00BFBFF34F8F084898
:10AB3000E438006800F4E06006490843001D044959
:10AB4000E4390860BFF34F8F00BF00BFFEE700008D
:10AB5000F0ED00E00000FA054AF6AA20014908607D
:10AB6000704700000030004030B50246002400234A
:10AB700005E012F8015B2819C4B2581CC3B28B421D
:10AB8000F7DB6042C0B230BD10B500242AF05AFD98
:10AB900064202AF0E5FB10BD2DE9F043ADF2DC7D29
:10ABA00080460E46144699460025002783A000687B
:10ABB000CDF8D80700200190042C7CDC8048007977
:10ABC000302101EB101004EBC40101EB04117D4AAC
:10ABD000114408717A48007900F00F00303004EB1E
:10ABE000C40101EB0411114448717548C07830214B
:10ABF00001EB101004EBC40101EB04111144887146
:10AC00006F48C07800F00F00303004EBC40101EB56
:10AC100004111144C871FEF7EFFC14287ED16A4874
:10AC20000078142809D004EBC40101EB0411654A33
:10AC30008818FEF7FCFC6449087063480078142803
:10AC40006DD1B6F57A7F01DD4FF47A76FEF702FD1D
:10AC500000215E4A03C25D480068FEF749FC58487F
:10AC6000C078302101EB10108DF808005448C078EE
:10AC700000F00F0030308DF809005148807801EB6A
:10AC800010108DF80A004E48807800F00F00303028
:10AC90008DF80B004A48407801EB10108DF80C003D
:10ACA0004748407800F00F0030308DF80D004848DC
:10ACB00090F80B0F00E07CE001EB10108DF80E0017
:10ACC000434890F80B0F00F00F0030308DF80F0064
:10ACD000B9F1000F03D154208DF8100005E0B9F14F
:10ACE000010F02D152208DF810003A208DF811008A
:10ACF00000252CE0284605EBD071491018F801100A
:10AD00000F110A2097FBF0F0C0EBC00107F13000F3
:10AD10000844C1B202AA05F10A0001E043E02EE0B6
:10AD20001154284605EBD071491018F8011001F0B4
:10AD30000F070A2097FBF0F0C0EBC00107F13000CD
:10AD40000844C1B205F10B001154A81C85B2B5EB43
:10AD5000460FCFDB0A2000EB460081B201AA02A811
:10AD6000FEF716FC01AA02210DF5FB60FEF710FCB0
:10AD70000120FEF74BFC00201349087019E012482F
:10AD80000078422808D104EBC40101EB04110D4AFC
:10AD90008818FEF742FC0CE00120FEF737FC00208B
:10ADA0000949087005E00021094880F80A1F2AF0C7
:10ADB00049FC0DF2DC7DBDE8F08300000D0A0000C7
:10ADC000C7310020600A0020380A0020400A002015
:10ADD000BC22002070B5BAB000213991389137916A
:10ADE00036913591349133913291002230923192E3
:10ADF0002E922F922D912C912B912A91299128916D
:10AE000027912691259124911691159114911391D2
:10AE10001291119110919FEDFE0A8DED0F0AFDA088
:10AE200006C8CDE90D12FDA006C8CDE90B12BAE0A7
:10AE3000FC48807858B30020FA498870FA48B0F886
:10AE40003005FA490968C1F57A7188421FD1F7487F
:10AE50000068C0F57A7081B2F348A0F82815002187
:10AE6000F248001FFEF79AFDF149F048001FFEF777
:10AE70007BFD0120EF4908704FF47A70EB498C3963
:10AE8000C1F88C000121E948001FFEF787FDE54865
:10AE9000807B50B30021E3488173E7484088E34951
:10AEA0008C39496CC1F57A7188421ED1DF488C38E3
:10AEB000406CC0F57A70E049083948800021DB48D1
:10AEC0004C38FEF76BFDDD49D8484C38FEF74CFD99
:10AED0000121DB4801704FF47A70D4498C39486401
:10AEE0000121D2484C38FEF759FDCE48807E50B340
:10AEF0000021CC488176D0488088CC498C3949697A
:10AF0000C1F57A7188421ED1C8488C384069C0F5B5
:10AF10007A70C949083988800021C4487C38FEF716
:10AF20003DFDC849C1487C38FEF71EFD0120C649D9
:10AF300008704FF47A70BD498C3948610121BB48D3
:10AF40007C38FEF72BFDB74890F8260058B3002157
:10AF5000B44880F82610B848C088B4498C39C96A0A
:10AF6000C1F57A7188421ED1B0488C38C06AC0F5EC
:10AF70007A70B1490839C8800021AC486438FEF7BE
:10AF80000DFDB249A9486438FEF7EEFC0121B04836
:10AF900001704FF47A70A5498C39C8620121A34829
:10AFA0006438FEF7FBFC9F488178807B01449D4814
:10AFB000807E01449B4890F82600084400287FF4D6
:10AFC00037AF12F08EBB9B48007820B10020994922
:10AFD00008702D9019E09A48007828B1002098490F
:10AFE000087001202D9010E09748007828B10020CB
:10AFF0009549087002202D9007E09548007820B10F
:10B0000000209349087003202D909DF8B41001EBA7
:10B010004100C0EBC1108F4911F83000C12836D172
:10B020009DF8B41001EB4100C0EBC110894901EB60
:10B03000C000807808282AD101217B4880F880153B
:10B040009DF8B40030B101280AD002280ED00328A0
:10B0500018D111E04FF480417F48FFF74FFD11E018
:10B060004FF400517C48FFF749FD0BE04FF480514D
:10B070007948FFF743FD05E04FF400617648FFF79C
:10B080003DFD00BF00BF00207449086099E7654896
:10B090000C389DF8B41010F811000121B1EBD01F4D
:10B0A00052F08B816E4890F80A0FB8B162490839A6
:10B0B0009DF8B40031F810100A919DF8B41001EB1E
:10B0C0004100C0EBC110634901EBC00101230991AC
:10B0D0009DF8B420DDE90901FFF75EFD9DF8B4108D
:10B0E00001EB410000EB01105E4901EB001081799A
:10B0F0002C919DF8B0000B2892F02981DFE810F028
:10B1000078810B00FB16A92AC23AF43C0E41014D8E
:10B11000565B0B6B79819DF8B41001EB4100C0EBDD
:10B12000C1104C4901EBC000417808460A9100214A
:10B130001AF0C6FBC1B22891002136911CE09DF89F
:10B14000B41001EB410000EB0110464901EB001186
:10B150003031BDF8D80001EB001041789DF8A00017
:10B16000814204D1BDF8D800C1B2289112E0BDF8E7
:10B17000D800401C81B236919DF8B40000EB40012C
:10B1800001EB0010374901EB0010C179BDF8D80080
:10B190008142D4DC00BF9DF8B40000EB4001C1EB5C
:10B1A000C0102C4901EBC000807800F0F000A0280E
:10B1B0000DD19DF8B41001EB4100C0EBC110254941
:10B1C00001EBC000807800F00F0129910AE09DF8A2
:10B1D000B41001EB4100C0EBC1101E4901EBC000EF
:10B1E00081782991BDF8A40008B9102029909DF814
:10B1F000B41001EB4100C0EBC110164901EBC001D6
:10B20000BDF8A400401C095C2691BDF8A4002BE009
:10B210000000000001693230313030000169323005
:10B2200045303000D83D0020BC7200208C600240C8
:10B230000088002012000020EC7700200080201001
:10B24000130000202080001014000020008800104F
:10B250001500002064860020001802408802424247
:10B26000BC22002004400020401C81B20A919DF8BD
:10B27000B40000EB4001C1EBC010FE4901EBC0017E
:10B280000991DDE909011AF0ABFF37909DF8B40090
:10B2900000EB4001C1EBC010F64901EBC001BDF865
:10B2A000A400801C095CBDF8DC00814242F02186CC
:10B2B0009DF8B40000EB4001C1EBC010ED4901EB7B
:10B2C000C0004078002842F314869DF8B40000EBDB
:10B2D0004001C1EBC010E74901EBC001BDF8A4007B
:10B2E000C01C0A5C9DF8B40040F2991110FB01F0FB
:10B2F000E14901EBC00101F552719DF8A00000EB9E
:10B30000400303EB001001EBC00080F84420002153
:10B31000DA4A9DF8B40002EB00129DF8A000115427
:10B32000D74890F82800012840D19DF8B40000EBE0
:10B33000400101EB0010D34901EB001030309DF8C3
:10B34000A01000EB0110801C0A90007820F0800013
:10B3500080300A990870BDF89800B62814D0C52826
:10B3600019D0D52802D0D9281CD106E0BDF8A400F8
:10B37000032801DA0020269017E0BDF8A400032876
:10B3800001DA0020269010E0BDF8A400032801DABD
:10B390000020269009E0BDF8A400032801DA00206F
:10B3A000269002E00020269000BF00BFBDF8980064
:10B3B000C52801F09C8519DCB5287DD00DDC11284D
:10B3C00002F01484122802F05984132802F0EB844E
:10B3D000B22842F08D8501F053BDB62801F00D84EE
:10B3E000B92801F08B83C328F3D1FCE3D9287CD0A2
:10B3F00007DCCA287AD0CE2802F0ED82D528E8D121
:10B4000009E0E12802F0FD82E52802F01083E72838
:10B41000DFD102F0D1BB9DF8B41001EB4100C0EBCD
:10B42000C110944901EBC000C178974880F8021D13
:10B430009DF8B41040F2991011FB00F08E4901EB19
:10B44000C00101F552719DF8A00000EB400202EB33
:10B45000001011F830109DF8B40040F2991210FB62
:10B4600002F0854A02EBC000407981427DDA9DF806
:10B47000B41001EB410000EB0110824901EB001018
:10B4800030309DF8A01000EB0110801C0A907E481F
:10B4900090F8020D0121A1EBD0100A99097860F310
:10B4A00000010A980170784890F8020DC0F340102E
:10B4B000F0BB9DF8B41000E0F5E301EB410000EBB8
:10B4C0000110704901EB001030309DF8A01000EB26
:10B4D00001108078C0F3401050B39DF8B40000EB29
:10B4E000400101EB0010674901E0FDE3FDE301EBE2
:10B4F000001030309DF8A01000EB0110801C0A9065
:10B50000007820F00200801C0A9908709DF8B410A1
:10B5100040F2991011FB00F0114601EBC00000F55C
:10B5200052709DF8A01001EB410202EB011100E006
:10B530000EE000EBC10018300A90007820F0020005
:10B54000801C0A9908709DF8B4100220FEF774FD63
:10B5500000219DF8B40040F2991210FB02F0464A17
:10B5600002EBC0000171022200E028E09DF8B40067
:10B5700040F2991110FB01F03F4901EBC00101F5C8
:10B5800052719DF8A00000EB400303EB001001F89E
:10B590003020B6229DF8B40040F2991110FB01F062
:10B5A000354901EBC00000F552709DF8A01001EB89
:10B5B000410303EB011100EBC1004271FDE332488E
:10B5C00090F8020DC0F3C000A8B9E5229DF8B400C0
:10B5D00040F2991110FB01F0274901EBC00000F582
:10B5E00052709DF8A01001EB410303EB011100EB39
:10B5F000C1004271E2E79DF8B41001EB410000EB9D
:10B600000110204901EB001030309DF8A01000EB34
:10B610000110801C0A901C4890F8020D0121A1EB3A
:10B62000D0100A990A7860F300020A709DF8B410ED
:10B6300001EB410000EB0110124901EB001030302A
:10B640009DF8A01000EB0110801C0A900E4890F8A5
:10B65000020D42090A98007862F341000A990870C5
:10B660009DF8B40000EB400101EB0010054901EB2F
:10B6700000100BE064860020C4440020383E002007
:10B68000BC12002004400020BC22002030309DF875
:10B69000A01000EB01108078C0F340029DF8B400C8
:10B6A00040F2991110FB01F0FE4901EBC00000F5DA
:10B6B00052709DF8A01001EB410303EB011100EB68
:10B6C000C100007EC0F3400082427BD09DF8B410E0
:10B6D00040F2991011FB00F0F24901EBC00000F5B7
:10B6E00052709DF8A01001EB410202EB011100EB3A
:10B6F000C10018300A909DF8B41001EB410000EB36
:10B700000111E94800EB011030309DF8A01000EB6A
:10B710000110807842080A98007862F341000A9983
:10B7200008709DF8B41001EB410000EB0110DE49F8
:10B7300001EB001030309DF8A01000EB0110807874
:10B74000C0F34000E8B3D9229DF8B40040F299114B
:10B7500010FB01F0D34901EBC00000F552709DF8D9
:10B76000A01001EB410303EB011100EBC10042719A
:10B77000CE4890F8900700287ED19DF8B40040F2A2
:10B78000991110FB01F0C74901EBC00000F55270A0
:10B790009DF8A01001EB410202EB011100EBC1008A
:10B7A00090F87F00002867D011239DF8B40040F284
:10B7B000991110FB01F0BB4901EBC00101F5527179
:10B7C00001E06EE088E19DF8A00000EB400202EB92
:10B7D000001001EBC00090F8800040F2991110FBBE
:10B7E00001F0B04901EBC00101F552719DF8B400C0
:10B7F00040F2991210FB02F0AA4A02EBC00202F5D5
:10B8000052729DF8A00000EB400404EB001002EB24
:10B81000C00090F8810000EB400202EB001001EB49
:10B82000C00080F87E30F3239DF8B40040F29911F7
:10B8300010FB01F09B4901EBC00101F552719DF82D
:10B84000A00000EB400202EB001001EBC00090F8FA
:10B85000800040F2991110FB01F0924901EBC00108
:10B8600001F552719DF8B40040F2991210FB02F0FC
:10B870008C4A02EBC00000E096E000F552709DF8A3
:10B88000A02002EB420404EB021200EBC20090F88D
:10B89000810000EB400202EB001001EBC00043719D
:10B8A00015E101229DF8B40040F2991110FB01F05E
:10B8B0007C4901EBC00101F552719DF8A00000EB3D
:10B8C000400303EB001001EBC0004273D9229DF846
:10B8D000B40040F2991110FB01F0724901EBC00174
:10B8E00001F552719DF8A00000EB400303EB00103E
:10B8F00001EBC000427101229DF8B40040F29911A1
:10B9000010FB01F0674901EBC00000F552709DF893
:10B91000A01001EB410303EB011100EBC10080F823
:10B920004620624890F89007F0BB9DF8B40040F2C2
:10B93000991110FB01F05B4901EBC00000F552705A
:10B940009DF8A01001EB410202EB011100EBC100D8
:10B9500090F87F0040B39DF8B41040F2991011FBAD
:10B9600000F0504901EBC00101F552719DF8A000B3
:10B9700000EB400202EB001001EBC00090F88010D9
:10B9800001EB410000EB0110474901EB00113031A0
:10B990009DF8B40040F2991210FB02F0414A02EB0C
:10B9A000C00202F5527200E091E09DF8A00000EBA9
:10B9B000400303EB001002EBC00090F8810001EBA4
:10B9C0000010801C0A90007820F004020A9802708F
:10B9D00000239DF8B40040F2991110FB01F03149A9
:10B9E00001EBC00000F552709DF8A01001EB410280
:10B9F00002EB011100EBC10090F8800040F29911B8
:10BA000010FB01F0274901EBC00000F552709DF8D2
:10BA1000B41040F2991211FB02F1224A02EBC1026A
:10BA200002F552729DF8A01001EB410404EB0111E4
:10BA300002EBC10191F8811001EB410202EB01110F
:10BA400000EBC10080F87E30F3239DF8B40040F293
:10BA5000991110FB01F0134901EBC00000F5527081
:10BA60009DF8A01001EB410202EB011100EBC100B7
:10BA700090F8800040F2991110FB01F0094901EBA8
:10BA8000C00000F552709DF8B41040F2991211FBFD
:10BA900002F1044A02EBC10101F552719DF8A020A8
:10BAA00006E00000C444002004400020BC32002016
:10BAB00002EB420404EB021201EBC20191F8811087
:10BAC00001EB410202EB011100EBC10043719DF853
:10BAD000B4100220FEF7B0FA9DF8B40000EB40016C
:10BAE00001EB0010FC4901EB001130319DF8A00082
:10BAF00001EB0010807800F001029DF8B40040F2E4
:10BB0000991110FB01F0F54901EBC00000F55270EE
:10BB10009DF8A01001EB410303EB011100EBC10004
:10BB2000007E00F0010082427BD09DF8B40040F21C
:10BB3000991110FB01F0E94901EBC00000F55270CA
:10BB40009DF8A01001EB410202EB011100EBC100D6
:10BB500018300A909DF8B41001EB410000EB011081
:10BB6000DD4901EB001030309DF8A01000EB011012
:10BB700082780A98007862F300000A9908709DF8AC
:10BB8000B41001EB410000EB0110D34901EB0010B0
:10BB900030309DF8A01000EB0110807800F001001B
:10BBA000F0BB9DF8B41001EB410000EB0110CA4955
:10BBB00001EB001030309DF8A01000EB01108078F0
:10BBC000C0F3401070B39DF8B41040F2991011FB0F
:10BBD00000F0C24901EBC00000F552709DF8A010C2
:10BBE00001EB410200E0FDE302EB011100EBC100BB
:10BBF00090F84600B0B99DF8B41040F2991011FBCE
:10BC000000F0B64901EBC00000F552709DF8A0109D
:10BC100001EB410202EB011100EBC100407B02E0AD
:10BC200071E0A9E23EE0E8BB9DF8B41001EB4100F1
:10BC300000EB0110A84901EB001030309DF8A01076
:10BC400000EB01108078C0F3400058BB01229DF842
:10BC5000B40040F2991110FB01F0A04901EBC001C2
:10BC600001F552719DF8A00000EB400303EB0010BA
:10BC700001EBC0004273D9229DF8B40040F2991143
:10BC800010FB01F0954901EBC00101F552719DF8DF
:10BC9000A00000EB400303EB001001EBC000427179
:10BCA000012201E015E0FDE39DF8B40040F2991196
:10BCB00010FB01F0894901EBC00000F552709DF8BE
:10BCC000A01001EB410303EB011100EBC10080F870
:10BCD000462000229DF8B40040F2991110FB01F0BB
:10BCE0007E4901EBC00001E0FBE3FBE300F552708D
:10BCF0009DF8A01001EB410303EB011100EBC10023
:10BD000080F8452033E29DF8B41040F2991011FB01
:10BD100000F0724901EBC00000F552709DF8A010D0
:10BD200001EB410202EB011100EBC10090F846006B
:10BD3000B0B901229DF8B40040F2991110FB01F056
:10BD4000664901EBC00000F552709DF8A01001EBB0
:10BD5000410303EB011100EBC10080F845202AE00C
:10BD600000229DF8B40040F2991110FB01F05B49EC
:10BD700001EBC00101F552719DF8A00000EB4003FA
:10BD800003EB001001EBC00080F845209DF8B410D3
:10BD900001EB410000EB01104F4901EB0011303184
:10BDA0009DF8A00001EB0010801C0A90007820F0A4
:10BDB00001020A9802704A4800E053E290F89007A6
:10BDC00080B19DF8B41001EB410000EB0110424935
:10BDD00001EB001030309DF8A01000EB0110807ACC
:10BDE00002288FD13F4890F8290001288AD13D4888
:10BDF000D0F80C023B49498D88426CD29DF8B400C2
:10BE000040F2991110FB01F0344901EBC00000F53C
:10BE100052709DF8A01001EB410202EB011100EB02
:10BE2000C10090F84500012854D19DF8B40040F2BB
:10BE3000991110FB01F0294901EBC00000F5527087
:10BE40009DF8A01001EB410202EB011100EBC100D3
:10BE500090F87F00F0BB9DF8B40000EB400101EBCF
:10BE600000101D4901EB001130319DF8A00001EBDD
:10BE7000001001789DF8B40040F2991210FB02F016
:10BE8000164A02EBC0004170C3229DF8B40040F294
:10BE9000991110FB01F0114901EBC00101F552713C
:10BEA0009DF8A00000EB400303EB001001EBC00085
:10BEB000427100229DF8B40000EB400101EB00103C
:10BEC000054901EB001130319DF8A00001EB001095
:10BED000426009E066E0FAE004400020C44400202B
:10BEE000BC320020BC12002001229DF8B40000EBFF
:10BEF000400101EB0010FE4901EB001130319DF8CB
:10BF0000A00001EB0010C2729DF8B4100220FEF7F1
:10BF100093F8002139911CE000229DF8B40040F212
:10BF2000991110FB01F0F34901EBC00101F55271C9
:10BF30009DF8A00000EB400303EB001001EBC001F3
:10BF40004731BDF8E4000A54BDF8E400401C81B25A
:10BF50003991BDF8E4000628DEDB002039901CE0B2
:10BF600000229DF8B40040F2991110FB01F0E14964
:10BF700001EBC00101F552719DF8A00000EB4003F8
:10BF800003EB001001EBC0016331BDF8E4000A547B
:10BF9000BDF8E400401C81B23991BDF8E4000F28DF
:10BFA000DEDBE4E09DF8B41040F2991011FB00F0E4
:10BFB000D04901EBC00000F552709DF8A01001EBD4
:10BFC000410202EB011100EBC10090F8450001288D
:10BFD0007DD19DF8B41040F2991011FB00F0C549D5
:10BFE00001EBC00101F552719DF8A00000EB400289
:10BFF00002EB001001EBC00090F8801040F29910A5
:10C0000011FB00F0BB4901EBC00101F552719DF835
:10C01000B40040F2991210FB02F0B64A02EBC000E5
:10C0200000F552709DF8A02002EB420303EB0212D0
:10C0300000EBC20090F8810000EB400202EB001020
:10C0400001EBC00090F87E00032840D100239DF84A
:10C05000B40040F2991110FB01F0A64901EBC001B8
:10C0600001F552719DF8A00000EB400202EB0010B8
:10C0700001EBC00090F8800040F2991110FB01F034
:10C080009C4901EBC00101F552719DF8B40040F2EA
:10C09000991210FB02F0974A02EBC00202F55272AD
:10C0A0009DF8A00000EB400404EB001002EBC00080
:10C0B00090F8810000EB400202EB001001EBC000A1
:10C0C00080F87E309DF8B40000EB400100E04EE0C7
:10C0D00001EB0010864901EB001130319DF8A00002
:10C0E00001EB001001789DF8B40040F2991210FBAA
:10C0F00002F0804A02EBC0004170C3229DF8B400F8
:10C1000040F2991110FB01F07A4901EBC00101F5F1
:10C1100052719DF8A00000EB400303EB001001EB0F
:10C12000C000427100229DF8B40000EB400101EB19
:10C1300000106F4901EB001130319DF8A00001EBB8
:10C140000010426002229DF8B40000EB400101EBB8
:10C150000010674901EB001130319DF8A00001EBA0
:10C160000010C2729DF8B4100220FDF765FF9DF823
:10C17000B4100220FDF760FF9DF8B40000EB400111
:10C1800001EB00105A4901EB001030309DF8A0106F
:10C1900000EB01108078C0F34000A0B1D9229DF8D7
:10C1A000B40040F2991110FB01F0524901EBC000BC
:10C1B00000F552709DF8A01001EB410303EB011153
:10C1C00000EBC10042719DF8B40040F2991110FBE0
:10C1D00001F0484901EBC00000F552709DF8A01035
:10C1E00001EB410202EB011100EBC1008078B228A3
:10C1F00038D19DF8B40000EB400101EB00103C4940
:10C2000001EB001030309DF8A01000EB0110807899
:10C21000C0F3400030BB9DF8B40000EB400101EBDF
:10C220000010334901EB001030309DF8A01000EBF6
:10C2300001108078C0F34010A0B9E5229DF8B40049
:10C2400040F2991110FB01F02A4901EBC00000F502
:10C2500052709DF8A01001EB410303EB011100EBBC
:10C26000C10042719DF8B40000EB400101EB0010E9
:10C270001F4901EB001030309DF8A01000EB0110B9
:10C2800080780121B1EBD01F7DD19DF8B40000EB87
:10C29000400101EB0010164901EB001030309DF811
:10C2A000A01000EB0110807800F0010000286AD196
:10C2B0009DF8B40040F2991110FB01F00D4901EB1B
:10C2C000C00000F552709DF8A01001EB410202EB96
:10C2D000011100EBC10090F84600002853D19DF8F1
:10C2E000B40000EB400101EB0010014904E0000044
:10C2F00004400020C444002001EB001030309DF8C1
:10C30000A01000EB01108078C0F3C000D8BB9DF8EE
:10C31000B40000EB400101EB0010FE4901EB0010FE
:10C3200030309DF8A01000EB0110407A00F00100C1
:10C3300048B39DF8B40040F2991110FB01F0F649A2
:10C3400001EBC00000F552709DF8A01001EB410216
:10C3500002EB011100EBC10090F8900000F0010029
:10C3600088B99DF8B40040F2991110FB01F0EA4938
:10C3700001EBC00000F552709DF8A01001EB4102E6
:10C3800002EB011100E02EE000EBC10090F882000A
:10C3900048B3002039902FE09DF8B40040F2991185
:10C3A00010FB01F0DC4901EBC00101F552719DF871
:10C3B000A00000EB400202EB001001EBC00000F116
:10C3C0008301BDF8E4000A5C9DF8B40000EB400175
:10C3D00001EB0010CF4901EB00100E30BDF8E41066
:10C3E000405C01E0C5E27AE0824200D008E0BDF89E
:10C3F000E400401C81B23991BDF8E4000628CBDB93
:10C4000000BFBDF8E400062869D139902CE09DF802
:10C41000B40040F2991110FB01F0BF4901EBC001DB
:10C4200001F552719DF8A00000EB400202EB0010F4
:10C4300001EBC00000F18301BDF8E4000A5C9DF847
:10C44000B40000EB400101EB0010B24901EB001019
:10C450000E30BDF8E410405C824200D008E0BDF828
:10C46000E400401C81B23991BDF8E4000A28CEDB1B
:10C4700000BFBDF8E4000A2831D09DF8B41040F2A6
:10C48000991011FB00F0A44901EBC00000F55270B7
:10C490009DF8A01001EB410202EB011100EBC1007D
:10C4A000903000E0B2E20A90007820F00100401CD9
:10C4B0000A99087012229DF8B40040F2991110FBFD
:10C4C00001F0954901EBC00000F552709DF8A010F5
:10C4D00001EB410303EB011100EBC100427101F0DC
:10C4E00007BD00E07CE29DF8B41001EB410000EBD9
:10C4F0000110884901EB0010007BD0BBBDF8A400FF
:10C50000082800D0EBE70020399028E09DF8B4100F
:10C5100001EB4100C0EBC110804901EBC001BDF847
:10C52000E400C01C085C00F00F00092800DD1AE0E0
:10C530009DF8B41001EB4100C0EBC110774901EB4D
:10C54000C001BDF8E400C01C085C00F0F0009028B9
:10C5500000DD08E0BDF8E400401C81B23991BDF86F
:10C56000E4000628D2DB00BFBDF8E400062801DAAB
:10C57000B5E76EE09DF8B41001EB4100C0EBC110CF
:10C58000664901EBC000C07801049DF8B40000EBDF
:10C590004002C2EBC010614A02EBC000007941EAE0
:10C5A00000219DF8B40000EB4002C2EBC0105B4AD2
:10C5B00002EBC000407901439DF8B40040F29912AB
:10C5C00010FB02F0544A02EBC00202F552729DF8D1
:10C5D000A00000EB400303EB001002EBC000C0F82A
:10C5E0001A109DF8B41001EB4100C0EBC1104B498B
:10C5F00001EBC000807901049DF8B40000EB40021B
:10C60000C2EBC010454A02EBC000C07941EA0021EC
:10C610009DF8B40000EB4002C2EBC0103F4A02EBB1
:10C62000C000007A01439DF8B40040F2991210FB5B
:10C6300002F0394A02EBC00000F552709DF8A020CC
:10C6400002EB420303EB021200EBC200C0F81E1023
:10C65000C7E0BDF8A4000A2800D040E700203990C8
:10C6600028E09DF8B40000EB4001C1EBC0102B495D
:10C6700001EBC001BDF8E400C01C085C00F00F0035
:10C68000092800DD1AE09DF8B40000EB4001C1EB81
:10C69000C010224901EBC001BDF8E400C01C085CD9
:10C6A00000F0F000902800DD08E0BDF8E400401C38
:10C6B00081B23991BDF8E4000828D2DB00BFBDF893
:10C6C000E400082800DA0AE79DF8B40000EB400116
:10C6D000C1EBC011114800EBC100C07801069DF804
:10C6E000B40000EB4002C2EBC0100C4A02EBC000E9
:10C6F000007941EA00419DF8B40000EB4002C2EB32
:10C70000C010064A02EBC000407941EA00219DF8C2
:10C71000B40005E004400020C444002064860020EA
:10C7200000EB4002C2EBC010FE4A02EBC000807971
:10C7300001439DF8B40040F2991210FB02F0FA4A4E
:10C7400002EBC00202F552729DF8A00000EB40031C
:10C7500003EB001002EBC000C0F81A109DF8B40003
:10C7600000EB4001C1EBC010EE4901EBC000C07905
:10C7700001069DF8B40000EB4002C2EBC010E94A8C
:10C7800002EBC000007A41EA00419DF8B40000EBE2
:10C790004002C2EBC010E34A02EBC000407A41EA1B
:10C7A00000219DF8B40000EB4002C2EBC010DD4A4E
:10C7B00002EBC000807A01439DF8B40040F2991268
:10C7C00010FB02F0D84A02EBC00000F552709DF851
:10C7D000A02002EB420303EB021200EBC200C0F800
:10C7E0001E109DF8B40040F2991110FB01F0CE49E3
:10C7F00001EBC00101F552719DF8A00000EB400271
:10C8000002EB001011F830109DF8B40040F29912BC
:10C8100010FB02F0C44A02EBC0004079814234DAD6
:10C8200000219DF8B40040F2991210FB02F0BE4ABC
:10C8300002EBC000017104229DF8B40040F299118E
:10C8400010FB01F0B84901EBC00101F552719DF8F0
:10C85000A00000EB400303EB001001F83020C522DC
:10C860009DF8B40040F2991110FB01F0AE4901EBC4
:10C87000C00000F552709DF8A01001EB410303EBDE
:10C88000011100EBC100427172E09DF8B41001EBA0
:10C89000410000EB0110A54901EB001030309DF87C
:10C8A000A01000EB01108078C0F34000A8B1D522A1
:10C8B0009DF8B40040F2991110FB01F09A4901EB88
:10C8C000C00000F552709DF8A01001EB410303EB8E
:10C8D000011100EBC10042714AE09DF8B41040F232
:10C8E000991011FB00F0904901EBC00000F5527067
:10C8F0009DF8A01001EB410202EB011100EBC10019
:10C90000807B012834D100229DF8B40040F29911B7
:10C9100010FB01F0844901EBC00101F552719DF853
:10C92000A00000EB400303EB001001EBC00082739A
:10C93000B6229DF8B40040F2991110FB01F07A493B
:10C9400001EBC00101F552719DF8A00000EB40031E
:10C9500003EB001001EBC000427100219DF8B40010
:10C9600040F2991210FB02F06F4A02EBC000017115
:10C97000B5E5D5229DF8B40040F2991110FB01F005
:10C98000694901EBC00101F552719DF8A00000EB6F
:10C99000400303EB001001EBC000427101219DF840
:10C9A000B40040F2991210FB02F05F4A02EBC000A3
:10C9B00001719DF8B41001EB410000EB01105B49DF
:10C9C00001EB001130319DF8A00001EB0010801C3C
:10C9D0000A90007820F0200020300A9908707EE547
:10C9E000D5229DF8B40040F2991110FB01F04E4998
:10C9F00001EBC00000F552709DF8A01001EB41035F
:10CA000003EB011100EBC100427168E59DF8B41021
:10CA100040F2991011FB00F0434901EBC00000F512
:10CA20005270BDF8D81001EB410202EB011100EB8E
:10CA3000C1008079012840D100229DF8B40040F265
:10CA4000991110FB01F0384901EBC00101F5527159
:10CA5000BDF8D80000EB400303EB001001EBC00071
:10CA60008271D5229DF8B40040F2991110FB01F0BB
:10CA70002D4901EBC00101F552719DF8A00000EBBA
:10CA8000400303EB001001EBC00042719DF8B410AD
:10CA900001EB410000EB0110244901EB00113031A2
:10CAA0009DF8A00001EB0010801C0A90007820F097
:10CAB0000400001D0A9908701FE0C3229DF8B4000D
:10CAC00040F2991110FB01F0174901EBC00101F58B
:10CAD00052719DF8A00000EB400303EB001001EB46
:10CAE000C000427100219DF8B40040F2991210FB81
:10CAF00002F00D4A02EBC0000171F0E49DF8B410A1
:10CB000040F2991011FB00F0074901EBC00000F55D
:10CB10005270BDF8D81001EB410202EB011100EB9D
:10CB2000C10005E064860020C444002004400020C9
:10CB30008079012840D100229DF8B40040F299117B
:10CB400010FB01F0FC4901EBC00101F55271BDF889
:10CB5000D80000EB400303EB001001EBC000827132
:10CB6000D5229DF8B40040F2991110FB01F0F24972
:10CB700001EBC00101F552719DF8A00000EB4003EC
:10CB800003EB001001EBC00042719DF8B41001EB03
:10CB9000410000EB0110E94901EB001130319DF833
:10CBA000A00001EB0010801C0A90007820F0040027
:10CBB000001D0A9908701FE0C3229DF8B40040F2DE
:10CBC000991110FB01F0DC4901EBC00101F5527134
:10CBD0009DF8A00000EB400303EB001001EBC00048
:10CBE000427100219DF8B40040F2991210FB02F04E
:10CBF000D14A02EBC000017171E49DF8B41001EB61
:10CC0000410000EB0110CD4901EB0010007B50BB4F
:10CC10009DF8B41001EB4100C0EBC110C84901EB15
:10CC2000C00001799DF8B40000EB4002C2EBC010D7
:10CC3000C34A02EBC000C07841EA00229DF8B4006C
:10CC400040F2991110FB01F0BB4901EBC00000F567
:10CC500052709DF8A01001EB410303EB011100EBB2
:10CC6000C100426335E09DF8B41001EB4100C0EB18
:10CC7000C110B34901EBC000C07801049DF8B400B5
:10CC800000EB4002C2EBC010AD4A02EBC0000079DD
:10CC900041EA00219DF8B40000EB4002C2EBC01055
:10CCA000A74A02EBC000407901439DF8B40040F26E
:10CCB000991210FB02F0A04A02EBC00000F552707E
:10CCC0009DF8A02002EB420303EB021200EBC2002E
:10CCD00041639DF8B41040F2991011FB00F09649A1
:10CCE00001EBC00101F552719DF8A00000EB40027C
:10CCF00002EB001011F830109DF8B40040F29912C8
:10CD000010FB02F08C4A02EBC0004079814234DA19
:10CD100000219DF8B40040F2991210FB02F0864AFF
:10CD200002EBC000017103229DF8B40040F299119A
:10CD300010FB01F0804901EBC00101F552719DF833
:10CD4000A00000EB400303EB001001F83020D922D3
:10CD50009DF8B40040F2991110FB01F0764901EB07
:10CD6000C00000F552709DF8A01001EB410303EBE9
:10CD7000011100EBC100427181E09DF8B41040F256
:10CD8000991011FB00F06C4901EBC00000F55270E6
:10CD9000BDF8D81001EB410202EB011100EBC1001C
:10CDA000807901284BD100229DF8B40040F29911FE
:10CDB00010FB01F0604901EBC00101F55271BDF8B3
:10CDC000D80000EB400303EB001001EBC0008271C0
:10CDD000D9229DF8B40040F2991110FB01F0564998
:10CDE00001EBC00101F552719DF8A00000EB40037A
:10CDF00003EB001001EBC00042719DF8B40000EBA2
:10CE0000400101EB00104D4901EB001130319DF85C
:10CE1000A00001EB0010801C0A90007820F00400B4
:10CE2000001D0A99087001209DF8B41040F2991273
:10CE300011FB02F1404A02EBC10108711FE0C5225B
:10CE40009DF8B40040F2991110FB01F03A4901EB52
:10CE5000C00101F552719DF8A00000EB400303EB07
:10CE6000001001EBC000427100219DF8B40040F2B7
:10CE7000991210FB02F0304A02EBC000017122E46B
:10CE800000219DF8B40040F2991210FB02F02A4AEA
:10CE900002EBC00001719DF8B40000EB400101EB12
:10CEA0000010264901EB001130319DF8A00001EB84
:10CEB0000010801C0A90007820F00400001D0A99E0
:10CEC0000870D5229DF8B40040F2991110FB01F0D2
:10CED000194901EBC00000F552709DF8A01001EB5C
:10CEE000410303EB011100EBC100427140E59DF8E5
:10CEF000B41001EB410000EB0110104901EB0010F0
:10CF0000007B88BBBDF8A4000C2800D030E50021D0
:10CF100039912FE09DF8B41001EB4100C0EBC11036
:10CF2000074901EBC001BDF8E400C01C085C00F03B
:10CF30000F00092806DD21E0C44400200440002041
:10CF4000648600209DF8B41001EB4100C0EBC110D5
:10CF5000FD4901EBC001BDF8E400C01C085C00F015
:10CF6000F000902801DD09E091E0BDF8E400401CEC
:10CF700081B23991BDF8E4000A28CBDB00BFBDF8CF
:10CF8000E4000A2800DAF3E400202E902F9000211C
:10CF900039911EE0DDE92E10000240EA116209021B
:10CFA000CDE92E129DF8B41001EB4100C0EBC11089
:10CFB000E54901EBC001BDF8E400C01C085CDDE9F7
:10CFC0002E341843CDE92E04BDF8E400401C80B295
:10CFD0003990BDF8E4000528DCDB9DF8B400DDE9FC
:10CFE0002E1240F2991310FB03F0D84B03EBC00351
:10CFF00003F552739DF8A00000EB400404EB001011
:10D0000003EBC00040F8221F426000222E922F92B4
:10D01000002139911EE0DDE92E10000240EA116284
:10D020000902CDE92E129DF8B41001EB4100C0EBCE
:10D03000C110C54901EBC001BDF8E4000830085C2F
:10D04000DDE92E341843CDE92E04BDF8E400401C80
:10D0500080B23990BDF8E4000528DCDB9DF8B4000F
:10D06000DDE92E1240F2991310FB03F0B74B03EBEE
:10D07000C00000F552709DF8A03003EB430404EBB0
:10D08000031300EBC30022308160C260BCE0BDF836
:10D09000A4000E2800D06BE40021399128E09DF80F
:10D0A000B41001EB4100C0EBC110A74901EBC00176
:10D0B000BDF8E400C01C085C00F00F00092800DD8A
:10D0C0001AE09DF8B41001EB4100C0EBC1109E497D
:10D0D00001EBC001BDF8E400C01C085C00F0F000EA
:10D0E000902800DD08E0BDF8E400401C81B23991D1
:10D0F000BDF8E4000C28D2DB00BFBDF8E4000C282A
:10D1000000DA35E400202E902F90002139911EE0A6
:10D11000DDE92E10000240EA11620902CDE92E126B
:10D120009DF8B41001EB4100C0EBC110864901EB42
:10D13000C001BDF8E400C01C085CDDE92E341843D2
:10D14000CDE92E04BDF8E400401C80B23990BDF852
:10D15000E4000628DCDB9DF8B400DDE92E2140F276
:10D16000991310FB03F0794B03EBC00303F55273E3
:10D170009DF8A00000EB400404EB001003EBC0009E
:10D1800040F8222F416000222E922F9200213991E7
:10D190001EE0DDE92E10000240EA11620902CDE92D
:10D1A0002E129DF8B41001EB4100C0EBC11066498E
:10D1B00001EBC001BDF8E4000930085CDDE92E3464
:10D1C0001843CDE92E04BDF8E400401C80B239902C
:10D1D000BDF8E4000628DCDB9DF8B400DDE92E2173
:10D1E00040F2991310FB03F0584B03EBC00000F51D
:10D1F00052709DF8A03003EB430404EB031300EBE3
:10D20000C30022308260C1609DF8B41040F29910D2
:10D2100011FB00F04D4901EBC00101F552719DF881
:10D22000A00000EB400202EB001011F830109DF856
:10D23000B40040F2991210FB02F0444A02EBC00025
:10D24000407981427ED19DF8B4009DF8A01001EB99
:10D250000010C217CDE92E023D4890F8900708B3A0
:10D260009DF8B41001EB410000EB0110394901EBCE
:10D27000001030309DF8A01000EB0110807A0228D9
:10D2800010D09DF8B41001EB410000EB01103149C2
:10D2900001EB001030309DF8A01000EB0110C07AB7
:10D2A00000287CDD00229DF8B40000EB400101EB7A
:10D2B0000010284901EB001030309DF8A01000EB61
:10D2C0000110C2722448D0F80C020521B0FBF1F223
:10D2D00001FB120000EB40011F482C3000EB411015
:10D2E0000D300A909DF8B40040F2991110FB01F046
:10D2F000164901EBC00000F552709DF8A01001EB3B
:10D30000410202EB011100EBC10022301022014664
:10D3100009900A98FAF799FF0F48D0F80C020521F6
:10D32000B0FBF1F201FB120000EB40010A482C3087
:10D3300000EB41129DF8B40040F2991110FB01F08E
:10D3400002490BE0DDE2000064860020C4440020B6
:10D35000BC32002004400020BC12002001EBC001C0
:10D3600001F552719DF8A00000EB400303EB0010A3
:10D3700001EBC00050F81A1F42F8011F40685060CE
:10D38000FE48D0F80C020521B0FBF1F201FB1200BF
:10D3900000EB4001F9482C3000EB411200E095E130
:10D3A0009DF8B40000EB400101EB0010F44901EBE3
:10D3B000001130319DF8A00001EB001000781070D2
:10D3C000EE48D0F80C020521B0FBF1F201FB12008F
:10D3D00000EB4001E9482C3000EB4111E9480268BC
:10D3E00041F81D2F80888880E448D0F80C02052180
:10D3F000B0FBF1F201FB120000EB4001DF482C30E2
:10D4000000EB41129DF8B40040F2991110FB01F0BD
:10D41000DD4901EBC00101F552719DF8A00000EB60
:10D42000400303EB001001EBC000406BC2F80900A1
:10D43000D248D0F80C020521B0FBF1F201FB12003A
:10D4400000EB4001CD482C3000EB41129DF8B400B8
:10D4500000EB400101EB0010C94901EB0011303134
:10D460009DF8A00001EB00104068C2F823000022E4
:10D470009DF8B40000EB400101EB0010C04901EB46
:10D48000001130319DF8A00001EB00104260002136
:10D49000399154E0B948D0F80C020521B0FBF1F203
:10D4A00001FB120000EB4001B4482C3000EB4111AD
:10D4B0002731BDF8E4409DF8B40040F2991210FB0A
:10D4C00002F0B14A02EBC00202F552729DF8A000D0
:10D4D00000EB400303EB001002EBC00090F880006B
:10D4E00040F2991210FB02F0A74A02EBC00202F5CB
:10D4F00052729DF8B40040F2991310FB03F0A24B56
:10D5000003EBC00303F552739DF8A00000EB400548
:10D5100005EB001003EBC00090F8810000EB400326
:10D5200003EB001002EBC0024732BDF8E400001D1F
:10D53000105C0855BDF8E400401C81B23991BDF87B
:10D54000E4000628A6DB0020399042E000239DF885
:10D55000B40040F2991110FB01F08B4901EBC001BE
:10D5600001F552719DF8A00000EB400202EB0010A3
:10D5700001EBC00090F8800040F2991110FB01F01F
:10D58000814901EBC00101F552719DF8B40040F2F0
:10D59000991210FB02F07C4A02EBC00202F55272B3
:10D5A0009DF8A00000EB400404EB001002EBC0006B
:10D5B00090F8810000EB400202EB001001EBC0018B
:10D5C0004731BDF8E4000B54BDF8E400401C81B2C3
:10D5D0003991BDF8E4000A28B8DB6848D0F80C029D
:10D5E0000521B0FBF1F080B201460A900220FBF762
:10D5F0006FFD00210620FCF71FFD6048D0F80C02EB
:10D600005E49498D884206D25C48D0F80C02401C25
:10D610005A49C1F80C0200210520FCF70DFD9DF8C8
:10D62000B41001EB410000EB0110554901EB001073
:10D6300030309DF8A01000EB0110801C0A9000789B
:10D6400020F00400001D0A9908704C48D0F80C0224
:10D650000521B0FBF1F201FB120000EB400147484D
:10D660002C3000EB4110D0F823202E9800EB400125
:10D67000464800EB4110C0F823200020399020E0FC
:10D680003E48D0F80C020521B0FBF1F201FB12007C
:10D6900000EB400139482C3000EB41102730BDF839
:10D6A000E410425C2E9800EB4001384800EB411139
:10D6B0002731BDF8E4000A54BDF8E400401C81B2F3
:10D6C0003991BDF8E4000628DADB65E09DF8B40086
:10D6D00000EB400101EB0010294901EB0010303054
:10D6E0009DF8A01000EB0110801C0A90007820F03B
:10D6F000080008300A9908709DF8B40000EB40015A
:10D7000001EB00101E4901EB001030309DF8A01015
:10D7100000EB011042682E9800EB40011B4800EB23
:10D720004110C0F823200020399025E09DF8B40076
:10D7300040F2991110FB01F0134901EBC00101F512
:10D7400052719DF8A00000EB400202EB001001EBCB
:10D75000C0014731BDF8E4000A5C2E9800EB40019F
:10D760000A4800EB41112731BDF8E4000A54BDF826
:10D77000E400401C81B239910AE00000BC12002094
:10D7800004400020C7310020C4440020D8140020E9
:10D79000BDF8E4000628C9DB9DF8B40000EB4001A9
:10D7A00001EB0010FE4901EB001030309DF8A01095
:10D7B00000EB0110801C0A90007820F020020A98EB
:10D7C00002709DF8B4100220FCF736FC9DF8B400FE
:10D7D00040F2991110FB01F0F24901EBC00000F595
:10D7E00052709DF8A01001EB410202EB011100EB19
:10D7F000C10022300A902E9800EB4001EA4800EB6D
:10D8000041100D30102209900A99FAF71EFD9DF87B
:10D81000B40040F2991110FB01F0E24901EBC001A4
:10D8200001F552719DF8A00000EB400202EB0010E0
:10D8300001EBC0012E9800EB4002DB4800EB4210E8
:10D8400051F81A2F40F8012F496841609DF8B40043
:10D8500000EB400101EB0010D14901EB0011303128
:10D860009DF8A00001EB001001782E9800EB40021B
:10D87000CD4800EB421001702E9800EB4001CA48E1
:10D8800000EB4111C948026841F81D2F808888804B
:10D890009DF8B40040F2991110FB01F0C14901EB71
:10D8A000C00101F552719DF8A00000EB400202EBAF
:10D8B000001001EBC000416B2E9800EB4002BA480B
:10D8C00000EB4210C0F809102E9881B208200A918E
:10D8D000FCF7B2FB00229DF8B40040F2991110FB56
:10D8E00001F0B04901EBC00000F552709DF8A010A6
:10D8F00001EB410303EB011100EBC10080F846206E
:10D9000053E09DF8B40000EB400101EB0010A44986
:10D9100001EB001030309DF8A01000EB0110801CCE
:10D920000A90007820F00400001D0A9908709DF804
:10D93000B40000EB400101EB0010994901EB00102D
:10D9400030309DF8A01000EB0110801C0A90007888
:10D9500020F0800080300A99087001209DF8B410F2
:10D9600040F2991211FB02F18E4A02EBC1010871DB
:10D970009DF8B40040F2991110FB01F0114601EB43
:10D98000C00042799DF8B40040F2991110FB01F0FB
:10D99000844901EBC00000F552709DF8A01001EB26
:10D9A000410303EB011100F83120D5229DF8B400AA
:10D9B00040F2991110FB01F07A4901EBC00000F52B
:10D9C00052709DF8A01001EB410303EB011100EB35
:10D9D000C10042718CE2D5229DF8B40040F2991149
:10D9E00010FB01F06F4901EBC00000F552709DF88B
:10D9F000A01001EB410303EB011100EBC1004271E8
:10DA000076E2D5229DF8B40040F2991110FB01F0A6
:10DA1000644901EBC00000F552709DF8A01001EBC5
:10DA2000410303EB011100EBC100427160E20121EF
:10DA30005E48F53080F8B4169DF8B40040F29911B4
:10DA400010FB01F0574901EBC00101F552719DF83F
:10DA5000A00000EB400202EB001011F830109DF81E
:10DA6000B40040F2991210FB02F04E4A02EBC000E3
:10DA70004079814234DA00219DF8B40040F29912D5
:10DA800010FB02F0474A02EBC000017101229DF831
:10DA9000B40040F2991110FB01F0424901EBC001C2
:10DAA00001F552719DF8A00000EB400303EB00105C
:10DAB00001F8302011229DF8B40040F2991110FBBA
:10DAC00001F0384901EBC00000F552709DF8A0103C
:10DAD00001EB410303EB011100EBC10042716AE06D
:10DAE0009DF8B41040F2991011FB00F02D4901EBA4
:10DAF000C00000F552709DF8A01001EB410202EB4E
:10DB0000011100EBC1008078B22835D100219DF8C9
:10DB1000B40040F2991210FB02F0224A02EBC0005E
:10DB20000171B2229DF8B40040F2991110FB01F08E
:10DB30001C4901EBC00101F552719DF8A00000EBFA
:10DB4000400303EB001001EBC000427100229DF87E
:10DB5000B40040F2991110FB01F0124901EBC00032
:10DB600000F552709DF8A01001EB410303EB011189
:10DB700000EBC10082701EE0D5229DF8B40040F297
:10DB8000991110FB01F0074901EBC00000F552703C
:10DB90009DF8A01001EB410303EB011108E0000028
:10DBA00004400020C4440020D8140020C7310020C5
:10DBB00000EBC10042719BE10021F74880F8B416E8
:10DBC000D5229DF8B40040F2991110FB01F0F34901
:10DBD00001EBC00000F552709DF8A01001EB41036D
:10DBE00003EB011100EBC100427181E101229DF8BC
:10DBF000B40040F2991110FB01F0E84901EBC001BB
:10DC000001F552719DF8A00000EB400303EB0010FA
:10DC100001EBC00080F882200021399129E09DF8B5
:10DC2000B41001EB4100C0EBC110DD4901EBC001B4
:10DC3000BDF8E400C01C0A5C9DF8B40040F29911E4
:10DC400010FB01F0D54901EBC00101F552719DF8BF
:10DC5000A00000EB400303EB001001EBC00000F15B
:10DC60008301BDF8E4000A54BDF8E400401C81B211
:10DC70003991BDF8E4000A28D1DB39E19DF8B410F0
:10DC800001EB4100C0EBC110C54901EBC000C078F9
:10DC900001049DF8B40000EB4002C2EBC010C04A82
:10DCA00002EBC000007941EA00209DF8B41001EBBE
:10DCB0004102C2EBC111BA4A02EBC10149790843E2
:10DCC000B0F5E13F6ED19DF8B41001EB410000EBDF
:10DCD0000110B44901EB001030309DF8A01000EBAA
:10DCE0000110801C0A90007820F004020A9802704B
:10DCF00000229DF8B40040F2991110FB01F0A749F1
:10DD000001EBC00000F552709DF8A01001EB41033B
:10DD100003EB011100EBC100A0F88E2013229DF847
:10DD2000B40040F2991110FB01F09C4901EBC000D6
:10DD300000F552709DF8A01001EB410303EB0111B7
:10DD400000EBC10042719DF8B41001EB410000EB03
:10DD50000110944901EB0010407903464FF48052C2
:10DD60004FF4E1310A909DF8B40018F04BFA9DF899
:10DD7000B41040F2991011FB00F0884901EBC0018A
:10DD800001F552719DF8A00000EB400202EB00107B
:10DD900001EBC00090300A90007820F008000830B5
:10DDA0000A990870A4E09DF8B41001EB4100C0EBA3
:10DDB000C1107B4901EBC00001799DF8B40000EB74
:10DDC0004002C2EBC010764A02EBC000C07841EAC4
:10DDD00000229DF8B40040F2991110FB01F06F4948
:10DDE00001EBC00101F552719DF8A00000EB40036A
:10DDF00003EB001001EBC000A0F88E209DF8B410DA
:10DE000040F2991011FB00F0644901EBC00101F5EB
:10DE100052719DF8A00000EB400202EB001001EBF4
:10DE2000C000B0F88E109DF8B40000EB400202EB89
:10DE300000105C4A02EB0010408B814257DBE52268
:10DE40009DF8B40040F2991110FB01F0534901EB29
:10DE5000C00101F552719DF8A00000EB400303EBF7
:10DE6000001001EBC000427100229DF8B40040F2A6
:10DE7000991110FB01F0494901EBC00101F5527104
:10DE80009DF8A00000EB400303EB001001F83020E8
:10DE90009DF8B40000EB400101EB0010414901EB9B
:10DEA000001130319DF8A00001EB0010801C0A9099
:10DEB000007820F080020A9802709DF8B40040F2C9
:10DEC000991110FB01F0354901EBC00000F55270CB
:10DED0009DF8A01001EB410202EB011100EBC10023
:10DEE00090300A90007820F001020A98027000BF7A
:10DEF00000BF0FF02CBA9DF8B40000EB4001C1EB5D
:10DF0000C010274911F83000042801D126900BE0F9
:10DF10009DF8B40000EB4001C1EBC010204911F89E
:10DF20003000152800D126909DF8B40000EB400188
:10DF3000C1EBC0101A4901EBC00041789DF8B40054
:10DF400000EB4002C2EBC010154A12F8300041EA63
:10DF5000002041F23001884202D1A620269045E0FF
:10DF60009DF8B40000EB4001C1EBC0100C4901EB7F
:10DF7000C00041789DF8B40000EB4002C2EBC01035
:10DF8000074A12F8300041EA002041F2310188428C
:10DF90000AD1A720269029E0BC320020C4440020EA
:10DFA00064860020044000209DF8B40000EB40018E
:10DFB000C1EBC010FC4911F83000022816D19DF8C1
:10DFC000B40000EB4001C1EBC010F74901EBC00009
:10DFD00001799DF8B40000EB4002C2EBC010F24A98
:10DFE00002EBC000C07841EA002126919DF8B40000
:10DFF00040F2991110FB01F0EC4901EBC00081786F
:10E0000028910021EA4A9DF8B40002EB00129DF825
:10E01000A0001154E74890F82800012815D19DF878
:10E02000B40000EB400101EB0010E34901EB0010EC
:10E0300030309DF8A01000EB0110801C0A90007891
:10E0400020F0800080300A990870BDF8981043F2E3
:10E050003002881A91427CD009DC04297AD0152933
:10E0600079D0A62910D0A72942F0F0825CE1B0F562
:10E07000C06F71D0A0F2016000286ED001286DD071
:10E080000428F1D101F078BE00219DF8B40040F2DF
:10E09000991210FB02F0C54A02EBC00001719DF815
:10E0A000B40040F2991110FB01F0114601EBC000E1
:10E0B00000F552709DF8A01001EB410202EB011136
:10E0C00010F83100052829DC06229DF8B40040F242
:10E0D000991110FB01F0B54901EBC00101F5527136
:10E0E0009DF8A00000EB400303EB001001F8302086
:10E0F000A8229DF8B40040F2991110FB01F0AB4941
:10E1000001EBC00000F552709DF8A01001EB410337
:10E1100003EB011100EBC100427103E19DF8B40073
:10E1200040F2991110FB01F0A04901EBC00000F58D
:10E1300052709DF8A01001EB410202EB011110F8A2
:10E1400031000A2830DC0B229DF8B40040F299110E
:10E1500005E0B9E138E2F4E3F4E3F4E3F4E310FBBF
:10E1600001F0924901EBC00101F552719DF8A00048
:10E1700000EB400303EB001001F83020A9229DF8CA
:10E18000B40040F2991110FB01F0884901EBC00086
:10E1900000F552709DF8A01001EB410303EB011153
:10E1A00000EBC1004271BDE09DF8B40040F299114E
:10E1B00010FB01F07D4901EBC00000F552709DF8A5
:10E1C000A01001EB410202EB011110F831000F2801
:10E1D00029DC10229DF8B40040F2991110FB01F0E7
:10E1E000724901EBC00101F552719DF8A00000EBEE
:10E1F000400303EB001001F83020A2229DF8B40088
:10E2000040F2991110FB01F0684901EBC00000F5E4
:10E2100052709DF8A01001EB410303EB011100EBDC
:10E22000C10042717EE09DF8B41040F2991011FBDC
:10E2300000F05E4901EBC00000F552709DF8A0109F
:10E2400001EB410202EB011100EBC1004079A5286E
:10E2500015D19DF8B40000EB400101EB00105649C8
:10E2600001EB001030309DF8A01000EB0110801C75
:10E270000A90007820F00400001D0A9908709DF8AB
:10E28000B40040F2991110FB01F0484901EBC000C5
:10E2900000F552709DF8A01001EB410202EB011154
:10E2A00000EBC1008078A1283CD09DF8B40040F27A
:10E2B000991110FB01F03D4901EBC00101F55271CC
:10E2C0009DF8A00000EB400202EB001001EBC00043
:10E2D00082789DF8B40040F2991110FB01F03349A7
:10E2E00001EBC00101F552719DF8A00000EB400365
:10E2F00003EB001001EBC0004271A1229DF8B400B5
:10E3000040F2991110FB01F0284901EBC00000F523
:10E3100052709DF8A01001EB410303EB011100EBDB
:10E32000C100827002F092B900219DF8B40040F261
:10E33000991210FB02F01D4A02EBC00001719DF81A
:10E34000B41040F2991011FB00F0114601EBC0002F
:10E3500000F552709DF8A01001EB410202EB011193
:10E3600010F83100082829DC00219DF8B40040F2A3
:10E37000991210FB02F00D4A02EBC0000171082255
:10E380009DF8B40040F2991110FB01F0074901EB30
:10E39000C00000F552709DF8A01001EB410303EBA3
:10E3A000011100F8312032E064860020C4440020CE
:10E3B000383E0020BC120020044000209DF8B4101C
:10E3C00040F2991011FB00F0FE4901EBC00000F58E
:10E3D00052709DF8A01001EB410202EB011110F800
:10E3E00031000B2813DC0C229DF8B40040F2991187
:10E3F00010FB01F0F34901EBC00000F552709DF8ED
:10E40000A01001EB410303EB011100F831209DF84E
:10E41000B41040F2991011FB00F0EA4901EBC00082
:10E4200000F552709DF8A01001EB410202EB0111C2
:10E4300000EBC1004079A42830D19DF8B41001EB65
:10E44000410000EB0110E04901EB001030309DF875
:10E45000A01000EB0110801C0A90007820F0200032
:10E4600020300A99087000229DF8B40040F29911FA
:10E4700010FB01F0D34901EBC00000F552709DF88C
:10E48000A01001EB410303EB011100EBC10080F888
:10E4900045209DF8B4100220FBF7CEFDA1229DF887
:10E4A000B40040F2991110FB01F0C64901EBC00025
:10E4B00000F552709DF8A01001EB410303EB011130
:10E4C00000EBC10042712DE70020399015E09DF866
:10E4D000B41001EB4100C0EBC110BC4901EBC0011D
:10E4E000BDF8E400C01C095C17AABDF8E400115493
:10E4F000BDF8E400401C81B23991BDF8E400062863
:10E50000E5DB062117A826F06FFF0021CDE93001D9
:10E51000DDE93021100A40EA0164309BE21841EB4A
:10E520002120CDE908204FF480724FF00003DDE98F
:10E530000801F9F747FE9DF8B40040F2991110FB6D
:10E5400001F0A04901EBC00000F552709DF8A01049
:10E5500001EB410303EB011100EBC100027100204C
:10E560009DF8B41040F2991211FB02F1954A02EBAA
:10E57000C101087104229DF8B40040F2991110FB0A
:10E5800001F0904901EBC00000F552709DF8A01019
:10E5900001EB410303EB011100F83120A7229DF8A4
:10E5A000B40040F2991110FB01F0864901EBC00064
:10E5B00000F552709DF8A01001EB410303EB01112F
:10E5C00000EBC1004271ADE69DF8B41040F2991025
:10E5D00011FB00F07B4901EBC00000F552709DF883
:10E5E000A01001EB410202EB011110F831000428E8
:10E5F00078DA00219DF8B40040F2991210FB02F085
:10E60000704A02EBC0000171A1229DF8B40040F2F3
:10E61000991110FB01F06B4901EBC00101F552713A
:10E620009DF8A00000EB400303EB001001EBC000DD
:10E6300042719DF8B41040F2991011FB00F061494D
:10E6400001EBC00101F552719DF8A00000EB400202
:10E6500002EB001001EBC0010A910878401CC1B226
:10E660000A9801709DF8B41040F2991011FB00F067
:10E67000544901EBC00000F552709DF8A01001EB69
:10E68000410202EB011110F83100042828D10A22BE
:10E690009DF8B40040F2991110FB01F0494901EBDB
:10E6A000C00101F552719DF8A00000EB400303EB9F
:10E6B000001001F83020A3229DF8B40040F2991117
:10E6C00010FB01F03F4901EBC00000F552709DF8CE
:10E6D000A01001EB410303EB011100EBC1004271FB
:10E6E000E5E2FFE79DF8B41040F2991011FB00F04D
:10E6F000344901EBC00000F552709DF8A01001EB09
:10E70000410202EB011110F83100042834D100213C
:10E710009DF8B40040F2991210FB02F0294A02EB76
:10E72000C000017105229DF8B40040F2991110FB60
:10E7300001F0244901EBC00101F552719DF8A000E0
:10E7400000EB400303EB001001F83020A3229DF8FA
:10E75000B40040F2991110FB01F01A4901EBC0001E
:10E7600000F552709DF8A01001EB410303EB01117D
:10E7700000EBC10042719AE29DF8B41040F299108A
:10E7800011FB00F00F4901EBC00000F552709DF83D
:10E79000A01001EB410202EB011110F83100082832
:10E7A0003BDC00219DF8B40040F2991210FB02F00E
:10E7B000044A02EBC000017109229DF8B40040F246
:10E7C000991105E0C4440020044000206486002024
:10E7D00010FB01F0FE4901EBC00101F552719DF8FB
:10E7E000A00000EB400303EB001001F83020A7224B
:10E7F0009DF8B40040F2991110FB01F0F44901EBCF
:10E80000C00000F552709DF8A01001EB410303EB2E
:10E81000011100EBC100427149E29DF8B41040F2D1
:10E82000991011FB00F0EA4901EBC00000F55270AD
:10E830009DF8A01001EB410202EB011110F831002C
:10E84000092834DC00219DF8B40040F2991210FB35
:10E8500002F0DF4A02EBC00001710A229DF8B40009
:10E8600040F2991110FB01F0D94901EBC00101F50B
:10E8700052719DF8A00000EB400303EB001001F87B
:10E880003020A3229DF8B40040F2991110FB01F052
:10E89000CF4901EBC00000F552709DF8A01001EBCC
:10E8A000410303EB011100EBC1004271FFE19DF850
:10E8B000B41040F2991011FB00F0C54901EBC00003
:10E8C00000F552709DF8A01001EB410202EB01111E
:10E8D00010F831000D2838DC00219DF8B40040F21A
:10E8E000991210FB02F0BA4A02EBC00001710E222D
:10E8F0009DF8B40040F2991110FB01F0B44901EB0E
:10E90000C00101F552719DF8A00000EB400303EB3C
:10E91000001001F83020A1229DF8B40040F29911B6
:10E9200010FB01F0AA4901EBC00000F552709DF800
:10E93000A01001EB410303EB011100EBC100427198
:10E94000B5E1B5E1E9E13EE21CE29DF8B41040F228
:10E95000991011FB00F09E4901EBC00000F55270C8
:10E960009DF8A01001EB410202EB011110F83100FB
:10E970000E2834DC00219DF8B40040F2991210FBFF
:10E9800002F0934A02EBC00001710F229DF8B4001F
:10E9900040F2991110FB01F08D4901EBC00101F526
:10E9A00052719DF8A00000EB400303EB001001F84A
:10E9B0003020A3229DF8B40040F2991110FB01F021
:10E9C000834901EBC00000F552709DF8A01001EBE7
:10E9D000410303EB011100EBC100427167E19DF8B7
:10E9E000B41040F2991011FB00F0794901EBC0001E
:10E9F00000F552709DF8A01001EB410202EB0111ED
:10EA000010F8310010287DDC11229DF8B40040F28E
:10EA1000991110FB01F06E4901EBC00101F5527133
:10EA20009DF8A00000EB400303EB001001F830203C
:10EA3000A1229DF8B40040F2991110FB01F0644945
:10EA400001EBC00101F552719DF8A00000EB4003FD
:10EA500003EB001001EBC00042719DF8B40040F2DE
:10EA6000991110FB01F05A4901EBC00101F55271F7
:10EA70009DF8A00000EB400303EB001001EBC00089
:10EA800082709DF8B41001EB410000EB0110514978
:10EA900001EB001130319DF8A00001EB0010801C4B
:10EAA0000A90007820F0800080300A9908709DF864
:10EAB000B41001EB410000EB0110464901EB0010DE
:10EAC00030309DF8A01000EB0110801C0A900078F7
:10EAD00020F00400001D0A9908709DF8B41001EBA5
:10EAE000410000EB01103B4901EB001030309DF874
:10EAF000A01000EB01108078C0F34010F0B39DF837
:10EB0000B41000E042E001EB410000EB011031499C
:10EB100001EB001030309DF8A01000EB0110801CBC
:10EB20000A90007820F020020A9802709DF8B41034
:10EB300001EB410000EB0110264901EB00103030E1
:10EB40009DF8A01000EB01108078C0F34000B8B928
:10EB50009DF8B41001EB410000EB01101D4901EBE1
:10EB6000001030309DF8A01000EB0110801C0A90BE
:10EB7000007820F0080008300A9900E076E008707C
:10EB80009DF8B4100220FBF757FA90E09DF8B410FE
:10EB900040F2991011FB00F00D4901EBC00101F5A5
:10EBA00052719DF8A00000EB400202EB001011F83A
:10EBB00030109DF8B40040F2991210FB02F0044AA4
:10EBC00002EBC0004079814271D19DF8B41003E09E
:10EBD000C44400200440002040F2991011FB00F0D2
:10EBE000114601EBC00000F552709DF8A01001EB3A
:10EBF000410202EB011100EBC1008078A12836D060
:10EC0000A3229DF8B40040F2991110FB01F0F849DD
:10EC100001EBC00101F552719DF8A00000EB40032B
:10EC200003EB001001EBC00042719DF8B41040F2FC
:10EC3000991011FB00F0EE4901EBC00000F5527095
:10EC40009DF8A01001EB410202EB011100EBC100A5
:10EC50008078A2282BD000209DF8B41040F29912A1
:10EC600011FB02F1E24A02EBC10108711FE0A1228F
:10EC70009DF8B40040F2991110FB01F0DC4901EB62
:10EC8000C00101F552719DF8A00000EB400303EBB9
:10EC9000001001EBC000427101219DF8B40040F268
:10ECA000991210FB02F0D24A02EBC00001710AE493
:10ECB000A1229DF8B40040F2991110FB01F0CC495B
:10ECC00001EBC00101F552719DF8A00000EB40037B
:10ECD00003EB001001EBC00082709DF8B40040F21D
:10ECE000991110FB01F0C24901EBC00101F552710D
:10ECF0009DF8A00000EB400303EB001001EBC00007
:10ED0000427100219DF8B40040F2991210FB02F00C
:10ED1000B74A02EBC000017155E400219DF8B40030
:10ED200040F2991210FB02F0B14A02EBC0000171EF
:10ED300009229DF8B40040F2991110FB01F0AC4992
:10ED400001EBC00101F552719DF8A00000EB4003FA
:10ED500003EB001001F83020A7229DF8B40040F228
:10ED6000991110FB01F0A24901EBC00000F55270AF
:10ED70009DF8A01001EB410303EB011100EBC10072
:10ED8000427120E400219DF8B40040F2991210FB7A
:10ED900002F0974A02EBC0000171A7229DF8B4006F
:10EDA00040F2991110FB01F0914901EBC00000F510
:10EDB00052709DF8A01001EB410303EB011100EB31
:10EDC000C100427173E700219DF8B40040F299122E
:10EDD00010FB02F0864A02EBC0000171A7229DF8E9
:10EDE000B40040F2991110FB01F0814901EBC00120
:10EDF00001F552719DF8A00000EB400303EB0010F9
:10EE000001EBC00042719DF8B41001EB4100C0EB72
:10EE1000C110784901EBC000407930287ED19DF8BF
:10EE2000B41040F2991011FB00F0714901EBC001E0
:10EE300001F552719DF8A00000EB400202EB0010BA
:10EE400011F830109DF8B40040F2991210FB02F056
:10EE5000674A02EBC000407981425FD19DF8B4005F
:10EE600040F2991110FB01F0114601EBC00000F5D2
:10EE700052709DF8A01001EB410202EB011100EB72
:10EE8000C100C078312830D19DF8B40000EB4001BA
:10EE900001EB0010584901EB001030309DF8A01034
:10EEA00000EB0110801C0A90007820F020020A98E4
:10EEB000027000229DF8B40040F2991110FB01F09D
:10EEC0004B4901EBC00000F552709DF8A01001EB1A
:10EED000410303EB011100EBC10080F845209DF8D0
:10EEE000B4100220FBF7A8F857E09DF8B40040F2F8
:10EEF000991110FB01F03E4901EBC00000F5527082
:10EF00009DF8A01001EB410202EB011100EBC100E2
:10EF1000C078332841D19DF8B40000E06EE000EBEA
:10EF2000400101EB0010344901EB001030309DF836
:10EF3000A01000EB0110801C0A90007820F0200245
:10EF40000A98027001229DF8B40040F2991110FB5A
:10EF500001F0274901EBC00000F552709DF8A010A8
:10EF600001EB410303EB011100EBC10080F84620E7
:10EF7000A9229DF8B40040F2991110FB01F01C4940
:10EF800001EBC00000F552709DF8A01001EB4103A9
:10EF900003EB011100EBC10082709DF8B40000EB9F
:10EFA000400101EB0010144901EB001030309DF8D6
:10EFB000A01000EB0110801C0A90007820F00102E4
:10EFC0000A9802709DF8B40000EB400101EB0010BC
:10EFD000094901EB001030309DF8A01000EB011042
:10EFE000801C0A90007820F002020A980270DBE38D
:10EFF000C444002064860020044000209DF8B40032
:10F0000000EB4001C1EBC010FE4901EBC0004079AC
:10F0100031287CD19DF8B40040F2991110FB01F029
:10F02000F94901EBC00101F552719DF8A00000EB18
:10F03000400202EB001011F830109DF8B40040F2CD
:10F04000991210FB02F0F04A02EBC00040798142B5
:10F05000DFD19DF8B41040F2991011FB00F0114679
:10F0600001EBC00000F552709DF8A01001EB4102C9
:10F0700002EB011100EBC10090F8460058BB0122E1
:10F080009DF8B40040F2991110FB01F0DE4901EB4C
:10F09000C00101F552719DF8A00000EB400303EBA5
:10F0A000001001EBC00080F845209DF8B41001EB82
:10F0B000410000EB0110D54901EB001130319DF802
:10F0C000A00001EB0010801C0A90007820F00100E5
:10F0D000401C0A9908709DF8B41001EB410000EB48
:10F0E0000110CA4901EB001030309DF8A01000EB70
:10F0F0000110801C0A90007820F002020A98027029
:10F10000C34890F8900790B19DF8B41000E006E273
:10F1100001EB410000EB0110BC4901EB0010303065
:10F120009DF8A01000EB0110807A022877D1B94831
:10F1300090F829000128F9D1B648D0F80C02B54959
:10F14000498D88426BD29DF8B41040F2991011FBA2
:10F1500000F0AD4901EBC00000F552709DF8A01021
:10F1600001EB410202EB011100EBC10090F84500F8
:10F17000012853D19DF8B41040F2991011FB00F012
:10F18000A14901EBC00000F552709DF8A01001EB01
:10F19000410202EB011100EBC10090F87F00E8BBD7
:10F1A00001229DF8B40000EB400101EB00109749EB
:10F1B00001EB001130319DF8A00001EB0010C2728C
:10F1C00000229DF8B40000EB400101EB00108F49D4
:10F1D00001EB001130319DF8A00001EB00104260FE
:10F1E0004FF010429DF8B40040F2991110FB01F06D
:10F1F000854901EBC00101F552719DF8A00000EBBB
:10F20000400303EB001001EBC00082609DF8B410D6
:10F2100001EB410000EB01107C4901E071E06FE07F
:10F2200001EB001130319DF8A00001EB00100178D6
:10F230009DF8B40040F2991210FB02F0724A02EB02
:10F24000C00041709DF8B41040F2991011FB00F01D
:10F25000114601EBC00101F552719DF8A00000EBD1
:10F26000400202EB001011F830109DF8B40040F29B
:10F27000991210FB02F0644A02EBC000407981420F
:10F280003ED100229DF8B40040F2991110FB01F02C
:10F290005D4901EBC00101F552719DF8A00000EB42
:10F2A000400303EB001001EBC000C271A4229DF8E3
:10F2B000B40040F2991110FB01F0534901EBC00179
:10F2C00001F552719DF8A00000EB400303EB001024
:10F2D00001EBC0008270A3229DF8B40040F29911A6
:10F2E00010FB01F0484901EBC00000F552709DF899
:10F2F000A01001EB410303EB011100EBC1004271CF
:10F3000052E29DF8B41040F2991011FB00F03E4912
:10F3100001EBC00000F552709DF8A01001EB410216
:10F3200002EB011100EBC10090F84500012873D1F8
:10F330009DF8B41040F2991011FB00F0324901EB36
:10F34000C00101F552719DF8A00000EB400202EBF4
:10F35000001001EBC00090F8801040F2991011FBF2
:10F3600000F0294901EBC00101F552719DF8B4008C
:10F3700040F2991210FB02F0234A02EBC00000F5A4
:10F3800052709DF8A02002EB420303EB021200EB47
:10F39000C20090F8810000EB400202EB001001EB8C
:10F3A000C00090F87E00032836D102229DF8B400F8
:10F3B00000EB400101EB0010144901EB001130316A
:10F3C0009DF8A00001EB0010C2724FF010429DF8B2
:10F3D000B40040F2991110FB01F00B4901EBC001A0
:10F3E00001F552719DF8A00000EB400303EB001003
:10F3F00001EBC00082609DF8B41001EB410000EB0E
:10F4000001100AE064860020C4440020044000206B
:10F41000BC320020BC120020B9E1FE4901EB001112
:10F4200030319DF8A00001EB001001789DF8B40088
:10F4300040F2991210FB02F0F74A02EBC000417053
:10F440009DF8B41040F2991011FB00F0114601EB49
:10F45000C00101F552719DF8A00000EB400202EBE3
:10F46000001011F830109DF8B40040F2991210FB12
:10F4700002F0E94A02EBC000407981423ED100220D
:10F480009DF8B40040F2991110FB01F0E24901EB44
:10F49000C00101F552719DF8A00000EB400303EBA1
:10F4A000001001EBC000C271A4229DF8B40040F22C
:10F4B000991110FB01F0D84901EBC00101F552711F
:10F4C0009DF8A00000EB400303EB001001EBC0002F
:10F4D0008270A3229DF8B40040F2991110FB01F054
:10F4E000CD4901EBC00000F552709DF8A01001EB72
:10F4F000410303EB011100EBC100427100229DF8B2
:10F50000B40000EB400101EB0010C24901EB001018
:10F5100030309DF8A01000EB0110426044E19DF8EE
:10F52000B41001EB4100C0EBC110BC4901EBC000BD
:10F53000407933287ED19DF8B41001EB410000EBF7
:10F540000110B44901EB001030309DF8A01000EB21
:10F550000110801C0A90007820F00101491C0A98D3
:10F5600001709DF8B41001EB410000EB0110A949B6
:10F5700001EB001130319DF8A00001EB0010801C60
:10F580000A90007820F020020A9802709DF8B410CA
:10F5900001EB410000EB01109E4901EB00103030FF
:10F5A0009DF8A01000EB0110801C0A90007820F05C
:10F5B0000200801C0A9908709DF8B41040F299105E
:10F5C00011FB00F0944901EBC00042799DF8B400B2
:10F5D00040F2991110FB01F08F4901EBC00000F5DA
:10F5E00052709DF8A01001EB410303EB011100F8EC
:10F5F00031209DF8B41001EB410000EB011085496A
:10F6000001EB001030309DF8A01000EB0110801CC1
:10F610000A90007820F0800080300A9908709DF8E8
:10F62000B41001EB410000EB01107A4901EB00102E
:10F63000303000E022E09DF8A01000EB011080784F
:10F64000C0F3400020B99DF8B4100220FAF7F4FC92
:10F65000A2229DF8B40040F2991110FB01F06E490E
:10F6600001EBC00000F552709DF8A01001EB4103C2
:10F6700003EB011100EBC100827095E09DF8B4101E
:10F6800001EB4100C0EBC110644901EBC0004079BF
:10F6900034287CD19DF8B41001EB410000EB01103F
:10F6A0005C4901EB001030309DF8A01000EB011018
:10F6B000801C0A90007820F020020A9802709DF8C1
:10F6C000B41001EB410000EB0110524901EB0010B6
:10F6D00030309DF8A01000EB0110801C0A900078DB
:10F6E00020F002020A98027001229DF8B40040F254
:10F6F000991110FB01F0484901EBC00000F5527070
:10F700009DF8A01001EB410303EB011100EBC100D8
:10F7100080F84620A9229DF8B40040F2991110FB10
:10F7200001F03D4901EBC00000F552709DF8A010BA
:10F7300001EB410303EB011100EBC10082709DF866
:10F74000B41040F2991011FB00F0334901EBC000F6
:10F7500042799DF8B40040F2991110FB01F02E4956
:10F7600001EBC00000F552709DF8A01001EB4103C1
:10F7700003EB011100F831209DF8B41001EB4100BA
:10F7800000EB0110234901EB0010303000E00BE0EA
:10F790009DF8A01000EB0110801C0A90007820F06A
:10F7A000800080300A99087000202E902F90002150
:10F7B000399122E0DDE92E10000140EA11720901C1
:10F7C000CDE92E129DF8B41001EB4100C0EBC11041
:10F7D000124901EBC001BDF8E400801D085C30381F
:10F7E000C117DDE92E34184341EA0402CDE92E02A7
:10F7F000BDF8E400401C80B23990BDF8E400062852
:10F80000D8DB9DF8B4002E9940F2991210FB02F05B
:10F81000014A05E004400020C44400206486002022
:10F8200002EBC00202F552729DF8A00000EB40030B
:10F8300003EB001002EBC000C0F81A1000222E9259
:10F840002F920021399122E0DDE92E10000140EADB
:10F8500011720901CDE92E129DF8B40000EB4001B0
:10F86000C1EBC010FE4901EBC001BDF8E4000D3052
:10F87000085C3038C117DDE92E34184341EA040230
:10F88000CDE92E02BDF8E400401C80B23990BDF8ED
:10F89000E4000428D8DB9DF8B4002E9940F29912B8
:10F8A00010FB02F0EF4A02EBC00202F552729DF823
:10F8B000A00000EB400303EB001002EBC00041632B
:10F8C00000222E922F920021399122E0DDE92E10A4
:10F8D000000140EA11720901CDE92E129DF8B41021
:10F8E00001EB4100C0EBC110DD4901EBC001BDF8E7
:10F8F000E4001130085C3038C117DDE92E341843BC
:10F9000041EA0402CDE92E02BDF8E400401C80B2B9
:10F910003990BDF8E4000628D8DB9DF8B4002E9994
:10F9200040F2991210FB02F0CE4A02EBC00202F53F
:10F9300052729DF8A00000EB400303EB001002EBB5
:10F94000C000C0F81E109DF8B41001EB4100C0EBE0
:10F95000C110C34901EBC00042799DF8B40040F2E8
:10F96000991110FB01F0BF4901EBC00101F5527183
:10F970009DF8A00000EB400303EB001001EBC0007A
:10F98000C2709DF8B41001EB410000EB0110B649C4
:10F9900001EB001130319DF8A00001EB00108278DE
:10F9A0009DF8B40040F2991110FB01F0AD4901EB54
:10F9B000C00101F552719DF8A00000EB400303EB7C
:10F9C000001001EBC00002769DF8B41040F29910CF
:10F9D00011FB00F0A34901EBC00101F552719DF844
:10F9E000A00000EB400202EB001011F830109DF86F
:10F9F000B40040F2991210FB02F09A4A02EBC000E8
:10FA0000407981427EDA9DF8B41040F2991011FBE2
:10FA100000F0114601EBC00000F552709DF8A010F7
:10FA200001EB410202EB011110F831000F2869DDF2
:10FA300000219DF8B40040F2991210FB02F0894AAF
:10FA400002EBC0000171A7229DF8B40040F29911A9
:10FA500010FB01F0834901EBC00101F552719DF8E3
:10FA6000A00000EB400303EB001001EBC00042716B
:10FA700001219DF8B40040F2991210FB02F0794A7E
:10FA800002EBC00001719DF8B41040F2991011FB17
:10FA900000F0114601EBC00042799DF8B40040F23D
:10FAA000991110FB01F06F4901EBC00101F5527192
:10FAB0009DF8A00000EB400303EB001001F830209C
:10FAC000A1229DF8B40040F2991110FB01F06549A4
:10FAD00001EBC00101F552719DF8A00000EB40035D
:10FAE00003EB001001EBC00042719DF8B41001EB74
:10FAF000410000EB01105C4901EB001130319DF831
:10FB0000A00000E082E001EB0010801C0A90007869
:10FB100020F0800080300A9908709DF8B41001EB45
:10FB2000410000EB0110504901EB001030309DF80E
:10FB3000A01000EB0110801C0A90007820F0040057
:10FB4000001D0A9908709DF8B41001EB410000EB0C
:10FB50000110454901EB001030309DF8A01000EB7A
:10FB600001108078C0F3401088B99DF8B41001EB03
:10FB7000410000EB01103C4901EB001030309DF8D2
:10FB8000A01000EB01108078C0F34000F0B39DF8A6
:10FB9000B41001EB410000EB0110334901EB001000
:10FBA00030309DF8A01000EB0110801C0A90007806
:10FBB00020F020020A9802709DF8B41001EB410079
:10FBC00000EB0110284901EB001030309DF8A01027
:10FBD00000EB0110801C0A90007820F002020A98C5
:10FBE00002709DF8B41001EB410000EB01101E49BA
:10FBF00001EB001030309DF8A01000EB0110801CCC
:10FC00000A90007820F00800083000E0B3E00A997C
:10FC100008709DF8B4009DF8A01001EB0010C21709
:10FC2000CDE92E029DF8B41040F2991011FB00F0BE
:10FC30000C4901EBC00000F552709DF8A01001EBDB
:10FC4000410202EB011100EBC10022300A902E9814
:10FC500000EB4001054800EB41100D30102207E099
:10FC600064860020C444002004400020D8140020F2
:10FC700009900A99F8F7E9FA9DF8B41040F2991042
:10FC800011FB00F0FD4901EBC00101F552719DF837
:10FC9000A00000EB400202EB001001EBC0012E9827
:10FCA00000EB4002F64800EB421051F81A2F40F8E2
:10FCB000012F496841609DF8B41001EB410000EB51
:10FCC0000110F04901EB001130319DF8A00001EB6B
:10FCD000001001782E9800EB4002E94800EB42103A
:10FCE00001702E9800EB4001E54800EB4111E64819
:10FCF000026841F81D2F808888809DF8B41040F27A
:10FD0000991011FB00F0DD4901EBC00101F55271C2
:10FD10009DF8A00000EB400202EB001001EBC000D8
:10FD2000416B2E9800EB4002D54800EB4210C0F822
:10FD300009109DF8B41001EB410000EB0110D1490E
:10FD400001EB001130319DF8A00001EB001041687B
:10FD50002E9800EB4002CA4800EB4210C0F8231076
:10FD60002E9881B208200A91FAF766F99DF8B4102E
:10FD70000220FAF761F9FCE300202E902F90002179
:10FD8000399122E0DDE92E10000140EA11720901EB
:10FD9000CDE92E129DF8B41001EB4100C0EBC1106B
:10FDA000BA4901EBC001BDF8E4000B30085C303803
:10FDB000C117DDE92E34184341EA0402CDE92E02D1
:10FDC000BDF8E400401C80B23990BDF8E4000A2878
:10FDD000D8DB9DF8B400DDE92E1240F2991310FB38
:10FDE00003F0A64B03EBC00303F552739DF8A0008C
:10FDF00000EB400404EB001003EBC00040F8221FAE
:10FE0000426000222E922F920021399122E0DDE9FA
:10FE10002E10000140EA11720901CDE92E129DF861
:10FE2000B41001EB4100C0EBC110984901EBC001D7
:10FE3000BDF8E4001530085C3038C117DDE92E3418
:10FE4000184341EA0402CDE92E02BDF8E400401C4B
:10FE500080B23990BDF8E4000A28D8DB9DF8B400E0
:10FE6000DDE92E1240F2991310FB03F0834B03EBF4
:10FE7000C00303F552739DF8A00000EB400404EBAF
:10FE8000001003EBC00022308160C26000219DF8A9
:10FE9000B40040F2991210FB02F0784A02EBC00065
:10FEA00001719DF8B41040F2991011FB00F0114659
:10FEB00001EBC00000F552709DF8A01001EB41026B
:10FEC00002EB011110F831000C2814DC0D229DF812
:10FED000B40040F2991110FB01F0684901EBC00039
:10FEE00000F552709DF8A01001EB410303EB0111E6
:10FEF00000F831207FE39DF8B40040F2991110FB27
:10FF000001F05E4901EBC00101F552719DF8A000BE
:10FF100000EB400202EB001011F830109DF8B40025
:10FF200040F2991210FB02F0544A02EBC0004079F3
:10FF30008142DFD19DF8B4009DF8A01001EB0010C4
:10FF4000C217CDE92E025048F53090F8900708B35B
:10FF50009DF8B40000EB400101EB0010494901EBB2
:10FF6000001030309DF8A01000EB0110807A0228BC
:10FF700010D09DF8B40000EB400101EB00104149A6
:10FF800001EB001030309DF8A01000EB0110C07A9A
:10FF900000287FDD00229DF8B40000EB400101EB5A
:10FFA0000010384901EB001030309DF8A01000EB34
:10FFB0000110C2723648D0F80C020521B0FBF1F2F4
:10FFC00001FB120000EB400131482C3000EB4110E6
:10FFD0000D300A909DF8B40040F2991110FB01F029
:10FFE000264901EBC00000F552709DF8A01001EB0E
:10FFF000410202EB011100EBC10022301022014648
:020000040801F1
:1000000009900A98F8F721F92148D0F80C02052147
:10001000B0FBF1F201FB120000EB40011C482C3058
:1000200000EB41129DF8B40040F2991110FB01F071
:10003000124901EBC00101F552719DF8A00000EBDF
:10004000400303EB001001EBC00050F81A1F42F808
:10005000011F406850600E48D0F80C020521B0FB2B
:10006000F1F201FB120000EB400109482C3000EBDB
:1000700041129DF8B40000EB40010CE0C4440020A4
:10008000D814002004400020C731002064860020DE
:10009000BC12002090E101EB0010FE4901EB0011C1
:1000A00030319DF8A00001EB001000781070FA4884
:1000B000D0F80C020521B0FBF1F201FB120000EBBD
:1000C0004001F5482C3000EB41129DF8B40040F29D
:1000D000991110FB01F0F14901EBC00101F55271DA
:1000E0009DF8A00000EB400303EB001001EBC00003
:1000F000406BC2F80900E848D0F80C020521B0FBBB
:10010000F1F201FB120000EB4001E3482C3000EB60
:100110004111E348026841F81D2F80888880DE483D
:10012000D0F80C020521B0FBF1F201FB120000EB4C
:100130004001D9482C3000EB41129DF8B40000EB8F
:10014000400101EB0010D34901EB001130319DF863
:10015000A00001EB00104068C2F8230000229DF8C7
:10016000B40000EB400101EB0010CA4901EB0011A3
:1001700030319DF8A00001EB001042600021399160
:1001800054E0C548D0F80C020521B0FBF1F201FBA8
:10019000120000EB4001C0482C3000EB4111273128
:1001A000BDF8E4409DF8B40040F2991210FB02F053
:1001B000BA4A02EBC00202F552729DF8A00000EBB1
:1001C000400303EB001002EBC00090F8800040F207
:1001D000991210FB02F0B14A02EBC00202F5527212
:1001E0009DF8B40040F2991310FB03F0AB4B03EB06
:1001F000C00303F552739DF8A00000EB400505EB2A
:10020000001003EBC00090F8810000EB400303EB0B
:10021000001002EBC0024732BDF8E400001D105C84
:100220000855BDF8E400401C81B23991BDF8E400E6
:100230000628A6DB0020399042E000239DF8B40098
:1002400040F2991110FB01F0944901EBC00101F556
:1002500052719DF8A00000EB400202EB001001EB90
:10026000C00090F8800040F2991110FB01F08B491A
:1002700001EBC00101F552719DF8B40040F29912F2
:1002800010FB02F0854A02EBC00202F552729DF8A3
:10029000A00000EB400404EB001002EBC00090F85B
:1002A000810000EB400202EB001001EBC00147317E
:1002B000BDF8E4000B54BDF8E400401C81B2399154
:1002C000BDF8E4000A28B8DB7348D0F80C02052119
:1002D000B0FBF1F080B201460A900220F8F7F8FE78
:1002E00000210620F9F7A8FE6B48D0F80C026A49F5
:1002F000498D884206D26848D0F80C02401C6649F5
:10030000C1F80C0200210520F9F796FE9DF8B40013
:1003100000EB400101EB00105E4901EB00103030B2
:100320009DF8A01000EB0110801C0A90007820F0CE
:1003300008020A9802705848D0F80C020521B0FB58
:10034000F1F201FB120000EB400153482C3000EBAE
:100350004110D0F823202E9800EB4001514800EBCB
:100360004110C0F823200020399020E04A48D0F8FE
:100370000C020521B0FBF1F201FB120000EB400181
:1003800045482C3000EB41102730BDF8E410425CAA
:100390002E9800EB4001434800EB41112731BDF896
:1003A000E4000A54BDF8E400401C81B23991BDF864
:1003B000E4000628DADB59E09DF8B40000EB4001C8
:1003C00001EB0010334901EB001030309DF8A01014
:1003D00000EB0110801C0A90007820F00800083023
:1003E0000A9908709DF8B40000EB400101EB001081
:1003F000284901EB001030309DF8A01000EB0110EF
:1004000042682E9800EB4001264800EB4110C0F8EE
:1004100023200020399025E09DF8B40040F2991186
:1004200010FB01F01D4901EBC00101F552719DF86F
:10043000A00000EB400202EB001001EBC0014731CD
:10044000BDF8E4000A5C2E9800EB4001154800EB73
:1004500041112731BDF8E4000A54BDF8E400401C06
:1004600081B23991BDF8E4000628D5DB00229DF861
:10047000B40040F2991110FB01F0084901EBC001F2
:1004800001F552719DF8A00000EB400303EB001052
:100490000AE0000004400020BC120020C4440020F8
:1004A000C7310020D814002001EBC00080F846209E
:1004B0009DF8B4100220F9F7BFFD9DF8B40040F29A
:1004C000991110FB01F0FE4901EBC00101F55271D9
:1004D0009DF8A00000EB400202EB001001EBC00011
:1004E00022300A902E9800EB4001F64800EB4111B3
:1004F0000D3110220991DDE90901F7F7A6FE9DF8FB
:10050000B40040F2991110FB01F0ED4901EBC0017C
:1005100001F552719DF8A00000EB400202EB0010C3
:1005200001EBC0012E9800EB4002E64800EB4210C0
:1005300051F81A2F40F8012F496841609DF8B40026
:1005400000EB400101EB0010DF4901EB00113031FD
:100550009DF8A00001EB001001782E9800EB4002FE
:10056000D84800EB421001702E9800EB4001D548AE
:1005700000E06BE000EB4111D448026841F81D2F08
:10058000808888809DF8B40040F2991110FB01F03A
:10059000CB4901EBC00101F552719DF8A00000EBC1
:1005A000400202EB001001EBC000416B2E9800EB03
:1005B0004002C44800EB4210C0F809109DF8B40096
:1005C00000EB400101EB0010BF4901EB001130319D
:1005D0009DF8A00001EB001041682E9800EB40024E
:1005E000B84800EB4210C0F823102E9881B20820C2
:1005F0000A91F9F721FDA7229DF8B40040F2991164
:1006000010FB01F0AE4901EBC00101F552719DF8FC
:10061000A00000EB400303EB001001EBC0004271AF
:10062000A2229DF8B40040F2991110FB01F0A449F8
:1006300001EBC00000F552709DF8A01001EB4103E2
:1006400003EB011100EBC100827000BF00BF0CF092
:100650007EBE9DF8B40000EB4001C1EBC0109C4988
:1006600011F83000042801D126900BE09DF8B40069
:1006700000EB4001C1EBC010954911F8300015287E
:1006800000D126909DF8B41001EB4100C0EBC110E1
:100690008F4901EBC00041789DF8B40000EB4002A7
:1006A000C2EBC0108A4A12F8300041EA002041F241
:1006B0003001884202D1A62026903DE09DF8B4107A
:1006C00001EB4100C0EBC110814901EBC000417852
:1006D0009DF8B40000EB4002C2EBC0107C4A12F857
:1006E000300041EA002041F23101884202D1A720C6
:1006F000269021E09DF8B41001EB4100C0EBC11041
:10070000734911F83000022816D19DF8B41001EB9E
:100710004100C0EBC1106E4901EBC00001799DF8AA
:10072000B40000EB4002C2EBC010694A02EBC0000B
:10073000C07841EA002126919DF8B41040F299104A
:1007400011FB00F05E4901EBC00081782891002187
:10075000604A9DF8B40002EB00129DF8A00011540D
:100760005D4890F82800012815D19DF8B41001EBE0
:10077000410000EB0110544901EB001030309DF8AE
:10078000A01000EB0110801C0A90007820F080007F
:1007900080300A990870BDF89800A7287DD007DC42
:1007A00004287BD015287AD0A62841F0688752E02B
:1007B000A0F55850303820B1112871D01228F4D14A
:1007C000FEE39DF8B41040F2991011FB00F03C4993
:1007D00001EBC00000F552709DF8A01001EB410242
:1007E00002EB011110F8310098BB00219DF8B40014
:1007F00040F2991210FB02F0314A02EBC000017185
:1008000001229DF8B40040F2991110FB01F02C492F
:1008100001EBC00101F552719DF8A00000EB40030F
:1008200003EB001001F83020A7229DF8B40040F23D
:10083000991110FB01F0224901EBC00000F5527044
:100840009DF8A01001EB410303EB011100EBC10087
:10085000427101F014BF00219DF8B40040F29912DA
:1008600010FB02F0164A02EBC00001719DF8B410B3
:1008700040F2991011FB00F0114601EBC00000F5A9
:1008800052709DF8A01001EB410202EB011110F82B
:10089000310002283EDC032203E0FAE061E1B0E22D
:1008A000E4E29DF8B40040F2991110FB01F0044914
:1008B00001EBC00101F552719DF8A0000EE00000AF
:1008C000C4440020D814002004400020C731002078
:1008D00064860020383E0020BC12002000EB40035C
:1008E00003EB001001F83020A9229DF8B40040F27B
:1008F000991110FB01F0FA4901EBC00000F55270AC
:100900009DF8A01001EB410303EB011100EBC100C6
:100910004271BDE09DF8B41040F2991011FB00F057
:10092000EF4901EBC00000F552709DF8A01001EBFB
:10093000410202EB011110F83100052829DC0622E2
:100940009DF8B40040F2991110FB01F0E44901EB6D
:10095000C00101F552719DF8A00000EB400303EBCC
:10096000001001F83020A2229DF8B40040F2991145
:1009700010FB01F0DA4901EBC00000F552709DF860
:10098000A01001EB410303EB011100EBC100427128
:100990007EE09DF8B41040F2991011FB00F0D049B0
:1009A00001EBC00000F552709DF8A01001EB410270
:1009B00002EB011100EBC1004079A52815D19DF88B
:1009C000B41001EB410000EB0110C64901EB00102F
:1009D00030309DF8A01000EB0110801C0A900078C8
:1009E00020F00400001D0A9908709DF8B41040F230
:1009F000991011FB00F0BA4901EBC00000F55270EC
:100A00009DF8A01001EB410202EB011100EBC100C7
:100A10008078A1283CD09DF8B41040F2991011FBC9
:100A200000F0AF4901EBC00101F552719DF8A00043
:100A300000EB400202EB001001EBC00082789DF851
:100A4000B40040F2991110FB01F0A54901EBC0017F
:100A500001F552719DF8A00000EB400303EB00107C
:100A600001EBC0004271A1229DF8B40040F299113F
:100A700010FB01F09A4901EBC00000F552709DF89F
:100A8000A01001EB410303EB011100EBC1008270E8
:100A9000DFE69DF8B41040F2991011FB00F0904988
:100AA00001EBC00000F552709DF8A01001EB41026F
:100AB00002EB011100EBC1004079A42830D19DF870
:100AC000B41001EB410000EB0110864901EB00106E
:100AD00030309DF8A01000EB0110801C0A900078C7
:100AE00020F0200120310A98017000229DF8B40006
:100AF00040F2991110FB01F0794901EBC00101F5B9
:100B000052719DF8A00000EB400303EB001001EBD5
:100B1000C00080F845209DF8B4100220F9F78CFA47
:100B200000219DF8B40040F2991210FB02F06C4ACB
:100B300002EBC0000171A1229DF8B40040F29911AE
:100B400010FB01F0664901EBC00000F552709DF802
:100B5000A01001EB410303EB011100EBC100427156
:100B600077E69DF8B41040F2991011FB00F05C4953
:100B700001EBC00000F552709DF8A01001EB41029E
:100B800002EB011110F83100012834DC00219DF83E
:100B9000B40040F2991210FB02F0514A02EBC0007F
:100BA000017102229DF8B40040F2991110FB01F08E
:100BB0004B4901EBC00101F552719DF8A00000EB1B
:100BC000400303EB001001F83020A3229DF8B4008D
:100BD00040F2991110FB01F0414901EBC00000F512
:100BE00052709DF8A01001EB410303EB011100EBE3
:100BF000C100427104E19DF8B41040F2991011FB5C
:100C000000F0374901EBC00000F552709DF8A010CC
:100C100001EB410202EB011110F83100042834DC31
:100C200000219DF8B40040F2991210FB02F02C4A0A
:100C300002EBC000017105229DF8B40040F2991149
:100C400010FB01F0264901EBC00101F552719DF83E
:100C5000A00000EB400303EB001001F83020A322BA
:100C60009DF8B40040F2991110FB01F01C4901EB12
:100C7000C00000F552709DF8A01001EB410303EB9A
:100C8000011100EBC1004271BAE09DF8B41040F2CE
:100C9000991011FB00F0124901EBC00000F55270F1
:100CA0009DF8A01001EB410202EB011110F8310098
:100CB000062819DCA1229DF8B40040F2991110FB1E
:100CC00001F0074901EBC00000F552709DF8A0103B
:100CD00001EB410303EB011100EBC10042718FE016
:100CE000C4440020044000209DF8B41040F2991044
:100CF00011FB00F0FE4901EBC00101F552719DF8B6
:100D0000A00000EB400202EB001011F830109DF83B
:100D1000B40040F2991210FB02F0F54A02EBC00059
:100D2000407981426CD19DF8B41040F2991011FBCA
:100D300000F0114601EBC00000F552709DF8A010C4
:100D400001EB410202EB011100EBC1008078A12808
:100D500036D0A3229DF8B40040F2991110FB01F0A7
:100D6000E34901EBC00101F552719DF8A00000EBD1
:100D7000400303EB001001EBC00042719DF8B4107A
:100D800040F2991011FB00F0D94901EBC00000F5C9
:100D900052709DF8A01001EB410202EB011100EB33
:100DA000C1008078A2282BD000209DF8B41040F21A
:100DB000991211FB02F1CE4A02EBC10108711FE04A
:100DC000A1229DF8B40040F2991110FB01F0C8492E
:100DD00001EBC00101F552719DF8A00000EB40034A
:100DE00003EB001001EBC000427101219DF8B4003B
:100DF00040F2991210FB02F0BD4A02EBC0000171F3
:100E000027E5A1229DF8B40040F2991110FB01F0F2
:100E1000B74901EBC00101F552719DF8A00000EB4C
:100E2000400303EB001001EBC00042719DF8B400D9
:100E300040F2991110FB01F0AD4901EBC00101F541
:100E400052719DF8A00000EB400303EB001001EB92
:100E5000C000827000219DF8B40040F2991210FB8E
:100E600002F0A34A02EBC0000171F2E400219DF8F8
:100E7000B40040F2991210FB02F09D4A02EBC00050
:100E80000171A7229DF8B40040F2991110FB01F006
:100E9000974901EBC00101F552719DF8A00000EBEC
:100EA000400303EB001001EBC00042719DF8B41049
:100EB00001EB4100C0EBC1108E4901EBC00040794D
:100EC00030287ED19DF8B41040F2991011FB00F04B
:100ED000874901EBC00101F552719DF8A00000EBBC
:100EE000400202EB001011F830109DF8B40040F2FF
:100EF000991210FB02F07E4A02EBC0004079814259
:100F00005FD19DF8B40000EB400101EB0010A2F5A9
:100F1000986101EB001030309DF8A01000EB01103B
:100F2000801C0A90007820F001020A9802709DF857
:100F3000B40000EB400101EB00106F4901EB001021
:100F400030309DF8A01000EB0110801C0A90007852
:100F500020F002020A9802709DF8B40040F2991144
:100F600010FB01F0624901EBC00000F552709DF8E2
:100F7000A01001EB410202EB011100EBC100C078AF
:100F8000312832D19DF8B40000EB400101EB001094
:100F9000594901EB001030309DF8A01000EB011012
:100FA000801C0A90007820F020020A98027000222B
:100FB0009DF8B40040F2991110FB01F04C4901E09A
:100FC000FDE33FE001EBC00000F552709DF8A0107A
:100FD00001EB410303EB011100EBC10080F8452058
:100FE0009DF8B4100220F9F727F89DF8B40040F2FC
:100FF000991110FB01F03E4901EBC00000F5527061
:101000009DF8A01001EB410202EB011100EBC100C1
:1010100090F84600012814D1A9229DF8B40040F2AE
:10102000991110FB01F0324901EBC00000F552703C
:101030009DF8A01001EB410303EB011100EBC1008F
:101040008270DCE39DF8B40000EB4001C1EBC010FE
:10105000284901EBC000407931287DD19DF8B400CA
:1010600040F2991110FB01F0214901EBC00101F59B
:1010700052719DF8A00000EB400202EB001011F845
:1010800030109DF8B40040F2991210FB02F0184A9B
:1010900002EBC000407981425ED19DF8B40040F27D
:1010A000991110FB01F0114601EBC00000F55270E0
:1010B0009DF8A01001EB410202EB011100EBC10011
:1010C00090F8460090BB01229DF8B40040F29911BF
:1010D00010FB01F0064901EBC00101F552719DF8CA
:1010E000A00000EB400303EB001001EBC00005E0A3
:1010F000C4440020648600200440002080F845207D
:101100009DF8B40000EB400101EB0010FE4901EB3B
:10111000001130319DF8A00001EB0010801C0A90F6
:10112000007820F00100401C0A9908709DF8B40076
:1011300000EB400101EB0010F34901EB00103030EF
:101140009DF8A01000EB0110801C0A90007820F0A0
:1011500002020A98027000E00BE2EC4890F8900757
:1011600080B19DF8B40000EB400101EB0010E649AE
:1011700001EB001030309DF8A01000EB0110807AD8
:10118000022878D1E24890F829000128F9D1E048F6
:10119000D0F80C02DE49498D88426CD29DF8B4002B
:1011A00040F2991110FB01F0DA4901EBC00000F5A3
:1011B00052709DF8A01001EB410202EB011100EB0F
:1011C000C10090F84500012854D19DF8B40040F2C8
:1011D000991110FB01F0CF4901EBC00000F55270EE
:1011E0009DF8A01001EB410202EB011100EBC100E0
:1011F00090F87F00F0BB01229DF8B40000EB4001A5
:1012000001EB0010C04901EB001130319DF8A00046
:1012100001EB0010C2724FF010429DF8B40040F292
:10122000991110FB01F0BB4901EBC00101F55271AE
:101230009DF8A00000EB400303EB001001EBC000A1
:1012400082609DF8B40000EB400101EB0010AE4954
:1012500001EB001130319DF8A00001EB0010017886
:101260009DF8B40040F2991210FB02F0A94A02EB7B
:10127000C00001E070E005E141709DF8B40040F26B
:10128000991110FB01F0114601EBC00101F55271FB
:101290009DF8A00000EB400202EB001011F83010A6
:1012A0009DF8B40040F2991210FB02F0994A02EB4B
:1012B000C000407981423ED100229DF8B40040F246
:1012C000991110FB01F0934901EBC00101F5527136
:1012D0009DF8A00000EB400303EB001001EBC00001
:1012E000C271A4229DF8B40040F2991110FB01F0E4
:1012F000884901EBC00101F552719DF8A00000EB97
:10130000400303EB001001EBC0008270A3229DF8A4
:10131000B40040F2991110FB01F07E4901EBC000CE
:1013200000F552709DF8A01001EB410303EB011191
:1013300000EBC100427100229DF8B40000EB4001B7
:1013400001EB0010704901EB001030309DF8A01047
:1013500000EB0110426052E29DF8B40040F2991196
:1013600010FB01F06B4901EBC00000F552709DF8D5
:10137000A01001EB410202EB011100EBC10090F85B
:10138000450001287ED19DF8B40040F2991110FB70
:1013900001F0604901EBC00101F552719DF8A00018
:1013A00000EB400202EB001001EBC00090F880005F
:1013B00040F2991110FB01F0564901EBC00101F513
:1013C00052719DF8B40040F2991210FB02F0514A9C
:1013D00002EBC00000F552709DF8A02002EB420322
:1013E00003EB021200EBC20090F8810000EB400218
:1013F00002EB001001EBC00090F87E00032841D101
:1014000002229DF8B40000EB400101EB00103E49C0
:1014100001EB001130319DF8A00001EB0010C27209
:101420004FF010429DF8B40040F2991110FB01F00A
:10143000384901EBC00101F552719DF8A00000EBA5
:10144000400303EB001001EBC00082609DF8B40084
:1014500000EB400101EB00102B4901EB0011303192
:101460009DF8A00001EB001001789DF8B40040F257
:10147000991210FB02F0274A02EBC00041709DF860
:10148000B40000E09CE140F2991110FB01F011461C
:1014900001EBC00101F552719DF8A00000EB400284
:1014A00002EB001011F830109DF8B40040F29912D0
:1014B00010FB02F0174A02EBC0004079814247D18D
:1014C00000229DF8B40040F2991110FB01F011497F
:1014D00001EBC00101F552719DF8A00000EB400343
:1014E00003EB001001EBC000C271A4229DF8B40010
:1014F00040F2991110FB01F0064901EBC00101F522
:1015000052719DF8A00007E004400020BC3200208A
:10151000BC120020C444002000EB400303EB001089
:1015200001EBC0008270A3229DF8B40040F2991133
:1015300010FB01F0F74901EBC00000F552709DF877
:10154000A01001EB410303EB011100EBC10042715C
:1015500000229DF8B40000EB400101EB0010EE49C1
:1015600001EB001030309DF8A01000EB011042603C
:1015700045E19DF8B40000EB4001C1EBC010E74924
:1015800001EBC000407933287ED19DF8B40000EB18
:10159000400101EB0010E04901EB001030309DF8F4
:1015A000A01000EB0110801C0A90007820F00100D0
:1015B000401C0A9908709DF8B40000EB400101EB53
:1015C0000010D54901EB001030309DF8A01000EB61
:1015D0000110801C0A90007820F020020A98027006
:1015E0009DF8B40000EB400101EB0010CA4901EB8B
:1015F000001030309DF8A01000EB0110801C0A9004
:10160000007820F00200801C0A9908709DF8B40050
:1016100040F2991110FB01F0BE4901EBC000427984
:101620009DF8B40040F2991110FB01F0B94901EBAB
:10163000C00000F552709DF8A01001EB410303EBD0
:10164000011100F831209DF8B40000EB400101EBDE
:101650000010B14901EB001030309DF8A01000EBF4
:101660000110801C0A90007820F0800080300A99D8
:1016700008709DF8B40000EB400101EB0010A64992
:1016800001EB0010303000E022E09DF8A01000EBEC
:1016900001108078C0F3400020B99DF8B4100220FA
:1016A000F8F7CAFCA2229DF8B40040F2991110FB91
:1016B00001F0984901EBC00000F552709DF8A010B0
:1016C00001EB410303EB011100EBC100827096E0D6
:1016D0009DF8B41001EB4100C0EBC1108F4901EB44
:1016E000C000407934286BD19DF8B41001EB410063
:1016F00000EB0110884901EB001030309DF8A0107C
:1017000000EB0110801C0A90007820F020020A985B
:1017100002709DF8B41001EB410000EB01107E490E
:1017200001EB001030309DF8A01000EB0110801C80
:101730000A90007820F002020A98027001229DF8B7
:10174000B40040F2991110FB01F0724901EBC000A6
:1017500000F552709DF8A01001EB410303EB01115D
:1017600000EBC10080F84620A9229DF8B40040F2A9
:10177000991110FB01F0674901EBC00000F55270B0
:101780009DF8A01001EB410303EB011100EBC10038
:1017900082709DF8B41040F2991011FB00F05D4981
:1017A00001EBC00042799DF8B40040F2991110FBA2
:1017B00001F0584901EBC00000F5527001E0DFE292
:1017C0001DE09DF8A01001EB410303EB011100F8AF
:1017D00031209DF8B41001EB410000EB01104E499F
:1017E00001EB001030309DF8A01000EB0110801CC0
:1017F0000A90007820F0800080300A99087000205C
:101800002E902F900021399122E0DDE92E10000169
:1018100040EA11720901CDE92E129DF8B41001EBD6
:101820004100C0EBC1103D4901EBC001BDF8E4002F
:10183000801D085C3038C117DDE92E34184341EAB9
:101840000402CDE92E02BDF8E400401C80B23990BC
:10185000BDF8E4000828D8DB9DF8B4002E9940F2CA
:10186000991210FB02F02B4A02EBC00202F55272F1
:101870009DF8A00000EB400303EB001002EBC0005A
:10188000C0F81A1000222E922F920021399122E0E6
:10189000DDE92E10000140EA11720901CDE92E1296
:1018A0009DF8B41001EB4100C0EBC1101B4901EBE6
:1018B000C001BDF8E4000F30085C3038C117DDE925
:1018C0002E24104341EA0402CDE92E02BDF8E400C3
:1018D000401C80B23990BDF8E4000628D8DB9DF8A2
:1018E000B4002E9940F2991210FB02F0094A02EB63
:1018F000C00202F552729DF8A00000EB400303EB1A
:10190000001002EBC000416300222E922F920021B2
:10191000399128E0C444002004400020648600205F
:10192000DDE92E10000140EA11720901CDE92E1205
:101930009DF8B41001EB4100C0EBC110FE4901EB72
:10194000C001BDF8E4001530085C3038C117DDE98E
:101950002E34184341EA0402CDE92E02BDF8E4001A
:10196000401C80B23990BDF8E4000828D8DB9DF80F
:10197000B4002E9940F2991210FB02F0EF4A02EBEC
:10198000C00202F552729DF8A00000EB400303EB89
:10199000001002EBC000C0F81E109DF8B41001EB5F
:1019A0004100C0EBC110E44901EBC00042799DF851
:1019B000B40040F2991110FB01F0E04901EBC001C5
:1019C00001F552719DF8A00000EB400303EB0010FD
:1019D00001EBC000C2709DF8B41001EB410000EBB8
:1019E0000110D74901EB001130319DF8A00001EB47
:1019F000001082789DF8B40040F2991110FB01F0BC
:101A0000CE4901EBC00101F552719DF8A00000EB39
:101A1000400303EB001001EBC00002769DF8B41008
:101A200040F2991011FB00F0C44901EBC00101F52F
:101A300052719DF8A00000EB400202EB001011F87B
:101A400030109DF8B40040F2991210FB02F0BB4A2E
:101A500002EBC000407981427DDA00219DF8B4009C
:101A600040F2991210FB02F0B44A02EBC00001717F
:101A7000A7229DF8B40040F2991110FB01F0AF4984
:101A800001EBC00101F552719DF8A00000EB40038D
:101A900003EB001001EBC000427101219DF8B4007E
:101AA00040F2991210FB02F0A44A02EBC00001714F
:101AB0009DF8B41040F2991011FB00F0114601EBB3
:101AC000C00042799DF8B40040F2991110FB01F07A
:101AD0009A4901EBC00101F552719DF8A00000EB9D
:101AE000400303EB001001F83020A1229DF8B40060
:101AF00040F2991110FB01F0904901EBC00101F592
:101B000052719DF8A00000EB400303EB001001EBC5
:101B1000C00042719DF8B41001EB410000EB0110D0
:101B2000874901EB001130319DF8A00001EB001056
:101B3000801C0A90007820F0800080300A9908709C
:101B40009DF8B41001EB410000EB01107C4901EB62
:101B50000010303000E05BE09DF8A01000EB0110B9
:101B6000801C0A90007820F00400001D0A9908707B
:101B70009DF8B41001EB410000EB0110704901EB3E
:101B8000001030309DF8A01000EB01108078C0F3F9
:101B90004010E8B39DF8B41001EB410000EB0110D8
:101BA000674901EB001030309DF8A01000EB0110E8
:101BB000801C0A90007820F020020A9802709DF89C
:101BC000B41001EB410000EB01105D4901EB001086
:101BD00030309DF8A01000EB01108078C0F3400079
:101BE000F0BB9DF8B41001EB410000EB011054492B
:101BF00001EB001030309DF8A01000EB0110801CAC
:101C00000A90007820F0080108310A98017000E07D
:101C1000B5E09DF8B4109DF8A00000EB0110C217CC
:101C2000CDE92E029DF8B41040F2991011FB00F09E
:101C3000424901EBC00000F552709DF8A01001EB85
:101C4000410202EB011100EBC10022300A902E98F4
:101C500000EB40013B4800EB41100D30102200E04A
:101C600088E009900A99F6F7F0FA9DF8B41040F26E
:101C7000991011FB00F0314901EBC00101F55271DF
:101C80009DF8A00000EB400202EB001001EBC00148
:101C90002E9800EB40022B4800EB421051F81A2F0F
:101CA00040F8012F496841609DF8B41001EB4100F4
:101CB00000EB0110224901EB001130319DF8A0002A
:101CC00001EB001001782E9800EB40021D4800EB5C
:101CD000421001702E9800EB40011A4800EB4111B0
:101CE0001948026841F81D2F808888809DF8B4103B
:101CF00040F2991011FB00F0104901EBC00101F511
:101D000052719DF8A00000EB400202EB001001EBC5
:101D1000C000416B2E9800EB40020A4800EB4210D5
:101D2000C0F809109DF8B41001EB410000EB011060
:101D3000034901EB001109E064860020C44400203F
:101D400004400020D8140020C731002030319DF815
:101D5000A00001EB001041682E9800EB4002FE4805
:101D600000EB4210C0F823102E9881B208200A918F
:101D7000F8F762F99DF8B4100220F8F75DF9FFE377
:101D800000202E902F900021399122E0DDE92E10C5
:101D9000000140EA11720901CDE92E129DF8B4103C
:101DA00001EB4100C0EBC110EC4901EBC001BDF8F3
:101DB000E4000B30085C3038C117DDE92E341843DD
:101DC00041EA0402CDE92E02BDF8E400401C80B2D5
:101DD0003990BDF8E4000C28D8DB9DF8B400DDE9AB
:101DE0002E1240F2991310FB03F0DD4B03EBC003FE
:101DF00003F552739DF8A00000EB400404EB0010C3
:101E000003EBC00040F8221F426000222E922F9266
:101E10000021399122E0DDE92E10000140EA117223
:101E20000901CDE92E129DF8B41001EB4100C0EB81
:101E3000C110CA4901EBC001BDF8E4001730085CCD
:101E40003038C117DDE92E34184341EA0402CDE9E8
:101E50002E02BDF8E400401C80B23990BDF8E400C9
:101E60000C28D8DB9DF8B400DDE92E1240F299135E
:101E700010FB03F0BA4B03EBC00303F552739DF85C
:101E8000A00000EB400404EB001003EBC000223084
:101E90008160C26000219DF8B40040F2991210FBED
:101EA00002F0AF4A02EBC00001719DF8B41040F29D
:101EB000991011FB00F0114601EBC00000F55270C3
:101EC0009DF8A01001EB410202EB011110F8310066
:101ED000032814DC04229DF8B40040F2991110FB91
:101EE00001F09F4901EBC00000F552709DF8A01071
:101EF00001EB410303EB011100F831207EE39DF873
:101F0000B41040F2991011FB00F0954901EBC001AB
:101F100001F552719DF8A00000EB400202EB0010A9
:101F200011F830109DF8B40040F2991210FB02F045
:101F30008B4A02EBC00040798142DFD19DF8B400AA
:101F40009DF8A01001EB0010C217CDE92E028548C4
:101F500090F8900708B39DF8B41001EB410000EB36
:101F60000110814901EB001030309DF8A01000EB0A
:101F70000110807A022810D09DF8B41001EB4100C6
:101F800000EB0110784901EB001030309DF8A010F3
:101F900000EB0110C07A00287EDD00229DF8B4001D
:101FA00000EB400101EB00106F4901EB00103030F5
:101FB0009DF8A01000EB0110C2726C48D0F80C0222
:101FC0000521B0FBF1F201FB120000EB4001674874
:101FD0002C3000EB41100D300A909DF8B40040F217
:101FE000991110FB01F05E4901EBC00000F5527041
:101FF0009DF8A01001EB410202EB011100EBC100C2
:1020000022301022014609900A98F6F71EF9574827
:10201000D0F80C020521B0FBF1F201FB120000EB3D
:10202000400152482C3000EB41129DF8B40040F2C0
:10203000991110FB01F04A4901EBC00101F5527101
:102040009DF8A00000EB400303EB001001EBC00083
:1020500050F81A1F42F8011F406850604348D0F8FA
:102060000C020521B0FBF1F201FB120000EB400174
:102070003E482C3000EB41129DF8B40000EB4001CB
:1020800001EB0010384901EB001130319DF8A00040
:1020900001EB0010007800E093E110703348D0F8B5
:1020A0000C020521B0FBF1F201FB120000EB400134
:1020B0002E482C3000EB41129DF8B40040F29911EB
:1020C00010FB01F0264901EBC00101F552719DF8AA
:1020D000A00000EB400303EB001001EBC000406BDD
:1020E000C2F809002148D0F80C020521B0FBF1F23A
:1020F00001FB120000EB40011C482C3000EB4111A9
:102100001848F538026841F81D2F808888801748E4
:10211000D0F80C020521B0FBF1F201FB120000EB3C
:10212000400112482C3000EB41129DF8B40000EB46
:10213000400101EB00100C4901EB001130319DF81A
:10214000A00001EB00104068C2F8230000229DF8B7
:10215000B40000EB40010BE0D8140020648600209E
:10216000C4440020BC32002004400020BC120020E7
:1021700001EB0010FD4901EB001130319DF8A0008A
:1021800001EB001042600021399154E0F848D0F88A
:102190000C020521B0FBF1F201FB120000EB400143
:1021A000F3482C3000EB41112731BDF8E4409DF895
:1021B000B40040F2991210FB02F0EE4A02EBC002AA
:1021C00002F552729DF8A00000EB400303EB0010F3
:1021D00002EBC00090F8800040F2991210FB02F070
:1021E000E44A02EBC00202F552729DF8B40040F2DC
:1021F000991310FB03F0DF4B03EBC00303F552739D
:102200009DF8A00000EB400505EB001003EBC000BB
:1022100090F8810000EB400303EB001002EBC002DA
:102220004732BDF8E400001D105C0855BDF8E4001D
:10223000401C81B23991BDF8E4000628A6DB0021DC
:10224000399142E000239DF8B40040F2991110FB4F
:1022500001F0C84901EBC00101F552719DF8A000E1
:1022600000EB400202EB001001EBC00090F8800090
:1022700040F2991110FB01F0BE4901EBC00101F5DC
:1022800052719DF8B40040F2991210FB02F0B94A65
:1022900002EBC00202F552729DF8A00000EB400470
:1022A00004EB001002EBC00090F8810000EB40024C
:1022B00002EB001001EBC0014731BDF8E4000B5404
:1022C000BDF8E400401C81B23991BDF8E4000A2851
:1022D000B8DBA748D0F80C020521B0FBF1F080B2C2
:1022E00001460A900220F6F7F3FE00210620F7F7D8
:1022F000A3FE9F48D0F80C029D49498D884206D222
:102300009B48D0F80C02401C9949C1F80C020021EE
:102310000520F7F791FE9DF8B41001EB410000EBAA
:102320000110924901EB001030309DF8A01000EB35
:102330000110801C0A90007820F008020A980270B0
:102340008B48D0F80C020521B0FBF1F201FB120022
:1023500000EB400186482C3000EB4110D0F82320E0
:102360002E9800EB4001844800EB4110C0F8232078
:102370000020399020E07E48D0F80C020521B0FB07
:10238000F1F201FB120000EB400179482C3000EB28
:1023900041102730BDF8E410425C2E9800EB40015C
:1023A000754800EB41112731BDF8E4000A54BDF82F
:1023B000E400401C81B23991BDF8E4000628DADB64
:1023C00059E09DF8B41001EB410000EB01106749A2
:1023D00001EB001030309DF8A01000EB0110801CC4
:1023E0000A90007820F0080008300A9908709DF8DB
:1023F000B41001EB410000EB01105C4901EB00104F
:1024000030309DF8A01000EB011042682E9800EBD0
:102410004001594800EB4110C0F8232000203990BA
:1024200025E09DF8B41040F2991011FB00F05149DD
:1024300001EBC00101F552719DF8A00000EB4002D4
:1024400002EB001001EBC0014731BDF8E4000A5C6B
:102450002E9800EB4001484800EB41112731BDF8B0
:10246000E4000A54BDF8E400401C81B23991BDF883
:10247000E4000628D5DB00229DF8B40040F2991153
:1024800010FB01F03B4901EBC00101F552719DF8D1
:10249000A00000EB400303EB001001EBC00080F84C
:1024A00046209DF8B4100220F7F7C6FD9DF8B40051
:1024B00040F2991110FB01F02E4901EBC00101F52A
:1024C00052719DF8A00000EB400202EB001001EBFE
:1024D000C00022300A902E9800EB4001264800EB05
:1024E00041110D3110220991DDE90901F5F7ADFE29
:1024F0009DF8B41040F2991011FB00F01D4901EB5A
:10250000C00101F552719DF8A00000EB400202EB02
:10251000001001EBC0012E9800EB4002164800EBC2
:10252000421051F81A2F40F8012F496841609DF878
:10253000B41001EB410000EB01100C4901EB00115C
:1025400030319DF8A00001EB001001782E9800EBCF
:102550004002094800EB421001702E9800EB400148
:10256000054800EB4111054802680AE004400020DC
:10257000BC120020C4440020D8140020C731002021
:102580007DE041F81D2F808888809DF8B41040F2CE
:10259000991011FB00F0F84901EBC00101F55271EF
:1025A0009DF8A00000EB400202EB001001EBC00020
:1025B000416B2E9800EB4002F04800EB4210C0F84F
:1025C00009109DF8B41001EB410000EB0110EC493B
:1025D00001EB001130319DF8A00001EB00104168C3
:1025E0002E9800EB4002E54800EB4210C0F82310A3
:1025F0002E9881B208200A91F7F71EFD00229DF85F
:10260000B40040F2991110FB01F0DB4901EBC0016D
:1026100001F552719DF8A00000EB400303EB0010A0
:1026200001EBC00080F84620A7229DF8B40040F2DC
:10263000991110FB01F0D04901EBC00101F5527175
:102640009DF8A00000EB400303EB001001EBC0007D
:102650004271A2229DF8B40040F2991110FB01F0E2
:10266000C54901EBC00000F552709DF8A01001EBC8
:10267000410303EB011100EBC100827000BF00BFFA
:102680000AF065BE0021BF4A9DF8B40002EB0012BB
:102690009DF8A00011549DF8B41001EB4100C0EB6F
:1026A000C110B94901EBC000407870280ED19DF8E7
:1026B000B41001EB4100C0EBC110B34901EBC00005
:1026C0008078FA2802D1B121269142E09DF8B41019
:1026D00001EB4100C0EBC110AB4901EBC0004078F9
:1026E00000F0F000C0280ED19DF8B41001EB4100BD
:1026F000C0EBC110A44901EBC0008078FA2802D1D8
:10270000B621269125E09DF8B41001EB4100C0EB05
:10271000C1109D4911F8300000F0F000502818D188
:102720009DF8B41001EB4100C0EBC110964901EBDC
:10273000C000407800F0F00030280AD19DF8B410B5
:1027400001EB4100C0EBC1108F4901EBC000817863
:1027500026919DF8B41040F2991011FB00F08649C3
:1027600001EBC000817828910021864A9DF8B400D1
:1027700002EB00129DF8A0001154844890F8280044
:10278000012815D19DF8B41001EB410000EB0110B8
:102790007B4901EB001030309DF8A01000EB0110D8
:1027A000801C0A90007820F0800080300A99087020
:1027B000BDF89800652876D004DC012809D00328EC
:1027C00005D17FE0B12802D0B62800D100E089E130
:1027D00088E19DF8B41001EB4100C0EBC1106A49DB
:1027E00001EBC0000079012806D0022805D003289B
:1027F00004D0052864D102E062E061E060E09DF869
:10280000B41040F2991011FB00F05B4901EBC000DD
:1028100000F552709DF8A01001EB410202EB01118E
:1028200010F83100F0BB00219DF8B40040F299127D
:1028300010FB02F0504A02EBC000017101229DF82A
:10284000B40040F2991110FB01F04B4901EBC001BB
:1028500001F552719DF8A00000EB400303EB00105E
:1028600001F83020B6229DF8B40040F2991110FB17
:1028700001F0414901EBC00101F552719DF8A00042
:1028800000EB400303EB001001EBC0004271B222E9
:102890009DF8B40040F2991110FB01F0364901EBAC
:1028A000C00001E00BE035E000F552709DF8A0108B
:1028B00001EB410303EB011100EBC100827000BF8B
:1028C00000BF0FE19DF8B41001EB4100C0EBC11057
:1028D0002D4901EBC000C1792D4880F8031D9DF8FA
:1028E000B41001EB410000EB0110254901EB001190
:1028F00030319DF8A00001EB0010801C0A902448A4
:1029000090F8030DC2080A98007862F300000A9953
:102910000870E7E09DF8B41001EB4100C0EBC11076
:10292000194901EBC000007900F0F00010B9B8219E
:10293000269101E0B9212691002139912FE09DF8DF
:10294000B41001EB410000EB01100D4901EB001147
:102950003031BDF8E40001EB001041789DF8B4007F
:1029600000EB4002C2EBC010074A12F830005038AA
:1029700081420FD121E00000C4440020D81400207F
:1029800004400020383E002064860020BC12002055
:10299000BC220020BDF8E400401C81B239919DF8B2
:1029A000B41001EB410000EB0110F74901EB0010FE
:1029B000C179BDF8E4008142C1DC00BF9DF8B410CC
:1029C00040F2991011FB00F0F04901EBC00000F556
:1029D00052709DF8A01001EB410202EB011110F8BA
:1029E0003100012834D100219DF8B40040F2991241
:1029F00010FB02F0E54A02EBC000017102229DF8D3
:102A0000B40040F2991110FB01F0E04901EBC00164
:102A100001F552719DF8A00000EB400303EB00109C
:102A200001F83020B9229DF8B40040F2991110FB52
:102A300001F0D64901EBC00000F552709DF8A010DE
:102A400001EB410303EB011100EBC100427148E0CF
:102A50009DF8B41040F2991011FB00F0CB4901EB46
:102A6000C00000F552709DF8A01001EB410202EB8E
:102A7000011110F83100012833D100219DF8B40074
:102A800040F2991210FB02F0C04A02EBC000017143
:102A900002229DF8B40040F2991110FB01F0BB49ED
:102AA00001EBC00101F552719DF8A00000EB40035D
:102AB00003EB001001F83020B9229DF8B40040F279
:102AC000991110FB01F0B14901EBC00000F5527003
:102AD0009DF8A01001EB410303EB011100EBC100D5
:102AE000427100BF00BFCBE59DF8B41001EB41007F
:102AF00000EB0110A44901EB0010007B20B101287C
:102B00007ED002287DD1EDE2A1499DF8B40031F8D4
:102B10001000801F81B20A919DF8B41001EB4100B2
:102B2000C0EBC1109B4901EBC000401C09900A9901
:102B3000F6F7D0FE0022CDE930029DF8B41001EB8B
:102B40004100C0EBC110934901EBC00290489DF8D1
:102B5000B41030F81100401F11180A9104210A988E
:102B60001DF092FBC217CDE92E022FA819C82E998D
:102B70005940604001437DD1874A9DF8B40002EB83
:102B8000001001709DF8B41001EB4100C0EBC110C2
:102B9000804901EBC00001792691BDF898003128E9
:102BA00002D0452867D1FBE079489DF8B41030F891
:102BB00011001838412190FBF1F0C217C1B2CDE9E4
:102BC0002E02764880F8AC1000203990D1E09DF8B4
:102BD000B41001EB4100C0EBC1106E4901EBC00124
:102BE000BDF8E40000EB80101430095C6B4AAD3294
:102BF000BDF8E40011549DF8B41001EB410001E070
:102C0000D1E06EE2C0EBC110624901EBC001BDF83A
:102C1000E40000EB80101A3001440A9108210A9860
:102C20001DF0F0FA8DED0F0A5C4AB932BDF8E400F0
:102C30000F9902EB001041609DF8B41001EB4100C8
:102C4000C0EBC110534901EBC001BDF8E40000EB3B
:102C50008010323001440A9108210A981DF0D2FAFE
:102C60008DED0F0A4D4AB932BDF8E4000F9902EB21
:102C7000001001E096E094E001609DF8B41001EBD3
:102C80004100C0EBC110434901EBC001BDF8E400B5
:102C900000EB80103A3001440A9108210A981DF097
:102CA000B1FA8DED0F0A3D4AB932BDF8E4000F9933
:102CB00002EB001081609DF8B40000EB4001C1EB15
:102CC000C010344901EBC001BDF8E40000EB8010F6
:102CD000423001440A9108210A981DF093FA8DEDC3
:102CE0000F0A2E4AB932BDF8E4000F9902EB00102A
:102CF000C1609DF8B40000EB400101EB00102249D7
:102D000001EB00113031BDF8E40001EB0010801C34
:102D10000A90007820F0800080300A9908709DF8B1
:102D2000B40000EB4001C1EBC0101A4901EBC00236
:102D300017489DF8B41030F81100401E125C9DF841
:102D4000B40040F2991110FB01F0104901EBC001F1
:102D500001F552719DF8A00000EB400303EB001059
:102D600001EBC00080F84420BDF8E400401C81B2B3
:102D70003991BDF8E4000021DDE92E34C01AA141EB
:102D8000FFF625AF0DE0000004400020C444002001
:102D9000E477002064860020383E0020BC3200200A
:102DA00000BF00BFB7E29DF8B40000EB4001C1EBEB
:102DB000C010FE4901EBC000407D9DF8B41001EB4E
:102DC0004102C2EBC111F94A02EBC101897D40EA1F
:102DD0000120C217CDE92E029DF8B40000EB40019E
:102DE000C1EBC010F14901EBC0010A9115210A980D
:102DF000F6F754FD0022CDE930022FA819C82E990C
:102E00005940604001437CD19DF8B40000EB400183
:102E1000C1EBC010E54911F83000401EC1B2289145
:102E20000021E34A9DF8B40002EB00129DF8A000D7
:102E300011540022DF499DF8A0000A549FEDDE0ADC
:102E400010EE101ADB4A0C329DF8A00002EB0010C5
:102E500041609DF8B40000EB4001C1EBC010D349C4
:102E600001EBC00081799DF8B40000EB4002C2EB99
:102E7000C010CE4A02EBC000407941EA002000EECB
:102E8000100AB8EEC00A9FEDCD1AC0EE010A9DF8F7
:102E9000B40000EB4001C1EBC010114601EBC000D3
:102EA00001799DF8B40000EB4002C2EBC010BF4AAC
:102EB00002EBC000C07841EA002000EE100AB8EE34
:102EC000C00A30EE800A10EE101ABA4A0C329DF891
:102ED000A00002EB001001609DF8B40000EB40017F
:102EE000C1EBC010B14901EBC000817A9DF8B4007C
:102EF00000EB4002C2EBC010AC4A02EBC000407ACB
:102F000000E0EEE041EA002000EE100AB8EEC00A50
:102F10009FEDAA1AC0EE010A9DF8B40000EB400133
:102F2000C1EBC010114601EBC000017A9DF8B4005E
:102F300000EB4002C2EBC0109C4A02EBC000C0791B
:102F400041EA002000EE100AB8EEC00A30EE800A16
:102F500010EE101A974A0C329DF8A00002EB0010F8
:102F600081609DF8B40000EB4001C1EBC0108F49B7
:102F700001EBC000C07A00F0800038BB9DF8B400BF
:102F800000EB4001C1EBC010884901EBC000017BA0
:102F90009DF8B40000EB4002C2EBC010834A02EB84
:102FA000C000C07A41EA002000EE100AF8EEC00A24
:102FB000B3EE001A80EE810A10EE100A7D4A0C3240
:102FC0009DF8A01002EB0111C86047E09DF8B40025
:102FD00000EB4001C1EBC010744901EBC000017B64
:102FE0009DF8B40000EB4002C2EBC0106F4A02EB48
:102FF000C000C07A41EA0020404280B200EE100AD0
:10300000B8EEC00A8DED030A0398F5F787FB9FED34
:103010006C0B53EC102BCDE904019DED040B51EC2E
:10302000100BF5F75FFA9FED680B53EC102BCDE911
:1030300006019DED060B51EC100BF5F7DEF9CDE91D
:1030400008019DED080B51EC100BF5F77AFB594A7E
:103050000C329DF8A01002EB0111C8609DF8B4007D
:1030600000EB400101EB0010594901EB001030303A
:103070009DF8A01000EB0110801C0A90007820F051
:10308000800080300A9908709DF8B40000EB400180
:10309000C1EBC010454901EBC000C27D9DF8B400F2
:1030A00040F2991110FB01F04A4901EBC00000F514
:1030B00052709DF8A01001EB410303EB011100EBEE
:1030C000C10080F844209DF8B40000EB400101EB02
:1030D00000103F4901EB0010C1793648AD3880F847
:1030E000AC1018E19DF8B41001EB4100C0EBC11128
:1030F0002E4800EBC100C0799DF8B41001EB4102ED
:10310000C2EBC111294A02EBC101097A40EA012050
:10311000C217CDE92E029DF8B41001EB4100C0EBBF
:10312000C110224901EBC0010A9107210A98F6F764
:10313000B5FB0022CDE93002DDE93043DDE92E1098
:103140006140584001437DD19DF8B41001EB41002E
:10315000C0EBC110154911F83000401EC1B22891D2
:103160000021134A9DF8B40002EB00100170002208
:1031700010499DF8A0000A549DF8B41001EB4100DD
:10318000C0EBC110094901EBC000817908460191EB
:10319000F5F73EFACDE902019DED021B9FED0E0B06
:1031A00020F07EFF8DED060B1AE000006486002003
:1031B000383E0020693300200000000000FF7F47F8
:1031C000000000000000304000000000000000008F
:1031D00004400020C44400200000000000002440FF
:1031E0009DF8B41001EB4100C0EBC110FE4901EBAA
:1031F000C00001799DF8B40000EB4002C2EBC010A2
:10320000F94A02EBC000C07841EA002000EE100A43
:10321000B8EEC00A8DED030A0398F5F77FFACDE901
:1032200004019DED060B53EC102B9DED040B51ECAE
:10323000100BF5F757F9CDE908019DED080B51EC9E
:10324000100B00E066E0F5F77CFAE84A9DF8A01064
:1032500002EB011148601FED280A10EE100A9DF8DC
:10326000A01002EB011108601FED2D0A10EE100AEC
:103270009DF8A01002EB011188601FED310A10EEDD
:10328000100A9DF8A01002EB0111C8609DF8B4105F
:1032900001EB410000EB011002F68F4101EB001041
:1032A00030309DF8A01000EB0110801C0A900078CF
:1032B00020F0800080300A9908709DF8B41001EB6E
:1032C0004100C0EBC110C84901EBC000427A9DF833
:1032D000B40040F2991110FB01F0C54901EBC000A8
:1032E00000F552709DF8A01001EB410303EB0111B2
:1032F00000EBC10080F844209DF8B41001EB4100C0
:1033000000EB0110BB4901EB0010C179B748B93897
:1033100080F8AC1000BF00BF0AF019B89DF8B410D7
:1033200001EB4100C0EBC110AF4901EBC000C17817
:103330009DF8B40000EB4002C2EBC010AA4A02EBB9
:10334000C000807841EA002129919DF8B41001EB7A
:103350004100C0EBC110114601EBC001BDF8A40053
:10336000401C095C9DF8B40000EB4002C2EBC010A9
:103370009D4A02EBC002BDF8A400105C41EA0020A7
:10338000C217CDE92E029DF8B41001EB4100C0EB4D
:10339000C110954901EBC0000A90BDF8A410F6F7E2
:1033A0007DFA0022CDE93002DDE93042DDE92E1060
:1033B0006140504001436FD19DF8B41001EB4100D2
:1033C000C0EBC110884901EBC00041782891002171
:1033D00039911CE09DF8B41001EB410000EB0110A5
:1033E000844901EB00113031BDF8E40001EB00101D
:1033F00041789DF8A000814204D1BDF8E400C1B23B
:10340000289112E0BDF8E400401C81B239919DF88A
:10341000B41001EB410000EB0110764901EB001004
:10342000C179BDF8E4008142D4DC00BF9DF8B4103E
:1034300001EB410000EB01106E4901EB0010303050
:103440009DF8A01000EB0110801C0A90007820F07D
:10345000800180310A9801709DF8B41001EB4100A1
:10346000C0EBC110604901EBC00001792691002139
:10347000614A9DF8B40002EB00129DF8A0001154BF
:10348000BDF89800F2287DD007DC05287BD00628FF
:103490000AD0F12878D1FAE3FAE3F32875D0F428BA
:1034A00074D0F628F6D1F4E306211191002136916B
:1034B000F0E3BDF84400401C81B211919DF8B410B6
:1034C00001EB4100C0EBC110474901EBC001BDF861
:1034D0004400095C2691BDF84400401C81B2119162
:1034E000BDF89800F12804D0F2287AD0F32879D1D9
:1034F000FEE39DF8B41001EB4100C0EBC1103A4966
:1035000001EBC001BDF84400095C2991BDF84400FD
:10351000401C81B211919DF8B41001EB410000EB09
:103520000110344901EB001130319DF8A020BDF8A5
:10353000D800104401EB0010407A00F0010030B3D5
:103540009DF8B41040F2991011FB00F0284901EBEE
:10355000C00101F552719DF8A020BDF8D8001044BB
:1035600000EB400202EB001001EBC00090F890006D
:1035700000F0010058B99DF8B41040F2991011FB09
:1035800000F005E0FEE3FEE3FEE3FEE3FEE32AE0F7
:10359000174901EBC00101F552719DF8A020BDF85B
:1035A000D800104400EB400202EB001001EBC00019
:1035B00090F88200B8B1002139913DE09DF8B41037
:1035C00040F2991011FB00F0094901EBC00101F52F
:1035D00052719DF8A020BDF8D800104400EB4002C5
:1035E0000CE0F8E3F6E38AE06486002075330020FF
:1035F000C444002004400020383E002002EB0010AC
:1036000001EBC00000F18301BDF8E4000A5C9DF805
:10361000B40000EB400101EB0010FE4901EB00108B
:103620000E30BDF8E410405C824200D008E0BDF8E6
:10363000E400401C81B23991BDF8E4000428BDDBF0
:1036400000BFBDF8E400042859D1042139912FE0CE
:103650009DF8B41040F2991011FB00F0EE4901EB17
:10366000C00101F552719DF8A020BDF8D8001044AA
:1036700000EB400202EB001001EBC00000F18301FF
:10368000BDF8E4000A5C9DF8B40000EB400101EBDA
:103690000010E04901EB00100E30BDF8E410405C72
:1036A000824200D008E0BDF8E400401C81B23991AC
:1036B000BDF8E4000A28CBDB00BFBDF8E4000A280F
:1036C0001DD09DF8B41040F2991011FB00F0D249C2
:1036D00001EBC00101F552719DF8A020BDF8D800A2
:1036E000104400EB400202EB001001EBC0009030F0
:1036F0000A90007820F00100401C0A990870BDF87B
:10370000A4000F287ED19DF8B41001EB410000EB1E
:103710000110C04901EB001130319DF8A020BDF827
:10372000D800104401EB0010801C0A90007820F0B3
:103730000400001D0A990870002039902DE09DF8C2
:10374000B41001EB4100C0EBC110B44901EBC00162
:10375000BDF84420BDF8E40010440A5C9DF8B400B4
:1037600040F2991110FB01F0AB4901EBC00101F5EA
:1037700052719DF8A030BDF8D800184400EB40030A
:1037800003EB001001EBC0014731BDF8E4000A541F
:10379000BDF8E400401C81B23991BDF8E4000A286C
:1037A000CDDBBDF844000A3081B21191002139917E
:1037B0002FE09DF8B41001EB4100C0EBC110974918
:1037C00001EBC001BDF84420BDF8E40010440A5CE0
:1037D0009DF8B40040F2991110FB01F08E4901EB05
:1037E000C00101F552719DF8A030BDF8D800184411
:1037F00000EB400303EB001001EBC0016031BDF8AA
:10380000E40000E07CE20A54BDF8E400401C81B210
:103810003991BDF8E4000228CBDBBDF84400801CE0
:1038200081B211919DF8B41001EB4100C0EBC110C1
:103830007A4901EBC001BDF84400085C01049DF821
:10384000B40000EB4002C2EBC010744A02EBC002AD
:10385000BDF84400401C105C41EA00219DF8B40012
:1038600000EB4002C2EBC0106C4A02EBC002BDF894
:103870004400801C105C01439DF8B40040F2991292
:1038800010FB02F0644A02EBC00202F552729DF88E
:10389000A030BDF8D800184400EB400303EB001043
:1038A00002EBC0004167BDF84400C01C81B2119119
:1038B0005B4890F89007E8BB0021399120E09DF823
:1038C000B41040F2991011FB00F0534901EBC00114
:1038D00001F552719DF8A020BDF8D800104400EB0E
:1038E000400202EB001001EBC0004730BDF8E410CD
:1038F000405C00B108E0BDF8E400401C81B23991A1
:10390000BDF8E4000A28DADB00BFBDF8E4000A28AD
:103910001BD140229DF8B40040F2991110FB01F038
:103920003D4901EBC00101F552719DF8A030BDF891
:10393000D80000E060E0184400EB400303EB001007
:1039400001EBC00080F87E2069E19DF8B41040F2E0
:10395000991011FB00F0304901EBC00101F55271E3
:103960009DF8A020BDF8D800104400EB400202EB07
:10397000001001EBC00090F87E00E8BB00212A9106
:1039800024E1002137912CE09DF8B41040F2991009
:1039900011FB00F0204901EBC00101F552719DF8C7
:1039A000A020BDF8D800104400EB400202EB00104C
:1039B00001EBC0014731BDF8DC00001D095C9DF83A
:1039C000A80000EB4002174800EB4202BDF8DC0003
:1039D000105C814200D008E0BDF8DC00401C81B2E0
:1039E0003791BDF8DC000628CEDB00BFBDF8DC0057
:1039F00006287CD1032200E011E19DF8B40040F2DA
:103A0000991110FB01F0044901EBC00101F552715D
:103A10000AE0000004400020C44400206486002026
:103A2000BC320020383400209DF8A030BDF8D8000A
:103A3000184400EB400303EB001001EBC00080F8DA
:103A40007E209DF8B41001EB410000EB0110FE490F
:103A500001EB001230329DF8A000BDF8D8100844E8
:103A600002EB0010801C0A90007820F004020A98F3
:103A70000270002039901FE020229DF8B40040F22F
:103A8000991110FB01F0F14901EBC00101F55271F0
:103A90009DF8A030BDF8D800184400EB400303EBBC
:103AA000001001EBC0015131BDF8E4000A54BDF82B
:103AB000E400401C81B23991BDF8E4000F28DBDB43
:103AC0000021399121E020229DF8B40040F29911A3
:103AD00010FB01F0DD4901EBC00101F552719DF8C9
:103AE000A030BDF8D800184400EB400300E068E0C7
:103AF00003EB001001EBC0016331BDF8E4000A5490
:103B0000BDF8E400401C81B23991BDF8E4000A28F8
:103B1000D9DB00229DF8B40040F2991110FB01F0AE
:103B2000CA4901EBC00101F552719DF8A030BDF802
:103B3000D800184400EB400303EB001001EBC00079
:103B400080F87820002139911FE000229DF8B40010
:103B500040F2991110FB01F0BC4901EBC00101F5E5
:103B600052719DF8A030BDF8D800184400EB400316
:103B700003EB001001EBC0017931BDF8E4000A54F9
:103B8000BDF8E400401C81B23991BDF8E40005287D
:103B9000DBDB9DF8B41040F2991011FB00F0AB494B
:103BA00001EBC00101F552719DF8A020BDF8D800CD
:103BB000104400EB400202EB001001EBC000406F2C
:103BC0000CE09DF8A800401CC1B22A91A048B0F8B2
:103BD0007A119DF8A80081423FF7D3AE00BF9C4800
:103BE000B0F87A019DF8A810884218D140229DF8BB
:103BF000B40040F2991110FB01F0944901EBC001AF
:103C000001F552719DF8A030BDF8D800184400EBC2
:103C1000400303EB001001EBC00080F87E209DF80C
:103C2000B41040F2991011FB00F0884901EBC0017B
:103C300001F552719DF8A020BDF8D800104400EBAA
:103C4000400202EB001001EBC00090F87E00032858
:103C500004D011281FD0402851D135E0F2229DF820
:103C6000B40040F2991110FB01F0784901EBC0015A
:103C700001F552719DF8A030BDF8D800184400EB52
:103C8000400303EB001001EBC000427137E028E174
:103C9000F1E3F1E315E1F3229DF8B40040F299114C
:103CA00010FB01F0694901EBC00101F552719DF86B
:103CB000A030BDF8D800184400EB400303EB00101F
:103CC00001EBC00042711AE0F2229DF8B40040F20C
:103CD000991110FB01F05D4901EBC00101F5527132
:103CE0009DF8A030BDF8D800184400EB400300E078
:103CF000C8E003EB001001EBC000427100BF69E0B7
:103D00009DF8B41001EB410000EB01104E4901EBAE
:103D1000001030309DF8A020BDF8D810114400EB01
:103D20000110801C0A90007820F004020A980270AA
:103D30009DF8B41040F2991011FB00F0434901EBDB
:103D4000C00000F552709DF8A020BDF8D8101144B5
:103D500001EB410202EB011100EBC10090F8900071
:103D600000F00100B0B300229DF8B40040F29911B8
:103D700010FB01F0354901EBC00101F552719DF8CE
:103D8000A03004E0FDE3FDE3FDE3FDE3FDE3BDF86A
:103D9000D800184400EB400303EB001001EBC00017
:103DA000A0F88E2005229DF8B40040F2991110FB76
:103DB00001F0264901EBC00101F552719DF8A030D8
:103DC000BDF8D800184400EB400303EB001001EBF2
:103DD000C00042716FE0FFE79DF8B41040F2991007
:103DE00011FB00F0194901EBC00101F552719DF87A
:103DF000A020BDF8D800104400EB400202EB0010F8
:103E000001EBC00090F87E00402819D100229DF8F7
:103E1000B40040F2991110FB01F00C4901EBC00114
:103E200001F552719DF8A030BDF8D800184400EBA0
:103E3000400303EB001001EBC00080F87E2000BFC0
:103E400000BFF12206E0000004400020C44400202E
:103E5000BC3200209DF8B40040F2991110FB01F033
:103E6000FE4901EBC00101F552719DF8A030BDF88B
:103E7000D800184400EB400303EB001001EBC00036
:103E8000427118E0F1229DF8B40040F2991110FB44
:103E900001F0F24901EBC00101F552719DF8A0302B
:103EA000BDF8D800184400EB400303EB001001EB11
:103EB000C000427100BF00BFBDF8D800401C81B2F5
:103EC00036919DF8B41001EB4100C0EBC110E449FC
:103ED00001EBC0004179BDF8D80081423FF7E9AA63
:103EE00051E39DF8B41040F2991011FB00F0DB494A
:103EF00001EBC00000F552709DF8A01001EB4102EB
:103F000002EB011110F8310048BB01229DF8B4000A
:103F100040F2991110FB01F0D04901EBC00101F50D
:103F200052719DF8A00000EB400303EB001001F874
:103F30003020F4229DF8B40040F2991110FB01F0FA
:103F4000C64901EBC00000F552709DF8A01001EBCE
:103F5000410303EB011100EBC1004271CDE09DF87C
:103F6000B41001EB410000EB0110BE4901EB001061
:103F700030309DF8A01000EB0110407A00F00100F5
:103F800080B39DF8B41040F2991011FB00F0B349D2
:103F900001EBC00000F552709DF8A01001EB41024A
:103FA00002EB011100EBC10090F8900000F001005D
:103FB000C0B99DF8B41040F2991011FB00F0A74968
:103FC00001EBC00000F552709DF8A01001EB41021A
:103FD00002EB011100EBC10090F8820010B100214A
:103FE00039912DE089E09DF8B41040F2991011FB51
:103FF00000F09A4901EBC00101F552719DF8A00053
:1040000000EB400202EB001001EBC00000F1830165
:10401000BDF8E4000A5C9DF8B40000EB400101EB40
:104020000010904901EB00100E30BDF8E410405C28
:10403000824200D008E0BDF8E400401C81B2399112
:10404000BDF8E4000428CEDB00BFBDF8E40004287E
:1040500053D1042139912CE09DF8B41040F299100D
:1040600011FB00F07D4901EBC00101F552719DF893
:10407000A00000EB400202EB001001EBC00000F1D9
:104080008301BDF8E4000A5C9DF8B40000EB400138
:1040900001EB0010734901EB00100E30BDF8E41085
:1040A000405C824200D008E0BDF8E400401C81B2D0
:1040B0003991BDF8E4000A28CEDB00BFBDF8E4006A
:1040C0000A281AD09DF8B41040F2991011FB00F0A4
:1040D000624901EBC00000F552709DF8A01001EBA1
:1040E000410202EB011100EBC10090300A90007810
:1040F00020F00100401C0A990870BDF8A4001128A6
:1041000077D19DF8B41001EB410000EB0110554947
:1041100001EB001030309DF8A01000EB0110801C66
:104120000A90007820F00400001D0A990870002011
:10413000399028E09DF8B41001EB4100C0EBC110AC
:10414000474901EBC001BDF8E400401D0A5C9DF841
:10415000B40040F2991110FB01F0404901EBC0019D
:1041600001F552719DF8A00000EB400303EB001035
:1041700001EBC0014731BDF8E4000A54BDF8E4008A
:10418000401C81B23991BDF8E4000A28D2DB00213D
:10419000399128E09DF8B41001EB4100C0EBC1104B
:1041A0002F4901EBC001BDF8E4000F300A5C9DF817
:1041B000B40040F2991110FB01F0284901EBC00155
:1041C00001F552719DF8A00000EB400303EB0010D5
:1041D00001EBC0016031BDF8E4000A54BDF8E40011
:1041E000401C81B23991BDF8E4000228D2DB09E31A
:1041F000FFE7BDF8A40014287ED19DF8B41001EBB0
:10420000410000EB0110174901EB001030309DF820
:10421000A01000EB0110801C0A90007820F0040030
:10422000001D0A9908700020399030E09DF8B41004
:1042300001EB4100C0EBC110094901EBC001BDF821
:10424000E400401D0A5C9DF8B40040F2991110FB97
:1042500001F0024901EBC00106E00000C444002067
:10426000648600200440002001F552719DF8A000F2
:1042700000EB400303EB001001EBC0014731BDF838
:10428000E4000A54BDF8E400401C81B23991BDF845
:10429000E4000A28CADB0021399128E09DF8B41017
:1042A00001EB4100C0EBC110FE4901EBC001BDF8BC
:1042B000E4000F300A5C9DF8B40040F2991110FB45
:1042C00001F0F94901EBC00101F552719DF8A00020
:1042D00000EB400303EB001001EBC0016031BDF8BF
:1042E000E4000A54BDF8E400401C81B23991BDF8E5
:1042F000E4000228D2DB00E02CE29DF8B41001EBD0
:104300004100C0EBC110E74901EBC000407C010453
:104310009DF8B40000EB4002C2EBC010E14A02EB92
:10432000C000807C41EA00219DF8B40000EB40020F
:10433000C2EBC010DB4A02EBC000C07C01439DF819
:10434000B40040F2991210FB02F0D74A02EBC00011
:1043500000F552709DF8A02002EB420303EB02121D
:1043600000EBC2004167D14890F89007F0BB0021F4
:1043700039911DE09DF8B41040F2991011FB00F046
:10438000C94901EBC00101F552719DF8A00000EB95
:10439000400202EB001001EBC0004730BDF8E41012
:1043A000405C00B108E0BDF8E400401C81B23991E6
:1043B000BDF8E4000A28DDDB00BFBDF8E4000A28F0
:1043C00018D140229DF8B40040F2991110FB01F081
:1043D000B54901EBC00000F552709DF8A01001EB4B
:1043E000410303EB011100EBC10000E045E080F860
:1043F0007E2045E19DF8B41040F2991011FB00F0C9
:10440000A94901EBC00000F552709DF8A01001EB26
:10441000410202EB011100EBC10090F87E0060BB8D
:1044200000212A9106E1002137912CE09DF8B4107B
:1044300040F2991011FB00F09B4901EBC00101F51E
:1044400052719DF8A00000EB400202EB001001EB5E
:10445000C0014731BDF8DC00001D095C9DF8A800D3
:1044600000EB4002924800EB4202BDF8DC00105C19
:10447000814203D00BE042E320E201E1BDF8DC0021
:10448000401C81B23791BDF8DC000628CEDB00BFAE
:10449000BDF8DC00062879D103229DF8B40040F273
:1044A000991110FB01F0804901EBC00101F5527137
:1044B0009DF8A00000EB400303EB001001EBC000EF
:1044C00080F87E209DF8B41001EB410000EB011054
:1044D000784901EB001130319DF8A00001EB00108C
:1044E000801C0A90007820F004020A9802700020D4
:1044F00039901CE020229DF8B40040F2991110FB85
:1045000001F0694901EBC00101F552719DF8A0006D
:1045100000EB400303EB001001EBC0015131BDF88B
:10452000E4000A54BDF8E400401C81B23991BDF8A2
:10453000E4000F28DEDB002139911CE020229DF8E9
:10454000B40040F2991110FB01F0574901EBC00192
:1045500001F552719DF8A00000EB400303EB001041
:1045600001EBC0016331BDF8E4000A54BDF8E4007A
:10457000401C81B23991BDF8E4000A28DEDB00223C
:1045800005E040E137E235E282E1C1E14DE09DF82E
:10459000B40040F2991110FB01F0434901EBC00156
:1045A00001F552719DF8A00000EB400303EB0010F1
:1045B00001EBC00080F87820002139911CE0002236
:1045C0009DF8B40040F2991110FB01F0364901EB5F
:1045D000C00101F552719DF8A00000EB400303EB10
:1045E000001001EBC0017931BDF8E4000A54BDF8B8
:1045F000E400401C81B23991BDF8E4000528DEDBFF
:104600009DF8B41040F2991011FB00F0264901EB1F
:10461000C00000F552709DF8A01001EB410202EBC2
:10462000011100EBC100406F0CE09DF8A800401C98
:10463000C1B22A911D48B0F87A019DF8A8108842AD
:104640003FF7F1AE00BF1948B0F87A019DF8A81005
:10465000884215D140229DF8B40040F2991110FB18
:1046600001F0114901EBC00000F552709DF8A01057
:1046700001EB410303EB011100EBC10080F87E2048
:104680009DF8B41040F2991011FB00F0064901EBBF
:10469000C00000F552709DF8A01001EB410202EB42
:1046A000011109E064860020C4440020BC320020CF
:1046B000383400200440002000EBC10090F87E0058
:1046C000032804D0112818D0402842D12BE0F22230
:1046D0009DF8B40040F2991110FB01F0FE4901EB86
:1046E000C00101F552719DF8A00000EB400303EBFF
:1046F000001001EBC00042712BE0F3229DF8B400E2
:1047000040F2991110FB01F0F34901EBC00000F5F4
:1047100052709DF8A01001EB410303EB011100EB77
:10472000C100427115E0F2229DF8B40040F29911E7
:1047300010FB01F0E84901EBC00000F552709DF854
:10474000A01001EB410303EB011100EBC10042712A
:1047500000BF57E09DF8B41001EB410000EB0110E1
:10476000DE4901EB001030309DF8A01000EB011085
:10477000801C0A90007820F004020A9802709DF8CC
:10478000B41040F2991011FB00F0D34901EBC000C6
:1047900000F552709DF8A01001EB410202EB0111EF
:1047A00000EBC10090F8900000F0010050B300222F
:1047B0009DF8B40040F2991110FB01F0C64901EBDD
:1047C000C00101F552719DF8A00000EB400303EB1E
:1047D000001001EBC000A0F88E2005229DF8B40067
:1047E00040F2991110FB01F0BB4901EBC00000F54C
:1047F00052709DF8A01001EB410303EB011100EB97
:10480000C10042717AE19DF8B41040F2991011FB99
:1048100000F0B14901EBC00000F552709DF8A01006
:1048200001EB410202EB011100EBC10090F87E00A8
:10483000402816D100229DF8B40040F2991110FBD7
:1048400001F0A54901EBC00000F552709DF8A010E1
:1048500001EB410303EB011100EBC10080F87E2066
:1048600000BF00BFF1229DF8B40040F2991110FB87
:1048700001F0994901EBC00000F552709DF8A010BD
:1048800001EB410303EB011100EBC100427135E183
:10489000F1229DF8B40040F2991110FB01F08E490D
:1048A00001EBC00000F552709DF8A01001EB410330
:1048B00003EB011100EBC10042711FE103229DF8DF
:1048C000B40040F2991110FB01F0834901EBC001E3
:1048D00001F552719DF8A00000EB400303EB0010BE
:1048E00001F83020F1229DF8B40040F2991110FB3C
:1048F00001F0794901EBC00000F552709DF8A0105D
:1049000001EB410303EB011100EBC1004271F5E043
:1049100002229DF8B40040F2991110FB01F06E499B
:1049200001EBC00101F552719DF8A00000EB4003BE
:1049300003EB001001F83020F6229DF8B40040F29D
:10494000991110FB01F0644901EBC00101F55271AE
:104950009DF8A00000EB400303EB001001EBC0004A
:10496000427101229DF8B40040F2991110FB01F050
:10497000594901EBC00101F552719DF8A00000EB0F
:10498000400303EB001001EBC00080F882200021FF
:10499000399129E09DF8B41001EB4100C0EBC11042
:1049A0004F4901EBC001BDF8E400401D0A5C9DF8D1
:1049B000B40040F2991110FB01F0474901EBC0012E
:1049C00001F552719DF8A00000EB400303EB0010CD
:1049D00001EBC00000F18301BDF8E4000A54BDF80A
:1049E000E400401C81B23991BDF8E4000A28D1DB13
:1049F000BDF8A40082E09DF8B41001EB4100C0EBCB
:104A0000C110374901EBC00081799DF8B40000EB7B
:104A10004002C2EBC010324A02EBC000407941EACA
:104A200000229DF8B40040F2991110FB01F02A49D0
:104A300001EBC00101F552719DF8A00000EB4003AD
:104A400003EB001001EBC000A0F88E209DF8B4101D
:104A500040F2991011FB00F01F4901EBC00101F574
:104A600052719DF8A00000EB400202EB001001EB38
:104A7000C000B0F88E109DF8B40000EB400202EBCD
:104A80000010164A02EB0010408B814235DBF12208
:104A90009DF8B40040F2991110FB01F00E4901EBB2
:104AA000C00101F552719DF8A00000EB400303EB3B
:104AB000001001EBC00042719DF8B41040F2991053
:104AC00011FB00F0044901EBC00101F552719DF8A2
:104AD000A00000EB400205E0C44400200440002098
:104AE0006486002002EB001001EBC00090300A90B9
:104AF000007820F001020A98027000BF00BF08F0A1
:104B000026BC9DF8B41001EB4100C0EBC110FE497A
:104B100001EBC00001792891002136911CE09DF83D
:104B2000B41001EB410000EB0110F84901EB00115A
:104B30003031BDF8D80001EB001041789DF8A0009D
:104B4000814204D1BDF8D800C1B2289112E0BDF86D
:104B5000D800401C81B236919DF8B41001EB4100A1
:104B600000EB0110E94901EB0010C179BDF8D80054
:104B70008142D4DC00BF9DF8B41001EB4100C0EBD2
:104B8000C110E14901EBC000C1782691BDF8980041
:104B9000172834D2DFE800F0330C0F331215181B3E
:104BA0001E33333333333321242733332A2D30005C
:104BB0000720299023E00721299120E0062129914F
:104BC0001DE0062129911AE00620299017E0122104
:104BD000299114E00721299111E0092129910EE082
:104BE000062029900BE00621299108E00B2129914C
:104BF00005E00B21299102E02A21299100BF00BF85
:104C0000BDF8A400001FC1B20A919DF8B41001EBD9
:104C10004100C0EBC110BC4901EBC000C01C0990B1
:104C20000A99F4F757FC37909DF8B41001EB410056
:104C3000C0EBC110B44901EBC001BDF8A400401E97
:104C4000095CBDF8DC0081427DD19DF8B41001EB18
:104C50004100C0EBC110AC4901EBC0004078002816
:104C600071DD9DF8B41001EB4100C0EBC110A64905
:104C700001EBC001BDF8A4000A5C9DF8B40040F24D
:104C8000991110FB01F0A24901EBC00101F552712D
:104C90009DF8A00000EB400303EB001001EBC00007
:104CA00080F8442000219B4A9DF8B40002EB0012DA
:104CB0009DF8A0001154984890F82800012815D1BB
:104CC0009DF8B41001EB410000EB01108F4901EB9E
:104CD000001030309DF8A01000EB0110801C0A90ED
:104CE000007820F0800080300A990870BDF89800A4
:104CF00007287CD00ADC07287AD2DFE810F0790098
:104D00006B06CD06790055061E06CF0C1038072815
:104D1000F2D2DFE810F0320D1C0D6D006D000700BF
:104D20000800F80600BFBDF8980014287DD19DF852
:104D3000B41001EB4100C0EBC110734901EBC0009E
:104D40004079010600E0FDE39DF8B40000EB40026D
:104D5000C2EBC0106C4A02EBC000807941EA00410E
:104D60009DF8B40000EB4002C2EBC010664A02EBB3
:104D7000C000C07941EA00219DF8B40000EB400278
:104D8000C2EBC010604A02EBC000007A01439DF8FC
:104D9000B40040F2991210FB02F05D4A02EBC0022F
:104DA00002F552729DF8A00000EB400303EB0010E7
:104DB00002EBC000C0F81A109DF8B41040F2991030
:104DC00011FB00F0524901EBC00101F552719DF851
:104DD000A00000EB400202EB001001EBC000D0F895
:104DE0001A1008460A91002110F06AFD01E0F3E371
:104DF000F3E3CDE92E019DF8B41001EB410000EB87
:104E00000110424901EB0010007F00F003019DF802
:104E1000B40000EB400202EB00103C4A02EB001031
:104E2000007FC0F30110014400E07EE09DF8B40073
:104E300000EB400202EB0010344A02EB0010007F4E
:104E4000C0F38100091A08460591F3F7D0FBCDE9BC
:104E500006019DED061B9FED310B1FF021F98DED35
:104E6000080B9DED080B51EC100BF3F732FCCDE96C
:104E700030019DF8B41040F2991011FB00F0244964
:104E800001EBC00101F552719DF8A00000EB40025A
:104E900002EB001001EBC000416B084607910021B6
:104EA00010F00EFDDDE92E32A0FB034501FB03519E
:104EB00000FB021502220023DDE93001F3F782F93D
:104EC00020186941CDE90801DDE93023F3F77AF9CB
:104ED000CDE92E01DDE92E0111F0A6FA01469DF87B
:104EE000B40040F2991210FB02F0094A02EBC00034
:104EF00000F552709DF8A02002EB420303EB021272
:104F000000EBC2000EE00000648600200440002098
:104F1000C4440020383E0020BC12002000000000E5
:104F200000002440C0F81E1046E0BDF89800152887
:104F300042D19DF8B41001EB4100C0EBC110FE4915
:104F400001EBC000407901069DF8B40000EB40027F
:104F5000C2EBC010F84A02EBC000807941EA004180
:104F60009DF8B40000EB4002C2EBC010F24A02EB25
:104F7000C000C07941EA00219DF8B40000EB400276
:104F8000C2EBC010EC4A02EBC000007A01439DF86E
:104F9000B40040F2991210FB02F0E84A02EBC000A4
:104FA00000F552709DF8A02002EB420303EB0212C1
:104FB00000EBC200C0F81E109DF8B41001EB4100D8
:104FC000C0EBC110DC4901EBC000427A9DF8B4008F
:104FD00040F2991110FB01F0D84901EBC00101F535
:104FE00052719DF8A00000EB400303EB001001EBB1
:104FF000C00080F894209DF8B41001EB410000EB54
:105000000110CF4901EB001130319DF8A00001EBF8
:105010000010801C0A909DF8B41040F2991011FB0A
:1050200000F0C64901EBC00000F552709DF8A010D9
:1050300001EB410202EB011100EBC10090F894007A
:10504000C2090A98007862F300000A9908709DF876
:10505000B41040F2991011FB00F0B84901EBC00008
:1050600000F552709DF8A01001EB410202EB011116
:1050700000EBC10090F8940000F00300012818D064
:105080009DF8B41040F2991011FB00F0AB4901EB10
:10509000C00000F552709DF8A01001EB410202EB38
:1050A000011100EBC10090F8940000F00300032808
:1050B0002BD19DF8B41001EB410000EB0110A04989
:1050C00001EB001030309DF8A01000EB0110801CA7
:1050D0000A90007820F00200801C0A9908709DF860
:1050E000B41001EB410000EB0110954901EB0010F9
:1050F00030309DF8A01000EB0110801C0A90007861
:1051000020F020020A98027014E09DF8B40000EB31
:10511000400101EB00108A4901EB001030309DF88E
:10512000A01000EB0110801C0A90007820F0020211
:105130000A9802709DF8B40000EB400101EB0010EA
:105140007F4901EB001130319DF8A00001EB001008
:105150008078C0F340029DF8B40040F2991110FB32
:1051600001F0764901EBC00000F552709DF8A010E7
:1051700001EB410303EB011100EBC100007EC0F322
:10518000400082426BD09DF8B40040F2991110FBB0
:1051900001F06A4901EBC00000F552709DF8A010C3
:1051A00001EB410202EB011100EBC10018300A9043
:1051B0009DF8B40000EB400101EB0010604901EBE9
:1051C000001130319DF8A00001EB001080784208FA
:1051D0000A98017862F3410101709DF8B40000EB78
:1051E000400101EB0010564901EB001030309DF8F2
:1051F000A01000EB01108078C0F3400050BB9DF878
:10520000B40000EB400101EB00104D4901EB001030
:1052100030309DF8A01000EB0110801C0A9000783F
:1052200020F020020A98027001229DF8B40040F29A
:10523000991110FB01F0414901EBC00000F55270DB
:105240009DF8A01001EB410303EB011100EBC1003D
:1052500080F846209DF8B4100220F4F7EDFE9DF88A
:10526000B40000EB400101EB0010354901EB0011E7
:1052700030319DF8A00001EB0010807800F00102B1
:105280009DF8B40040F2991110FB01F02B4901EB9D
:10529000C00000F552709DF8A01001EB410303EB34
:1052A000011100EBC100007E00F0010082426DD0D0
:1052B0009DF8B40040F2991110FB01F01F4901EB79
:1052C000C00000F552709DF8A01001EB410202EB06
:1052D000011100EBC10018300A909DF8B40000EBFA
:1052E000400101EB0010164901EB001030309DF831
:1052F000A01000EB011080780A990A7860F3000290
:105300000A709DF8B40000EB400101EB00100C495D
:1053100001EB001030309DF8A01000EB01108078F8
:1053200000F0010098BB9DF8B40000EB400101EBD8
:105330000010034906E0000064860020C4440020F9
:105340000440002001EB001030309DF8A01000EB6D
:105350000110801C0A90007820F020020A98027048
:1053600000229DF8B40040F2991110FB01F0FE49B3
:1053700001EBC00000F552709DF8A01001EB410355
:1053800003EB011100EBC10080F8452014E2FFE7B8
:105390009DF8B40040F2991110FB01F0F24901EBC5
:1053A000C00000F552709DF8A01001EB410202EB25
:1053B000011100EBC10090F84600B0B901229DF840
:1053C000B40040F2991110FB01F0E74901EBC00075
:1053D00000F552709DF8A01001EB410303EB0111A1
:1053E00000EBC10080F845202AE000229DF8B400BF
:1053F00040F2991110FB01F0DB4901EBC00101F50E
:1054000052719DF8A00000EB400303EB001001EB8C
:10541000C00080F845209DF8B40000EB400101EB8E
:105420000010D24901EB001130319DF8A00001EBD2
:105430000010801C0A90007820F001020A98027087
:10544000CB4890F8900780B19DF8B40000EB400184
:1054500001EB0010C54901EB001030309DF8A010A1
:1054600000EB0110807A02286DD1C24890F8290023
:10547000012869D1BF48D0F80C02BE49498D884245
:1054800062D29DF8B40040F2991110FB01F0B649C8
:1054900001EBC00000F552709DF8A01001EB410235
:1054A00002EB011100EBC10090F8450001284AD140
:1054B0009DF8B40040F2991110FB01F0AA4901EBEC
:1054C000C00000F552709DF8A01001EB410202EB04
:1054D000011100EBC10090F87F00A0BB01229DF8F4
:1054E000B40000EB400101EB0010A04901EB0011FA
:1054F00030319DF8A00001EB0010C2729DF8B4009D
:1055000000EB400101EB0010984901EB0011303134
:105510009DF8A00001EB001001789DF8B40040F266
:10552000991210FB02F0904A02EBC0004170052274
:105530009DF8B40040F2991110FB01F08A4901EB8B
:10554000C00102E0FDE300E16AE001F552719DF85F
:10555000A00000EB400303EB001001EBC000427120
:1055600000229DF8B40000EB400101EB00107F49E0
:1055700001EB001130319DF8A00001EB00104260FA
:105580009DF8B4100220F4F757FD002139911CE07A
:1055900000229DF8B40040F2991110FB01F072490D
:1055A00001EBC00101F552719DF8A00000EB400332
:1055B00003EB001001EBC0014731BDF8E4000A54D1
:1055C000BDF8E400401C81B23991BDF8E400142814
:1055D000DEDB002139911EE078E35CE200229DF8D9
:1055E000B40040F2991110FB01F05F4901EBC001DA
:1055F00001F552719DF8A00000EB400303EB001091
:1056000001EBC0016331BDF8E4000A54BDF8E400C9
:10561000401C81B23991BDF8E4000A28DEDBCBE002
:105620009DF8B40040F2991110FB01F04E4901EBD6
:10563000C00000F552709DF8A01001EB410202EB92
:10564000011100EBC10090F8450001287DD19DF8C3
:10565000B40040F2991110FB01F0434901EBC00185
:1056600001F552719DF8A00000EB400202EB001022
:1056700001EBC00090F8800040F2991110FB01F09E
:10568000394901EBC00101F552719DF8B40040F2B7
:10569000991210FB02F0344A02EBC00000F5527080
:1056A0009DF8A02002EB420303EB021200EBC200C4
:1056B00090F8810000EB400202EB001001EBC0000B
:1056C00090F87E00032877D102229DF8B40000EB09
:1056D000400101EB0010254901EB001130319DF82C
:1056E000A00001EB0010C2729DF8B40000EB400175
:1056F00001EB00101D4901EB001130319DF8A000B5
:1057000001EB001001789DF8B40040F2991210FBF3
:1057100002F0154A02EBC00041709DF8B40040F25F
:10572000991110FB01F0114601EBC00101F5527116
:105730009DF8A00000EB400202EB001011F83010C1
:105740009DF8B40040F2991200E035E010FB02F041
:10575000054A02EBC000407981421DD105229DF827
:10576000B40040F2991107E0C44400200440002036
:10577000BC320020BC12002010FB01F0FE4901EBFE
:10578000C00000F552709DF8A01001EB410303EB3F
:10579000011100EBC100427100229DF8B40000EB42
:1057A000400101EB0010F54901EB001030309DF88D
:1057B000A01000EB011042609DF8B40040F2991176
:1057C00010FB01F0EC4901EBC00000F552709DF8B0
:1057D000A01001EB410202EB011110F83100012889
:1057E00014DC02229DF8B40040F2991110FB01F084
:1057F000E14901EBC00000F552709DF8A01001EBEB
:10580000410303EB011100F8312095E09DF8B4004D
:1058100040F2991110FB01F0D74901EBC00000F5EF
:1058200052709DF8A01001EB410202EB011110F83B
:105830003100022834DC00219DF8B40040F29912B6
:1058400010FB02F0CC4A02EBC000017103229DF86C
:10585000B40040F2991110FB01F0C74901EBC001FF
:1058600001F552719DF8A00000EB400303EB00101E
:1058700001F8302007229DF8B40040F2991110FB86
:1058800001F0BD4901EBC00000F552709DF8A01079
:1058900001EB410303EB011100EBC10042714BE04E
:1058A0009DF8B40040F2991110FB01F0B24901EBF0
:1058B000C00101F552719DF8A00000EB400202EB1F
:1058C000001011F830109DF8B40040F2991210FB4E
:1058D00002F0A94A02EBC000407981422CD19DF828
:1058E000B40040F2991110FB01F0114601EBC00029
:1058F00000F552709DF8A01001EB410202EB01117E
:1059000000EBC10090F89400C0F34010A0B1162243
:105910009DF8B40040F2991110FB01F0964901EB9B
:10592000C00000F552709DF8A01001EB410303EB9D
:10593000011100EBC1004271ADE014229DF8B400EA
:1059400040F2991110FB01F08B4901EBC00101F508
:1059500052719DF8A00000EB400303EB001001EB37
:10596000C000427101219DF8B40040F2991210FB71
:1059700002F0814A02EBC00001719DF8B40000EB17
:10598000400101EB00107D4901EB001130319DF821
:10599000A00001EB0010801C0A90007820F020008D
:1059A00020300A99087076E014229DF8B40040F285
:1059B000991110FB01F0704901EBC00000F5527025
:1059C0009DF8A01001EB410303EB011100EBC100B6
:1059D000427160E09DF8B40040F2991110FB01F0B3
:1059E000654901EBC00000F55270BDF8D81001EB1D
:1059F000410202EB011100EBC100807901282AD19C
:105A000000229DF8B40040F2991110FB01F05A49B0
:105A100001EBC00101F55271BDF8D80000EB400365
:105A200003EB001001EBC000827114229DF8B4005A
:105A300040F2991110FB01F04F4901EBC00000F555
:105A400052709DF8A01001EB410303EB011100EB34
:105A5000C10042711FE000219DF8B40040F299128C
:105A600010FB02F0444A02EBC000017105229DF8D0
:105A7000B40040F2991110FB01F03F4901EBC00066
:105A800000F552709DF8A01001EB410303EB0111EA
:105A900000EBC1004271FDE301219DF8B40040F22A
:105AA000991210FB02F0344A02EBC000017114227B
:105AB0009DF8B40040F2991110FB01F02E4901EB62
:105AC000C00101F552719DF8A00000EB400303EB0B
:105AD000001001EBC00042719DF8B40000EB4001E2
:105AE00001EB0010254901EB001130319DF8A000B9
:105AF00001EB0010801C0A90007820F00400001DCB
:105B00000A990870C6E300202E902F900021399149
:105B10001EE0DDE92E10000240EA11620902CDE923
:105B20002E129DF8B40000EB4001C1EBC0101449E7
:105B300001EBC001BDF8E400401D085CDDE92E3436
:105B40001843CDE92E04BDF8E400401C80B2399022
:105B5000BDF8E4000328DCDBDDE92E0110F064FC75
:105B600001469DF8B40040F2991210FB02F0024A7F
:105B700002EBC00206E00000C44400200440002004
:105B80006486002002F552729DF8A00000EB4003ED
:105B900003EB001002EBC000C0F81E1000222E9292
:105BA0002F92002139911EE0DDE92E10000240EA1B
:105BB00011620902CDE92E129DF8B40000EB4001FC
:105BC000C1EBC010FE4901EBC001BDF8E400083094
:105BD000085CDDE92E341843CDE92E04BDF8E4005D
:105BE000401C80B23990BDF8E4000328DCDBDDE91D
:105BF0002E0110F019FC01469DF8B40040F29912F4
:105C000010FB02F0EF4A02EBC00202F552729DF85F
:105C1000A00000EB400303EB001002EBC000C0F853
:105C20001A1000222E922F92002139911FE0DDE9F7
:105C30002E10000240EA11620902CDE92E129DF8F1
:105C4000B40000EB4001C1EBC010DD4901EBC00125
:105C5000BDF8E4001330085CDDE92E3440EA0302AD
:105C6000CDE92E24BDF8E400401C81B23991BDF885
:105C7000E4000328DBDB9DF8B4002E9940F2991272
:105C800010FB02F0CF4A02EBC00202F552729DF8FF
:105C9000A00000EB400303EB001002EBC0004163E7
:105CA00007229DF8B40040F2991110FB01F0C5499C
:105CB00001EBC00000F552709DF8A01001EB41030C
:105CC00003EB011100EBC1004271E3E200202E90D2
:105CD0002F90002139911EE0DDE92E10000240EAEC
:105CE00011620902CDE92E129DF8B40000EB4001CB
:105CF000C1EBC010B24901EBC001BDF8E400401D8A
:105D0000085CDDE92E341843CDE92E04BDF8E4002B
:105D1000401C80B23990BDF8E4000428DCDBDDE9EA
:105D20002E0110F081FB9DF8B42040F2991312FB74
:105D300003F2A44B03EBC20303F552739DF8A020BA
:105D400000E0FCE302EB420404EB021203EBC202AC
:105D500022329060D16000212E912F910020399045
:105D60001EE0DDE92E10000240EA11620902CDE9D1
:105D70002E129DF8B40000EB4001C1EBC010904919
:105D800001EBC001BDF8E4000930085CDDE92E3408
:105D90001843CDE92E04BDF8E400401C80B23990D0
:105DA000BDF8E4000428DCDBDDE92E0110F03CFB4B
:105DB0009DF8B42040F2991312FB03F2814B03EBE0
:105DC000C20303F552739DF8A02002EB420404EBDA
:105DD000021203EBC20242F8220F51609DF8B40098
:105DE00040F2991110FB01F0764901EBC00101F579
:105DF00052719DF8A00000EB400202EB001011F878
:105E000030109DF8B40040F2991210FB02F06D4A78
:105E100002EBC000407981427ED19DF8B40040F28F
:105E2000991110FB01F0114601EBC00000F5527012
:105E30009DF8A01001EB410202EB011100EBC10043
:105E400090F89400C0F34010A8B117229DF8B40058
:105E500040F2991110FB01F05A4901EBC00000F526
:105E600052709DF8A01001EB410303EB011100EB10
:105E7000C100427114E014229DF8B40040F299115F
:105E800010FB01F04F4901EBC00000F552709DF886
:105E9000A01001EB410303EB011100EBC1004271C3
:105EA0009DF8B4009DF8A01001EB0010C217CDE9D9
:105EB0002E02454890F8900708B39DF8B40000EB17
:105EC000400101EB0010414901EB001030309DF81A
:105ED000A01000EB0110807A022810D09DF8B400C9
:105EE00000EB400101EB0010384901EB00103030AD
:105EF0009DF8A01000EB0110C07A00285FDD0022A1
:105F00009DF8B40040F2991110FB01F02D4901EB0E
:105F1000C00101F5527100E037E39DF8A00000EBED
:105F2000400303EB001001EBC00080F846209DF811
:105F3000B40000EB400101EB0010244901EB00111B
:105F400030319DF8A00001EB0010C2722048D0F85B
:105F50000C020521B0FBF1F201FB120000EB400145
:105F60001B482C3000EB41100D300A909DF8B41006
:105F700040F2991011FB00F0124901EBC00000F54E
:105F800052709DF8A02002EB420101EB021100EBE0
:105F9000C10022301022014609900A98F2F755F903
:105FA0000B48D0F80C020521B0FBF1F201FB120006
:105FB00000EB400106482C3000EB41120AE0C7E13B
:105FC00064860020C4440020BC320020044000202D
:105FD000BC1200209DF8B40040F2991110FB01F0B2
:105FE000FE4901EBC00101F552719DF8A00000EBE4
:105FF000400303EB001001EBC00050F81A1F42F8F9
:10600000011F40685060F648D0F80C020521B0FB33
:10601000F1F201FB120000EB4001F1482C3000EBE3
:1060200041129DF8B40000EB400101EB0010ED4976
:1060300001EB001130319DF8A00001EB0010007859
:106040001070E748D0F80C020521B0FBF1F201FB1B
:10605000120000EB4001E2482C3000EB41129DF8A9
:10606000B40040F2991110FB01F0DC4901EBC001D2
:1060700001F552719DF8A00000EB400303EB001006
:1060800001EBC000406BC2F80900D548D0F80C0203
:106090000521B0FBF1F201FB120000EB4001D048FA
:1060A0002C3000EB4111D048026841F81D2F808848
:1060B0008880CB48D0F80C020521B0FBF1F201FB3F
:1060C000120000EB4001C6482C3000EB41129DF855
:1060D000B40000EB400101EB0010C24901EB0011DC
:1060E00030319DF8A00001EB00104068C2F8230099
:1060F00000229DF8B40000EB400101EB0010B9490B
:1061000001EB001130319DF8A00001EB001042605E
:106110000021399154E0B248D0F80C020521B0FBBF
:10612000F1F201FB120000EB4001AD482C3000EB16
:1061300041112731BDF8E4409DF8B40040F29912B6
:1061400010FB02F0A54A02EBC00202F552729DF864
:10615000A00000EB400303EB001002EBC00090F83E
:10616000800040F2991210FB02F09C4A02EBC00240
:1061700002F552729DF8B40040F2991310FB03F03F
:10618000964B03EBC00303F552739DF8A00000EBA0
:10619000400505EB001003EBC00090F8810000EB18
:1061A000400303EB001002EBC0024732BDF8E400ED
:1061B000001D105C0855BDF8E400401C81B2399107
:1061C000BDF8E4000628A6DB0021399142E0002357
:1061D0009DF8B40040F2991110FB01F07F4901EBEA
:1061E000C00101F552719DF8A00000EB400202EBE6
:1061F000001001EBC00090F8800040F2991110FBF4
:1062000001F0764901EBC00101F552719DF8B4002F
:1062100040F2991210FB02F0704A02EBC00202F544
:1062200052729DF8A00000EB400404EB001002EB5A
:10623000C00090F8810000EB400202EB001001EB7F
:10624000C0014731BDF8E4000B54BDF8E400401C28
:1062500081B23991BDF8E4000A28B8DB6048D0F873
:106260000C020521B0FBF1F080B201460A90022039
:10627000F2F72EFF00210620F3F7DEFE5848D0F893
:106280000C025749498D884208D25548D0F80C0273
:10629000401C00E001E25249C1F80C020021052037
:1062A000F3F7CAFE9DF8B41001EB410000EB0110BA
:1062B0004C4901EB001030309DF8A01000EB0110AC
:1062C000801C0A90007820F008020A980270444866
:1062D000D0F80C020521B0FBF1F201FB120000EB3B
:1062E00040013F482C3000EB4110D0F823202E987D
:1062F00000EB40013D4800EB4110C0F82320002096
:10630000399020E03648D0F80C020521B0FBF1F2BC
:1063100001FB120000EB400131482C3000EB411032
:106320002730BDF8E410425C2E9800EB40012F4866
:1063300000EB41112731BDF8E4000A54BDF8E40038
:10634000401C81B23991BDF8E4000628DADB79E01F
:1063500000229DF8B40040F2991110FB01F01F4992
:1063600001EBC00101F552719DF8A00000EB400364
:1063700003EB001001EBC00080F846209DF8B4103C
:1063800001EB410000EB0110164901EB0011303127
:106390009DF8A00001EB0010801C0A90007820F00E
:1063A000080108310A9801709DF8B41001EB410012
:1063B00000EB01100B4901EB001130319DF8A000FA
:1063C00001EB001041682E9800EB4002074800EBFB
:1063D0004210C0F82310002139912FE0C44400205E
:1063E000BC12002004400020C7310020D814002037
:1063F0009DF8B41040F2991011FB00F0FE4901EB3A
:10640000C00101F552719DF8A00000EB400202EBC3
:10641000001001EBC0014731BDF8E4000A5C2E9882
:1064200000EB4001F54800EB41112731BDF8E400D5
:106430000A54BDF8E400401C81B23991BDF8E40073
:106440000628D5DB9DF8B4100220F3F7F5FD9DF882
:10645000B41040F2991011FB00F0E74901EBC000C5
:1064600000F552709DF8A01001EB410202EB011102
:1064700000EBC10022300A902E9800EB4001DF486B
:1064800000EB41100D30102209900A99F1F7DDFE62
:106490009DF8B41040F2991011FB00F0D64901EBC1
:1064A000C00101F552719DF8A00000EB400202EB23
:1064B000001001EBC0012E9800EB4002CF4800EB2A
:1064C000421051F81A2F40F8012F496841609DF899
:1064D000B41001EB410000EB0110C94901EB0011C0
:1064E00030319DF8A00001EB001001782E9800EBF0
:1064F0004002C24800EB421001702E9800EB4001B0
:10650000BE4800EB4111BF48026841F81D2F80884A
:1065100088809DF8B41040F2991011FB00F0B64944
:1065200001EBC00101F552719DF8A00000EB4002A3
:1065300002EB001001EBC000416B2E9800E033E14C
:1065400000EB4002AD4800EB4210C0F809109DF886
:10655000B41001EB410000EB0110A94901EB00115F
:1065600030319DF8A00001EB001041682E9800EB3F
:106570004002A24800EB4210C0F823102E9881B2CE
:1065800008200A91F3F758FD87E09DF8B41040F217
:10659000991011FB00F0984901EBC00101F552710F
:1065A0009DF8A00000EB400202EB001011F8301043
:1065B0009DF8B40040F2991210FB02F08E4A02EBF3
:1065C000C0004079814268DA9DF8B41001EB4100C7
:1065D00000EB01108A4901EB001030309DF8A0104B
:1065E00000EB0110801C0A90007820F00400001DD0
:1065F0000A9908709DF8B41001EB410000EB0110FE
:106600007F4901EB001030309DF8A01000EB011025
:10661000801C0A90007820F0800080300A99087071
:1066200001209DF8B41040F2991211FB02F1724A58
:1066300002EBC10108719DF8B41040F2991011FBF2
:1066400000F0114601EBC00042799DF8B40040F221
:10665000991110FB01F0684901EBC00101F552717D
:106660009DF8A00000EB400303EB001001F8302080
:1066700014229DF8B40040F2991110FB01F05E491C
:1066800001EBC00000F552709DF8A01001EB410332
:1066900003EB011100EBC100427184E00121594874
:1066A000F53080F8B4169DF8B41040F2991011FB43
:1066B00000F0514901EBC00101F552719DF8A000B5
:1066C00000EB400202EB001011F830109DF8B4000E
:1066D00040F2991210FB02F0474A02EBC0004079E9
:1066E000814233DA00219DF8B40040F2991210FB88
:1066F00002F0414A02EBC000017101229DF8B40092
:1067000040F2991110FB01F03B4901EBC00101F58A
:1067100052719DF8A00000EB400303EB001001F85C
:10672000302014229DF8B40040F2991110FB01F0C2
:10673000314901EBC00000F552709DF8A01001EB4B
:10674000410303EB011100EBC10042712BE0142265
:106750009DF8B40040F2991110FB01F0264901EBBD
:10676000C00000F552709DF8A01001EB410303EB4F
:10677000011100EBC100427115E014229DF8B40034
:1067800040F2991110FB01F01B4901EBC00000F52C
:1067900052709DF8A01001EB410303EB011100EBD7
:1067A000C100427100BF00BF06F0D1BD9DF8B4101A
:1067B00040F2991011FB00F00F4901EBC000817805
:1067C00028919DF8B41001EB4100C0EBC1100E49B7
:1067D00011F8301029919DF8B41040F2991011FB76
:1067E00000F0054901EBC00101F552719DF8A000D0
:1067F00000EB40020AE00000C4440020D81400204E
:1068000004400020C73100206486002002EB001005
:1068100001EBC000417926919DF8B41001EB4100D5
:10682000C0EBC110FD4901EBC0010A91BDF8A410F5
:106830000A98F4F799F937909DF8B41001EB4100EC
:10684000C0EBC110F54901EBC001BDF8A400095C23
:10685000BDF8DC00814241F05C879DF8B41001EB8B
:106860004100C0EBC110ED4901EBC00040780028A9
:1068700041F34F870021EA4A9DF8B40002EB001271
:106880009DF8A0001154BDF8980089287ED00FDC37
:10689000142801F01F8705DC082878D0102841F063
:1068A0003787FDE3152801F06D868028F7D1F8E3DE
:1068B0008B286DD08C286CD08E286BD08F28EED191
:1068C000BDF8A4000D2866D19DF8B41001EB41007D
:1068D000C0EBC110D14901EBC0004178D14880F82C
:1068E000041D9DF8B41001EB4100C0EBC110CB4971
:1068F00001EBC000C17ACB4880F8051D9DF8B410AB
:1069000040F2991011FB00F0C74901EBC00000F5FF
:1069100052709DF8A01001EB410202EB011110F83A
:10692000310003287EDCBF4890F8050D00287ADD91
:106930009DF8B41040F2991011FB00F0BA4901EB38
:10694000C00101F552719DF8A00000EB400202EB7E
:10695000001001EBC0010A910878401CC1B20A98EE
:1069600001709DF8B41040F2991011FB00F0AE498F
:1069700001EBC00000F552709DF8A01001EB410240
:1069800002EB011110F83100042805E0FEE3FEE3FC
:10699000FEE3FEE3FEE3FEE345DB9DF8B41001EB0E
:1069A000410000EB0110A14901EB001030309DF8CF
:1069B000A01000EB0110801C0A909A4890F8050D79
:1069C000C0F30010C0F101000A99097860F30001DA
:1069D0000A980170934890F8040DC0F3C000E0BB22
:1069E0009DF8B41001EB410000EB01108F4901EB61
:1069F000001030309DF8A01000EB01108078C0F33B
:106A0000401050B39DF8B41001EB410000EB0110B1
:106A1000864901EB001030309DF8A01000EB01100A
:106A2000801C01E05EE0F8E00A90007820F00200AF
:106A3000801C0A9908709DF8B41040F2991011FB5F
:106A400000F0794901EBC00000F552709DF8A010EC
:106A500001EB410202EB011100E00EE000EBC1008E
:106A600018300A90007820F00200801C0A99087003
:106A70009DF8B4100220F3F7DFFA00219DF8B4006E
:106A800040F2991210FB02F0674A02EBC00001715C
:106A900004229DF8B40040F2991110FB01F0624904
:106AA00001EBC00101F552719DF8A00000EB40031D
:106AB00003EB001001F830208C229DF8B40040F266
:106AC000991110FB01F0584901EBC00000F552701C
:106AD0009DF8A01001EB410303EB011100EBC10095
:106AE00042719AE09DF8B41040F2991011FB00F049
:106AF0004D4901EBC00101F552719DF8A00000EB7A
:106B0000400202EB001011F830109DF8B40040F282
:106B1000991210FB02F0444A02EBC0004079814216
:106B20007BD19DF8B41001EB410000EB01103F490F
:106B300001EB001030309DF8A01000EB0110801C1C
:106B40000A90384890F8050DC0F30010C0F101001C
:106B50000A990A7860F300020A709DF8B41001EBFC
:106B6000410000EB0110314901EB001030309DF87D
:106B7000A01000EB0110801C0A902A4890F8040D28
:106B8000C2080A98007862F341000A9908709DF8DB
:106B9000B41001EB410000EB0110244901EB00109F
:106BA00030309DF8A01000EB01108078C0F3400257
:106BB0009DF8B40040F2991110FB01F01A4901EB65
:106BC000C00000F552709DF8A01001EB410303EBEB
:106BD000011100EBC100007EC0F34000824277D07B
:106BE0009DF8B41040F2991011FB00F00E4901EB32
:106BF000C00000F552709DF8A01001EB410202EBBD
:106C0000011100EBC10018300A909DF8B41001EB9F
:106C1000410000EB011005490AE0CCE36486002046
:106C2000383E0020BC220020C44400200440002044
:106C300001EB001030309DF8A01000EB01108078BF
:106C400042080A98007862F341000A9908709DF89A
:106C5000B41001EB410000EB0110FE4901EB001004
:106C600030309DF8A01000EB01108078C0F3400098
:106C700048BB01229DF8B40040F2991110FB01F0CD
:106C8000F54901EBC00101F552719DF8A00000EB40
:106C9000400303EB001001EBC00042739DF8B40009
:106CA00040F2991110FB01F0EB4901EBC00000F537
:106CB00052709DF8A01001EB410303EB011100EBB2
:106CC000C10080F846209DF8B4100220F3F7B4F913
:106CD0009DF8B41001EB410000EB0110DD4901EB20
:106CE000001130319DF8A00001EB0010807800F019
:106CF00001029DF8B40040F2991110FB01F0D64951
:106D000001EBC00000F552709DF8A01001EB4103AB
:106D100003EB011100EBC100007E00F00100824294
:106D200079D09DF8B41040F2991011FB00F0CA49D7
:106D300001EBC00000F552709DF8A01001EB41027C
:106D400002EB011100EBC10018300A909DF8B4105D
:106D500001EB410000EB0110BE4901EB00103030A7
:106D60009DF8A01000EB011080780A990A7860F372
:106D700000020A709DF8B41001EB410000EB011015
:106D8000B44901EB001030309DF8A01000EB011069
:106D9000807800F00100E8BB9DF8B41001EB4100E1
:106DA00000EB0110AB4901EB001030309DF8A01052
:106DB00000EB01108078C0F3401068B39DF8B41068
:106DC00040F2991011FB00F0A34901EBC00000F55F
:106DD00052709DF8A01001EB410202EB011100EB93
:106DE000C10090F84600B8B99DF8B41040F299106F
:106DF00011FB00F0984901EBC00000F552709DF8BE
:106E0000A01001EB410202EB011100EBC100407B3D
:106E100010B902E054E058E23BE09DF8B41001EBF9
:106E2000410000EB01108B4901EB001030309DF860
:106E3000A01000EB01108078C0F3400048BB012295
:106E40009DF8B40040F2991110FB01F0824901EB6A
:106E5000C00101F552719DF8A00000EB400303EB67
:106E6000001001EBC00042739DF8B40040F299118C
:106E700010FB01F0784901EBC00000F552709DF85D
:106E8000A01001EB410303EB011100EBC10080F8FE
:106E9000462000229DF8B40040F2991110FB01F049
:106EA0006D4901EBC00000F552709DF8A01001EB98
:106EB000410303EB011100EBC10080F84520FFE125
:106EC0009DF8B41040F2991011FB00F0624901EBFB
:106ED000C00000F552709DF8A01001EB410202EBDA
:106EE000011100EBC10090F84600B0B901229DF8F5
:106EF000B40040F2991110FB01F0574901EBC000BA
:106F000000F552709DF8A01001EB410303EB011155
:106F100000EBC10080F845202AE000229DF8B40073
:106F200040F2991110FB01F04B4901EBC00101F552
:106F300052719DF8A00000EB400303EB001001EB41
:106F4000C00080F845209DF8B41001EB410000EB33
:106F50000110404901EB001130319DF8A00001EB18
:106F60000010801C0A90007820F001020A9802703C
:106F70003A4890F8900780B19DF8B41001EB4100B9
:106F800000EB0110334901EB001030309DF8A010E8
:106F900000EB0110807A022865D1314890F8290071
:106FA000012860D12E48D0F80C022D49498D884225
:106FB00059D29DF8B41040F2991011FB00F0264907
:106FC00001EBC00000F552709DF8A01001EB4102EA
:106FD00002EB011100EBC10090F84500012841D1FE
:106FE0009DF8B41040F2991011FB00F01A4901EB22
:106FF000C00000F552709DF8A01001EB410202EBB9
:10700000011100EBC10090F87F0058BB01229DF8F0
:10701000B40000EB400101EB00100E4901EB001140
:1070200030319DF8A00001EB0010C2729DF8B41041
:1070300001EB410000EB0110064901EB001130317A
:107040009DF8A00001EB001001789DF8B40040F21B
:10705000991209E004400020C4440020BC32002002
:10706000BC1200207CE016E110FB02F0FE4A02EBAD
:10707000C000417008229DF8B40040F2991110FB45
:1070800001F0F94901EBC00101F552719DF8A00032
:1070900000EB400303EB001001EBC000427101E084
:1070A00017E3FDE300229DF8B40000EB400101EB83
:1070B0000010EE4901EB001130319DF8A00001EB0A
:1070C000001042609DF8B4100220F2F7B5FF0021D5
:1070D00039911CE000229DF8B40040F2991110FB98
:1070E00001F0E14901EBC00101F552719DF8A000EA
:1070F00000EB400303EB001001EBC0014731BDF88A
:10710000E4000A54BDF8E400401C81B23991BDF896
:10711000E4001428DEDB002039901CE000229DF8FA
:10712000B40040F2991110FB01F0CF4901EBC0010E
:1071300001F552719DF8A00000EB400303EB001035
:1071400001EBC0016331BDF8E4000A54BDF8E4006E
:10715000401C81B23991BDF8E4000A28DEDBAFE0C3
:107160009DF8B40040F2991110FB01F0BE4901EB0B
:10717000C00000F552709DF8A01001EB410202EB37
:10718000011100EBC10090F8450005E0BBE27BE295
:107190001FE38AE3FEE376E201287CD19DF8B40088
:1071A00040F2991110FB01F0AF4901EBC00101F56C
:1071B00052719DF8A00000EB400202EB001001EBC1
:1071C000C00090F8800040F2991110FB01F0A64930
:1071D00001EBC00101F552719DF8B40040F2991223
:1071E00010FB02F0A04A02EBC00000F552709DF8BF
:1071F000A02002EB420303EB021200EBC20090F866
:10720000810000EB400202EB001001EBC00090F89F
:107210007E00032854D102229DF8B40000EB400107
:1072200001EB0010914901EB001130319DF8A000F5
:1072300001EB0010C2729DF8B40000EB400101EBBD
:1072400000108A4901EB001130319DF8A00001EBDC
:10725000001001789DF8B40040F2991210FB02F082
:10726000814A02EBC000417008229DF8B40040F250
:10727000991110FB01F07C4901EBC00101F552713D
:107280009DF8A00000EB400303EB001001EBC000F1
:107290004271002200E013E09DF8B40000EB4001D1
:1072A00001EB0010714901EB001130319DF8A00095
:1072B00001EB001042609DF8B4100220F2F7BCFE12
:1072C0009DF8B4100220F2F7B7FE9DF8B40040F22A
:1072D000991110FB01F0644901EBC00000F55270F8
:1072E0009DF8A01001EB410202EB011100EBC1007F
:1072F0008078802838D19DF8B40000EB400101EB84
:1073000000105A4901EB001030309DF8A01000EB3E
:1073100001108078C0F3400030BB9DF8B40000EB52
:10732000400101EB0010514901EB001030309DF895
:10733000A01000EB01108078C0F34010A0B9152216
:107340009DF8B40040F2991110FB01F0464901EBA1
:10735000C00000F552709DF8A01001EB410303EB53
:10736000011100EBC10042719DF8B40000EB400137
:1073700001EB00103D4901EB001030309DF8A010EA
:1073800000EB01108078C0F34000A8B18F229DF877
:10739000B40040F2991110FB01F0334901EBC00039
:1073A00000F552709DF8A01001EB410303EB0111B1
:1073B00000EBC10042714AE09DF8B40040F299111F
:1073C00010FB01F0284901EBC00000F552709DF858
:1073D000A01001EB410202EB011100EBC100807B28
:1073E000012834D100229DF8B40040F2991110FB1D
:1073F00001F01D4901EBC00101F552719DF8A0009B
:1074000000EB400303EB001001EBC00082738C2201
:107410009DF8B40040F2991110FB01F0124901EB04
:10742000C00101F552719DF8A00000EB400303EB91
:10743000001001EBC000427100219DF8B40040F241
:10744000991210FB02F0084A02EBC00001719DF88E
:10745000B40000EB400101EB0010044901EB001007
:10746000007BE0BB04E00000C44400200440002096
:107470009DF8B40000EB4001C1EBC010F74901EBEF
:10748000C000807801049DF8B40000EB4002C2EB1C
:10749000C010F24A02EBC000C07841EA00219DF81A
:1074A000B40000EB4002C2EBC010EC4A02EBC0009B
:1074B00000790843C117CDE908010EF0B5FF9DF82A
:1074C000B41040F2991211FB02F1E54A02EBC1023D
:1074D00002F552729DF8A01001EB410300E042E07A
:1074E00003EB011102EBC101C1F81E009DF8B410BD
:1074F00001EB4100C0EBC110D84901EBC00040795D
:1075000000049DF8B41001EB4102C2EBC111D34A53
:1075100002EBC101897940EA01209DF8B41001EB2A
:107520004102C2EBC111CD4A02EBC101C979084346
:10753000C117CDE908010EF077FF9DF8B41040F2B5
:10754000991211FB02F1C64A02EBC10101F5527119
:107550009DF8A02002EB420303EB021201EBC201F3
:10756000C1F81A008FE09DF8B40000EB4001C1EBB8
:10757000C010BA4901EBC000807801069DF8B40044
:1075800000EB4002C2EBC010B44A02EBC000C0786E
:1075900041EA00419DF8B40000EB4002C2EBC0108C
:1075A000AE4A02EBC000007941EA00209DF8B41019
:1075B00001EB4102C2EBC111A84A02EBC1014979BA
:1075C0000843C117CDE908010EF02EFF9DF8B41055
:1075D00040F2991211FB02F1A14A02EBC10202F53D
:1075E00052729DF8A01001EB410303EB011102EB75
:1075F000C101C1F81E009DF8B40000EB4001C1EBD1
:10760000C010964901EBC000807900069DF8B410C7
:1076100001EB4102C2EBC111904A02EBC101C979F1
:1076200040EA01409DF8B41001EB4102C2EBC111E8
:107630008A4A02EBC101097A40EA01209DF8B410A0
:1076400001EB4102C2EBC111844A02EBC101497A4C
:107650000843C117CDE908010EF0E6FE9DF8B4100D
:1076600040F2991211FB02F17D4A02EBC10101F5D2
:1076700052719DF8A02002EB420303EB021201EBD2
:10768000C201C1F81A001EE2BDF8A40003281FD1F0
:107690008F229DF8B40040F2991110FB01F070495F
:1076A00001EBC00101F552719DF8A00000EB400311
:1076B00003EB001001EBC000427101219DF8B40002
:1076C00040F2991210FB02F0654A02EBC000017112
:1076D000F9E1BDF8A400032814D18F229DF8B4006D
:1076E00040F2991110FB01F05D4901EBC00101F579
:1076F00052719DF8A00000EB400303EB001001EB7A
:10770000C0004271DFE1BDF8A400032860D19DF8FC
:10771000B40040F2991110FB01F0514901EBC00097
:1077200000F55270BDF8D81001EB410202EB0111D7
:1077300000EBC100807901282AD100229DF8B40015
:1077400040F2991110FB01F0454901EBC00101F530
:107750005271BDF8D80000EB400303EB001001EBC1
:10776000C00082718F229DF8B40040F2991110FB85
:1077700001F03B4901EBC00000F552709DF8A010EC
:1077800001EB410303EB011100EBC10042711FE06B
:1077900008229DF8B40040F2991110FB01F0304925
:1077A00001EBC00101F552719DF8A00000EB400310
:1077B00003EB001001EBC000427100219DF8B40002
:1077C00040F2991210FB02F0254A02EBC000017151
:1077D00079E1BDF8A400032866D19DF8B40040F219
:1077E000991110FB01F01E4901EBC00000F5527029
:1077F000BDF8D81001EB410202EB011100EBC10012
:10780000807901282ED100229DF8B40040F2991110
:1078100010FB01F0124901EBC00101F55271BDF8F6
:10782000D80000EB400303EB001001EBC0008271B5
:107830008F229DF8B40040F2991110FB01F0084925
:1078400001EBC00000F552709DF8A01001EB410360
:1078500003EB011100EBC100427125E064860020BA
:10786000C444002008229DF8B40040F2991110FB96
:1078700001F0FE4901EBC00101F552719DF8A00035
:1078800000EB400303EB001001EBC000427100214C
:107890009DF8B40040F2991210FB02F0F34A00E0A8
:1078A00012E102EBC00001710DE1BDF8A40008284F
:1078B00071D19DF8B40000EB4001C1EBC010EC4960
:1078C00001EBC000807801069DF8B40000EB400297
:1078D000C2EBC010E64A02EBC000C07841EA0041AA
:1078E0009DF8B40000EB4002C2EBC010E04A02EB8E
:1078F000C000007941EA00219DF8B40000EB40028D
:10790000C2EBC010DA4A02EBC00040790843C1174D
:10791000CDE908010EF088FD9DF8B41040F29912EF
:1079200011FB02F1D14A02EBC10202F552729DF83D
:10793000A01001EB410303EB011102EBC10148630D
:107940009DF8B40040F2991110FB01F0C74901EB1A
:10795000C00000F552709DF8A01001EB410202EB4F
:10796000011110F831009DF8B41040F2991211FB8A
:1079700002F1BE4A02EBC1014979884237DA00219F
:107980009DF8B40040F2991210FB02F0B74A02EBE6
:10799000C00001E0D2E096E0017105229DF8B4003C
:1079A00040F2991110FB01F0B04901EBC00101F563
:1079B00052719DF8A00000EB400303EB001001F8AA
:1079C00030208E229DF8B40040F2991110FB01F096
:1079D000A64901EBC00000F552709DF8A01001EB24
:1079E000410303EB011100EBC10042716BE09DF814
:1079F000B40040F2991110FB01F09C4901EBC0006A
:107A000000F55270BDF8D81001EB410202EB0111F4
:107A100000EBC1008079012835D100229DF8B40027
:107A200040F2991110FB01F0904901EBC00101F502
:107A30005271BDF8D80000EB400303EB001001EBDE
:107A4000C00082718F229DF8B40040F2991110FBA2
:107A500001F0864901EBC00101F552719DF8A000CB
:107A600000EB400303EB001001EBC0004271012169
:107A70009DF8B40040F2991210FB02F07B4A02EB31
:107A8000C00001711FE08E229DF8B40040F29911F0
:107A900010FB01F0754901EBC00101F552719DF831
:107AA000A00000EB400303EB001001EBC0004271AB
:107AB00000219DF8B40040F2991210FB02F06B4ACD
:107AC00002EBC0000171EEE3BDF8A400032834D13D
:107AD00000219DF8B40040F2991210FB02F0634AB5
:107AE00002EBC000017101229DF8B40040F299112F
:107AF00010FB01F05D4901EBC00101F55271BDF8C9
:107B0000D80000EB400303EB001001EBC0008271D2
:107B10008C229DF8B40040F2991110FB01F05349FA
:107B200001EBC00000F552709DF8A01001EB41037D
:107B300003EB011100EBC1004271B4E3BDF8A400F6
:107B40000F287DD19DF8B40000EB400101EB00103F
:107B5000484901EB0010007BE8BB00202E902F90DD
:107B6000002139911FE0DDE92E10000240EA116288
:107B70000902CDE92E129DF8B41001EB4100C0EBD3
:107B8000C1103B4901EBC001BDF8E400C0F10600A3
:107B9000085CDDE92E341843CDE92E04BDF8E4007D
:107BA000401C80B23990BDF8E4000528DBDB9DF86D
:107BB000B400DDE92E2140F2991310FB03F02B4BAA
:107BC00003EBC00303F552739DF8A00000EB4004E3
:107BD00004EB001000E04FE003EBC00040F8222F60
:107BE000416000222E922F92002139911FE0DDE9A1
:107BF0002E10000240EA11620902CDE92E129DF812
:107C0000B40000EB4001C1EBC010194901EBC00109
:107C1000BDF8E400C0F10B00085CDDE92E34184328
:107C2000CDE92E04BDF8E400401C80B23990BDF8C7
:107C3000E4000528DBDB9DF8B400DDE92E1200E04E
:107C4000FEE340F2991310FB03F0084B03EBC00076
:107C500000F552709DF8A03003EB430404EB0313CE
:107C600000EBC30022308160C2608AE0C44400207F
:107C7000648600200440002000202E902F900021D8
:107C800039911FE0DDE92E10000240EA116209027D
:107C9000CDE92E129DF8B40000EB4001C1EBC010FD
:107CA000FE4901EBC001BDF8E400C0F10700085C2B
:107CB000DDE92E341843CDE92E04BDF8E400401C64
:107CC00080B23990BDF8E4000628DBDB9DF8B400F3
:107CD000DDE92E1240F2991310FB03F0F04B03EB99
:107CE000C00303F552739DF8A00000EB400404EBC1
:107CF000001003EBC00040F8221F426000222E92C9
:107D00002F920021399120E0DDE92E10000240EA97
:107D100011620902CDE92E129DF8B40000EB40017A
:107D2000C1EBC010DD4901EBC001BDF8E400C0F1BA
:107D30000D00085CDDE92E3440EA0302CDE92E2473
:107D4000BDF8E400401C81B23991BDF8E40006287A
:107D5000DADB9DF8B400DDE92E2140F2991310FB27
:107D600003F0CF4B03EBC00000F552709DF8A0303C
:107D700003EB430404EB031300EBC30022308260E7
:107D8000C1609DF8B40040F2991110FB01F0C449A4
:107D900001EBC00101F552719DF8A00000EB40021B
:107DA00002EB001011F830109DF8B40040F2991267
:107DB00010FB02F0BA4A02EBC000407981427DD14B
:107DC0009DF8B4009DF8A01001EB0010C217CDE99A
:107DD0002E02B44890F8900708B39DF8B40000EB69
:107DE000400101EB0010B04901EB001030309DF86C
:107DF000A01000EB0110807A022810D09DF8B4008A
:107E000000EB400101EB0010A74901EB00103030FE
:107E10009DF8A01000EB0110C07A00287DDD002243
:107E20009DF8B40000EB400101EB00109E4901EB0E
:107E3000001030309DF8A01000EB0110C2729B487A
:107E4000D0F80C020521B0FBF1F201FB120000EBAF
:107E5000400196482C3000EB41100D300A909DF8FF
:107E6000B41040F2991011FB00F08D4901EBC000F5
:107E700000F552709DF8A01001EB410202EB0111D8
:107E800000EBC10022301022014609900A98F0F759
:107E9000DCF98648D0F80C020521B0FBF1F201FBB9
:107EA000120000EB400181482C3000EB41129DF89C
:107EB000B40040F2991110FB01F000E0ECE27849C7
:107EC00001EBC00101F552719DF8A00000EB4003E9
:107ED00003EB001001EBC00050F81A1F42F8011F1D
:107EE000406850607148D0F80C020521B0FBF1F2F7
:107EF00001FB120000EB40016C482C3000EB4112FA
:107F00009DF8B40000EB400101EB0010664901EB65
:107F1000001130319DF8A00000E094E101EB001069
:107F2000007810706148D0F80C020521B0FBF1F226
:107F300001FB120000EB40015C482C3000EB4111CA
:107F40005848F538026841F81D2F808888805748C6
:107F5000D0F80C020521B0FBF1F201FB120000EB9E
:107F6000400152482C3000EB41129DF8B40040F221
:107F7000991110FB01F14A4800EBC10101F5527162
:107F80009DF8A00000EB400303EB001001EBC000E4
:107F9000406BC2F809004548D0F80C020521B0FB3F
:107FA000F1F201FB120000EB400140482C3000EBE5
:107FB00041129DF8B40000EB400101EB00103A497A
:107FC00001EB001130319DF8A00001EB001040687A
:107FD000C2F8230000229DF8B40000EB400101EB41
:107FE0000010314901EB001130319DF8A00001EB88
:107FF00000104260002139915FE02C48D0F80C025B
:108000000521B0FBF1F201FB120000EB4001274813
:108010002C3000EB41112731BDF8E4409DF8B4004D
:1080200040F2991210FB02F01D4A02EBC00202F569
:1080300052729DF8A00000EB400303EB001002EB2E
:10804000C00090F8800040F2991210FB02F0144A30
:1080500002EBC00202F552729DF8B40040F299138F
:1080600010FB03F00E4B03EBC00303F552739DF8B6
:10807000A00000EB400505EB001003EBC00090F8FA
:10808000810000EB400303EB001002EBC00247321B
:10809000BDF8E400001D105C085509E0648600206E
:1080A000C4440020BC32002004400020BC12002048
:1080B000BDF8E400401C81B23991BDF8E400062807
:1080C0009BDB0020399042E000239DF8B40040F291
:1080D000991110FB01F0FE4901EBC00101F552714D
:1080E0009DF8A00000EB400202EB001001EBC00085
:1080F00090F8800040F2991110FB01F0F44901EB77
:10810000C00101F552719DF8B40040F2991210FBC4
:1081100002F0EF4A02EBC00202F552729DF8A00095
:1081200000EB400404EB001002EBC00090F881006B
:1081300000EB400202EB001001EBC0014731BDF83B
:10814000E4000B54BDF8E400401C81B23991BDF845
:10815000E4000A28B8DBDF48D0F80C020521B0FBA8
:10816000F1F080B201460A900220F0F7B1FF002141
:108170000620F1F761FFD748D0F80C02D549498DA8
:10818000884206D2D348D0F80C02401CD149C1F82D
:108190000C0200210520F1F74FFF9DF8B40000EB21
:1081A000400101EB0010CC4901EB001030309DF88C
:1081B000A01000EB0110801C0A90007820F008024B
:1081C0000A980270C348D0F80C020521B0FBF1F206
:1081D00001FB120000EB4001BE482C3000EB4110C7
:1081E000D0F823202E9800EB4001BC4800EB411052
:1081F000C0F823200020399020E0B648D0F80C02C7
:108200000521B0FBF1F201FB120000EB4001B14887
:108210002C3000EB41102730BDF8E410425C2E9862
:1082200000EB4001AD4800EB41112731BDF8E400FF
:108230000A54BDF8E400401C81B23991BDF8E40055
:108240000628DADB5AE09DF8B41001EB410000EBA0
:108250000110A14901EB001030309DF8A01000EB97
:108260000110801C0A90007820F0080008300A995C
:1082700008709DF8B41001EB410000EB0110964925
:1082800001EB001130319DF8A00001EB00104168B6
:108290002E9800EB4002914800EB4210C0F82310EA
:1082A0000021399126E014E29DF8B41040F29910B3
:1082B00011FB00F0864901EBC00101F552719DF8F8
:1082C000A00000EB400202EB001001EBC0014731BF
:1082D000BDF8E4000A5C2E9800EB40017F4800EBFB
:1082E00041112731BDF8E4000A54BDF8E400401CF8
:1082F00081B23991BDF8E4000628D5DB9DF8B410B1
:1083000001EB410000EB0110734901EB001030302C
:108310009DF8A01000EB0110801C0A90007820F05E
:1083200020020A9802709DF8B4100220F1F784FE32
:108330009DF8B41040F2991011FB00F0644901EB74
:10834000C00000F552709DF8A01001EB410202EB55
:10835000011100EBC10022300A902E9800EB400181
:108360005E4800EB41100D30102209900A99EFF79A
:108370006CFF9DF8B41040F2991011FB00F05449C5
:1083800001EBC00101F552719DF8A00000EB400225
:1083900002EB001001EBC0012E9800EB40024F48A9
:1083A00000EB421051F81A2F40F8012F4968416044
:1083B0009DF8B41001EB410000EB0110464901EBC0
:1083C000001130319DF8A00001EB001001782E98CB
:1083D00000EB4002414800EB421001702E9800EB88
:1083E00040013E4800EB41113D48026841F81D2F15
:1083F000808888809DF8B41040F2991011FB00F03D
:10840000334901EBC00101F552719DF8A00000EB6A
:10841000400202EB001001EBC000416B2E9800EB14
:1084200040022E4800EB4210C0F809109DF8B4102D
:1084300001EB410000EB0110274901EB001100E0C6
:108440009FE030319DF8A00001EB001041682E98AC
:1084500000EB4002214800EB4210C0F823102E9898
:1084600081B208200A91F1F7E7FD00229DF8B400DF
:1084700040F2991110FB01F0154901EBC00000F525
:1084800052709DF8A01001EB410303EB011100EBCA
:10849000C10080F846205FE09DF8B41001EB410078
:1084A00000EB01100C4901EB001030309DF8A010DA
:1084B00000EB0110801C0A90007820F00400001DE1
:1084C0000A9908709DF8B41001EB41000AE0000021
:1084D000C4440020BC12002004400020D814002016
:1084E000C731002000EB0110FE4901EB00103030D5
:1084F0009DF8A01000EB0110801C0A90007820F07D
:10850000800080300A99087001209DF8B41040F274
:10851000991211FB02F1F44A02EBC10108719DF8B6
:10852000B41040F2991011FB00F0114601EBC000AD
:1085300042799DF8B40040F2991110FB01F0EA492C
:1085400001EBC00000F552709DF8A01001EB410353
:1085500003EB011100F831208F229DF8B40040F2A6
:10856000991110FB01F0E04901EBC00000F55270D9
:108570009DF8A01001EB410303EB011100EBC100DA
:108580004271C5E0BDF8A400032856D10121D748A7
:1085900080F8B4169DF8B41040F2991011FB00F069
:1085A000D14901EBC00101F552719DF8A00000EB2B
:1085B000400202EB001011F830109DF8B40040F2B8
:1085C000991210FB02F0C84A02EBC00040798142C8
:1085D00034DA00219DF8B40040F2991210FB02F049
:1085E000C14A02EBC000017101229DF8B40040F2C3
:1085F000991110FB01F0BC4901EBC00101F552716A
:108600009DF8A00000EB400303EB001001F83020C0
:108610008F229DF8B40040F2991110FB01F0B2498D
:1086200001EBC00000F552709DF8A01001EB410372
:1086300003EB011100EBC10042714AE09DF8B41058
:1086400040F2991011FB00F0A74901EBC00000F5C2
:1086500052709DF8A01001EB410202EB011100EBFA
:10866000C1008078802834D100219DF8B40040F208
:10867000991210FB02F09C4A02EBC00001718022AB
:108680009DF8B40040F2991110FB01F0964901EBFE
:10869000C00101F552719DF8A00000EB400303EB0F
:1086A000001001EBC000427100229DF8B40040F2BE
:1086B000991110FB01F08C4901EBC00000F55270DC
:1086C0009DF8A01001EB410303EB011100EBC10089
:1086D00082701DE0BDF8A400032818D10021834852
:1086E00080F8B4168F229DF8B40040F2991110FB67
:1086F00001F07D4901EBC00000F552709DF8A0101B
:1087000001EB410303EB011100EBC100427100BF1B
:1087100000BF04F01CBE9DF8B41001EB4100C0EB9B
:10872000C110734911F83000042802D104212691A8
:108730000CE09DF8B41001EB4100C0EBC1106C4996
:1087400011F83000152801D1152126919DF8B4109B
:1087500001EB4100C0EBC110654901EBC00041785D
:108760009DF8B40000EB4002C2EBC010604A12F862
:10877000300041EA002041F23001884202D1A621B6
:1087800026913DE09DF8B41001EB4100C0EBC11013
:10879000574901EBC00041789DF8B40000EB40025E
:1087A000C2EBC010524A12F8300041EA002041F2F8
:1087B0003101884202D1A721269121E09DF8B41011
:1087C00001EB4100C0EBC110494911F8300002280B
:1087D00016D19DF8B41001EB4100C0EBC110444923
:1087E00001EBC00001799DF8B40000EB4002C2EB40
:1087F000C0103F4A02EBC000C07841EA0021269138
:108800009DF8B41040F2991011FB00F0364901EBCD
:10881000C000C17827919DF8B41040F2991011FB67
:1088200000F0314901EBC00108319DF89C0000EBDC
:10883000800202EBC00001EB800082789DF8B4005A
:1088400040F2991110FB01F0274901EBC0010831FA
:108850009DF89C0000EB800303EBC00001EB80005F
:10886000C0781044C1B228910021224A9DF8B4007A
:1088700002EB00129DF89C00115439914AE09DF8DA
:10888000B41040F2991011FB00F0174901EBC00140
:1088900008319DF89C0000EB800202EBC00001EB68
:1088A000800002799DF8B40040F2991110FB01F0AC
:1088B0000D4901EBC00108319DF89C0000EB8003DD
:1088C00003EBC00001EB80008178BDF8E4000844B0
:1088D00000EB400101EB00119DF8B40040F2991348
:1088E0000AE0000004400020C4440020BC32002004
:1088F00064860020383E002010FB03F0FE4B03EBA3
:10890000C00000F5527000F83120BDF8E400401CB2
:1089100081B239919DF8B41040F2991011FB00F02A
:10892000F54901EBC00108319DF89C0000EB800285
:1089300002EBC00011F82010BDF8E40081429EDC7B
:10894000BDF8981043F23002881A91427ED009DCBB
:1089500004297CD015297BD0A62910D0A72942F064
:10896000468565E1B0F5C06F73D0A0F201600028C4
:1089700070D001286FD00428F1D102F05AB800213C
:108980009DF8B40040F2991210FB02F0DA4A02EBB3
:10899000C00001719DF8B41040F2991011FB00F075
:1089A000114601EBC00008309DF89C1001EB8102DC
:1089B00002EBC10100EB81000079052828DC0622CA
:1089C0009DF8B40040F2991110FB01F0CA4901EB87
:1089D000C00108319DF89C0000EB800303EBC00050
:1089E00001EB80000271A8229DF8B40040F29911B9
:1089F00010FB01F0C04901EBC00008309DF89C104D
:108A000001EB810303EBC10100EB810042710DE139
:108A10009DF8B41040F2991011FB00F0B64901EB3B
:108A2000C00008309DF89C1001EB810202EBC101EF
:108A300000EB810000790A282FDC0B229DF8B4009E
:108A400040F2991110FB01F0AB4905E0BAE137E2C1
:108A5000FDE3FDE3FDE3FDE301EBC00108319DF81B
:108A60009C0000EB800303EBC00001EB800002716F
:108A7000A9229DF8B40040F2991110FB01F09E4923
:108A800001EBC00008309DF89C1001EB810303EB63
:108A9000C10100EB81004271C8E09DF8B41040F2C2
:108AA000991011FB00F0944901EBC00008309DF8CB
:108AB0009C1001EB810202EBC10100EB8100007907
:108AC0000F2828DC10229DF8B40040F2991110FB09
:108AD00001F0894901EBC00108319DF89C0000EBD1
:108AE000800303EBC00001EB80000271A2229DF81D
:108AF000B40040F2991110FB01F07F4901EBC00076
:108B000008309DF89C1001EB810303EBC10100EBE1
:108B1000810042718AE09DF8B41040F2991011FB77
:108B200000F0754901EBC00008309DF89C1001EB86
:108B3000810202EBC10100EB81004079A52826D11A
:108B40009DF8B41040F2991011FB00F06A4901EB56
:108B5000C00108319DF89C0000EB800202EBC000D0
:108B600001EB8000C1789DF8B40000EB400202EBFD
:108B70000010624A02EB0010303000EB0110801C44
:108B80000A90007820F00400001D0A9908709DF8F2
:108B9000B41040F2991011FB00F0574901EBC000EE
:108BA00008309DF89C1001EB810202EBC10100EB43
:108BB00081008079A12839D09DF8B41040F2991035
:108BC00011FB00F04C4901EBC00108319DF89C00FD
:108BD00000EB800202EBC00001EB800082799DF87F
:108BE000B40040F2991110FB01F0434901EBC001C0
:108BF00008319DF89C0000EB800303EBC00001EB03
:108C000080004271A1229DF8B40040F2991110FB3E
:108C100001F0394901EBC00008309DF89C1001EBD0
:108C2000810303EBC10100EB8100827102F0DFBB25
:108C300000219DF8B40040F2991210FB02F02E4A78
:108C400002EBC00001719DF8B41040F2991011FBC5
:108C500000F0114601EBC00008309DF89C1001EBBC
:108C6000810202EBC10100EB8100007908281FDCC2
:108C700000219DF8B40040F2991210FB02F01E4A48
:108C800002EBC000017108229DF8B40040F2991176
:108C900010FB01F0184901EBC00008309DF89C1052
:108CA00001EB810303EBC10100EB810002712EE0B7
:108CB0009DF8B41040F2991011FB00F00E4901EB41
:108CC000C00008309DF89C1001EB810202EBC1014D
:108CD00000EB810000790B2819DC0C229DF8B40010
:108CE00040F2991110FB01F0034901EBC00008307C
:108CF0009DF89C1004E00000C444002004400020C3
:108D000001EB810303EBC10100EB810002719DF8CF
:108D1000B41040F2991011FB00F0F84901EBC000CB
:108D200008309DF89C1001EB810202EBC10100EBC1
:108D300081004079A42830D19DF8B41001EB4100A6
:108D400000EB0110EE4901EB001030309DF8A0104F
:108D500000EB0110801C0A90007820F020012031E7
:108D60000A98017000229DF8B40040F2991110FB9E
:108D700001F0E24901EBC00101F552719DF8A0003C
:108D800000EB400303EB001001EBC00080F845202E
:108D90009DF8B4100220F1F74FF9A1229DF8B4001C
:108DA00040F2991110FB01F0D44901EBC0000830EA
:108DB0009DF89C1001EB810303EBC10100EB8100E6
:108DC000427133E70021399115E09DF8B41001EBB1
:108DD0004100C0EBC110CB4901EBC001BDF8E4007C
:108DE000C01C095C17AABDF8E4001154BDF8E400EA
:108DF000401C81B23991BDF8E4000628E5DB06216C
:108E000017A81CF0F1FA0021CDE93001DDE930218D
:108E1000100A40EA0160309C001941EB21214FF417
:108E200080724FF00003CDE90801EFF7CBF99DF810
:108E3000B40040F2991110FB01F0B04901EBC00001
:108E400000F552709DF89C1001EB410303EB0111FA
:108E500000EBC100027100209DF8B41040F299129D
:108E600011FB02F1A54A02EBC101087104229DF831
:108E7000B40040F2991110FB01F0A04901EBC000D1
:108E800000F552709DF89C1001EB410303EB0111BA
:108E900000F83120A7229DF8B40040F2991110FB90
:108EA00001F0964901EBC00000F552709DF89C104E
:108EB00001EB410303EB011100EBC1004271B5E688
:108EC0009DF8B41040F2991011FB00F08B4901EBB2
:108ED000C00008309DF89C1001EB810202EBC1013B
:108EE00000EB81000079042876DA00219DF8B400B7
:108EF00040F2991210FB02F0804A02EBC0000171AF
:108F0000A1229DF8B40040F2991110FB01F07B49B9
:108F100001EBC00108319DF89C0000EB800303EBDE
:108F2000C00001EB800042719DF8B41040F299102E
:108F300011FB00F0714901EBC00108319DF89C0064
:108F400000EB800202EBC00001EB8000001D0A90E4
:108F50000078401CC2B20A9802709DF8B41040F22A
:108F6000991011FB00F0654901EBC00008309DF835
:108F70009C1001EB810202EBC10100EB8100007942
:108F8000042827D10A229DF8B40040F2991110FB61
:108F900001F05A4901EBC00108319DF89C0000EB3B
:108FA000800303EBC00001EB80000271A3229DF857
:108FB000B40040F2991110FB01F0504901EBC000E0
:108FC00008309DF89C1001EB810303EBC10100EB1D
:108FD0008100427120E3FFE79DF8B41040F2991040
:108FE00011FB00F0454901EBC00008309DF89C10D2
:108FF00001EB810202EBC10100EB81000079042842
:1090000033D100219DF8B40040F2991210FB02F018
:109010003A4A02EBC000017105229DF8B40040F20B
:10902000991110FB01F0354901EBC00108319DF8A1
:109030009C0000EB800303EBC00001EB8000027199
:10904000A3229DF8B40040F2991110FB01F02B49C6
:1090500001EBC00008309DF89C1001EB810303EB8D
:10906000C10100EB81004271D6E29DF8B41040F2DC
:10907000991011FB00F0214901EBC00008309DF868
:109080009C1001EB810202EBC10100EB8100007931
:10909000082839DC00219DF8B40040F2991210FB39
:1090A00002F0164A02EBC000017109229DF8B400DB
:1090B00040F2991110FB01F0104901EBC001083199
:1090C0009DF89C0000EB800303EBC00001EB8000E7
:1090D0000271A7229DF8B40040F2991110FB01F033
:1090E000064901EBC00108319DF89C0000EB8003AC
:1090F00003EBC00001EB800042718DE2C44400200C
:1091000004400020648600209DF8B41040F29910BD
:1091100011FB00F0FA4901EBC00008309DF89C10EB
:1091200001EB810202EBC10100EB8100007909280B
:1091300033DC00219DF8B40040F2991210FB02F0DC
:10914000EF4A02EBC00001710A229DF8B40040F220
:10915000991110FB01F0EA4901EBC00108319DF8BB
:109160009C0000EB800303EBC00001EB8000027168
:10917000A3229DF8B40040F2991110FB01F0E049E0
:1091800001EBC00008309DF89C1001EB810303EB5C
:10919000C10100EB810042713EE29DF8B41040F243
:1091A000991011FB00F0D64901EBC00008309DF882
:1091B0009C1001EB810202EBC10100EB8100007900
:1091C0000D2833DC00219DF8B40040F2991210FB09
:1091D00002F0CB4A02EBC00001710E229DF8B400F0
:1091E00040F2991110FB01F0C54901EBC0010831B3
:1091F0009DF89C0000EB800303EBC00001EB8000B6
:109200000271A1229DF8B40040F2991110FB01F007
:10921000BB4901EBC00008309DF89C1001EB8103B5
:1092200003EBC10100EB81004271F5E19DF8B41040
:1092300040F2991011FB00F0B14901EBC000083079
:109240009DF89C1001EB810202EBC10103E0E4E117
:1092500016E269E248E200EB810000790E2833DC77
:1092600000219DF8B40040F2991210FB02F0A44ACC
:1092700002EBC00001710F229DF8B40040F2991179
:1092800010FB01F09E4901EBC00108319DF89C00E4
:1092900000EB800303EBC00001EB80000271A3220E
:1092A0009DF8B40040F2991110FB01F0944901EBD4
:1092B000C00008309DF89C1001EB810303EBC10155
:1092C00000EB81004271A7E19DF8B41040F29910C3
:1092D00011FB00F08A4901EBC00008309DF89C109A
:1092E00001EB810202EBC10100EB81000079102843
:1092F0007EDC11229DF8B40040F2991110FB01F0C0
:109300007F4901EBC00108319DF89C0000EB800310
:1093100003EBC00001EB80000271A1229DF8B400B4
:1093200040F2991110FB01F0754901EBC0010831C1
:109330009DF89C0000EB800303EBC00001EB800074
:1093400042719DF8B40040F2991110FB01F06C4994
:1093500001EBC00108319DF89C0000EB800303EB9A
:10936000C00001EB80008271002139915AE09DF824
:10937000B41040F2991011FB00F0614901EBC001FB
:1093800008319DF89C0000EB800202EBC00001EB6D
:1093900080008178BDF8E40001449DF8B40000EB42
:1093A000400202EB0010574A02EB0010303000EB95
:1093B0000110801C0A90007820F0800180310A980A
:1093C00001709DF8B41040F2991011FB00F04C4967
:1093D00001EBC00108319DF89C0000EB800202EB1C
:1093E000C00001EB80008178BDF8E400014400E09A
:1093F0008AE09DF8B40000EB400202EB0010414A05
:1094000002EB0010303000EB0110801C0A90007855
:1094100020F00400001D0A990870BDF8E400401C0B
:1094200080B239909DF8B41040F2991011FB00F011
:10943000334901EBC00108319DF89C0000EB80022C
:1094400002EBC00011F82010BDF8E40081428EDC70
:109450009DF8B41001EB410000EB0110294901EB2C
:10946000001030309DF8A01000EB01108078C0F3A0
:109470004010E8B39DF8B41001EB410000EB01107F
:10948000204901EB001030309DF8A01000EB0110D6
:10949000801C0A90007820F020020A9802709DF843
:1094A000B41001EB410000EB0110164901EB001074
:1094B00030309DF8A01000EB01108078C0F3400020
:1094C000A8B99DF8B41001EB410000EB01100D4963
:1094D00001EB001030309DF8A01000EB0110801C53
:1094E0000A90007820F0080008300A99087000E01F
:1094F00072E09DF8B4100220F0F79EFD8CE00000B1
:10950000C4440020044000209DF8B41040F299109B
:1095100011FB00F0FD4901EBC00108319DF89C00F2
:1095200000EB800202EBC00001EB800001799DF8A6
:10953000B40040F2991210FB02F0F44A02EBC000B2
:109540004079814268D19DF8B41040F2991011FB26
:1095500000F0114601EBC00008309DF89C1001EBB3
:10956000810202EBC10100EB81008079A12834D097
:10957000A3229DF8B40040F2991110FB01F0E349D9
:1095800001EBC00108319DF89C0000EB800303EB68
:10959000C00001EB800042719DF8B41040F29910B8
:1095A00011FB00F0D94901EBC00008309DF89C1078
:1095B00001EB810202EBC10100EB81008079A2285E
:1095C0002AD000219DF8B40040F2991210FB02F05D
:1095D000CE4A02EBC00001711EE0A1229DF8B4004A
:1095E00040F2991110FB01F0C84901EBC0010831AC
:1095F0009DF89C0000EB800303EBC00001EB8000B2
:10960000427101219DF8B40040F2991210FB02F062
:10961000BE4A02EBC000017151E4A1229DF8B400E2
:1096200040F2991110FB01F0B84901EBC00108317B
:109630009DF89C0000EB800303EBC00001EB800071
:1096400082719DF8B40040F2991110FB01F0AF490E
:1096500001EBC00108319DF89C0000EB800303EB97
:10966000C00001EB8000427100219DF8B40040F27F
:10967000991210FB02F0A54A02EBC00001711EE432
:1096800000219DF8B40040F2991210FB02F09F4AAD
:1096900002EBC000017109229DF8B40040F299115B
:1096A00010FB01F0994901EBC00108319DF89C00C5
:1096B00000EB800303EBC00001EB80000271A722E6
:1096C0009DF8B40040F2991110FB01F08F4901EBB5
:1096D000C00008309DF89C1001EB810303EBC10131
:1096E00000EB8100427197E700219DF8B40040F241
:1096F000991210FB02F0854A02EBC0000171A7220B
:109700009DF8B40040F2991110FB01F07F4901EB84
:10971000C00008309DF89C1001EB810303EBC101F0
:1097200000EB8100427177E79DF8B41040F2991088
:1097300011FB00F0754901EBC00108319DF89C0058
:1097400000EB800202EBC00001EB800081789DF805
:10975000B40000EB4002C2EBC0106D4A02EBC00047
:10976000C07D0844313881B236919DF8B41040F282
:10977000991011FB00F0654901EBC00108319DF81B
:109780009C0000EB800202EBC00011F820109DF855
:10979000B40000EB4002C2EBC0105D4A02EBC00017
:1097A000C07D313881427DDD9DF8B41001EB410070
:1097B000C0EBC110114601EBC000C07D3138C2B210
:1097C0009DF8B40040F2991110FB01F04F4901EBF4
:1097D000C00108319DF89C0000EB800303EBC00042
:1097E00001EB8000C27000219DF8B40040F2991294
:1097F00010FB02F0454A02EBC0000171A7229DF860
:10980000B40040F2991110FB01F0404901EBC00196
:1098100008319DF89C0000EB800303EBC00001EBD6
:10982000800042719DF8B41001EB4100C0EBC11003
:10983000374901EBC000407930286DD19DF8B41054
:1098400040F2991011FB00F0304901EBC0010831E2
:109850009DF89C0000EB800202EBC00001EB800051
:1098600001799DF8B40040F2991210FB02F0274AEA
:1098700002EBC000407981424ED19DF8B41040F215
:10988000991011FB00F0114601EBC00000F5527079
:10989000BDF8D81001EB410202EB011100EBC10051
:1098A000C07800E0FEE3312837D19DF8B41001EB19
:1098B000410000EB0110174901EB00103030BDF8FA
:1098C000D81000EB0110801C0A90007820F02002D4
:1098D0000A98027000229DF8B40040F2991110FB22
:1098E00001F00A4901EBC00101F55271BDF8D80041
:1098F00000EB400303EB001001EBC00080F84520B3
:109900009DF8B4100220F0F797FB5BE0C444002000
:1099100064860020044000207FE09DF8B41040F2EF
:10992000991011FB00F0FE4901EBC00000F55270E8
:10993000BDF8D81001EB410202EB011100EBC100B0
:10994000C07833283ED19DF8B41001EB410000EB04
:109950000110F44901EB00103030BDF8D81000EBD5
:109960000110801C0A90007820F020020A980270F2
:1099700001229DF8B40040F2991110FB01F0E84972
:1099800001EBC00000F55270BDF8D81001EB4103A7
:1099900003EB011100EBC10080F84620A9229DF8DD
:1099A000B40040F2991110FB01F0DD4901EBC00059
:1099B00008309DF89C1001EB810303EBC10100EB23
:1099C000810082719DF8B41001EB410000EB0110A1
:1099D000D44901EB00103030BDF8D81000EB011075
:1099E000801C0A90007820F001020A9802709DF80D
:1099F000B41001EB410000EB0110CA4901EB00106B
:109A00003030BDF8D81000EB0110801C0A900078AF
:109A100020F002020A98027011E19DF8B41001EBE7
:109A20004100C0EBC110C04901EBC00040793128B2
:109A30007ED19DF8B41040F2991011FB00F0B849A6
:109A400001EBC00108319DF89C0000EB800202EBA5
:109A5000C00001EB800001799DF8B40040F299123A
:109A600010FB02F0AE4A02EBC000407981425FD1A8
:109A70009DF8B41040F2991011FB00F0114601EB73
:109A8000C00000F55270BDF8D81001EB410202EBA6
:109A9000011100EBC10090F8460058BB01229DF86F
:109AA000B40040F2991110FB01F09D4901EBC00197
:109AB00001F55271BDF8D80000EB400303EB001034
:109AC00001EBC00080F845209DF8B41001EB410087
:109AD00000EB0110934901EB00113031BDF8D800C3
:109AE00001EB0010801C0A90007820F00100401C5F
:109AF0000A9908709DF8B41001EB410000EB0110C9
:109B0000884901EB00103030BDF8D81000EB01108F
:109B1000801C0A90007820F002020A9802708348A4
:109B200090F8900790B19DF8B41001EB410000E06F
:109B30000EE200EB01107B4901EB00103030BDF864
:109B4000D81000EB0110807A022878D1784890F87C
:109B50002900012873D17648D0F80C027449498D48
:109B600088426CD29DF8B41040F2991011FB00F0BD
:109B70006B4901EBC00000F55270BDF8D81001EB45
:109B8000410202EB011100EBC10090F845000128F1
:109B900054D19DF8B41040F2991011FB00F06049C7
:109BA00001EBC00000F55270BDF8D81001EB410286
:109BB00002EB011100EBC10090F87F00F0BB012225
:109BC0009DF8B40000EB400101EB0010554901EB9A
:109BD00000113031BDF8D80001EB0010C272002234
:109BE0009DF8B40000EB400101EB00104D4901EB82
:109BF00000113031BDF8D80001EB001042609DF833
